:100000000C942B0E0C9404630C945C0E0C945C0EFC
:100010000C945C0E0C94493B0C946D9A0C945C0E01
:100020000C945C0E0C945C0E0C945C0E0C945C0EA8
:100030000C945C0E0C945C0E0C945C0E0C945C0E98
:100040000C945C0E0C94DF560C94868C0C945C0E15
:100050000C945C0E0C945C0E0C945C0E0C949493BB
:100060000C945C0E0C945F5F0C94365F0C945C0EE9
:100070000C945C0E0C945C0E0C945C0E0C945C0E58
:100080000C94F1840C945C0E0C945C0E0C945C0E3D
:100090000C940D5F0C94E45E0C945C0E0C945C0E5E
:1000A0000C945C0E0C945C0E0C945C0E0C945C0E28
:1000B0000C945C0E0C9429750C945C0E0C945C0EE4
:1000C0000C945C0E0C945C0E0C945C0E0C94BB5E59
:1000D0000C94925E0C945C0E0C94695E0C94405EE1
:1000E0000C945C0E211B241B2B1B2E1B311B341B61
:1000F0003B1B421B451B4C1B531B5A1B1521432109
:100100007A21B1218C22C322F1221F23E623E62388
:10011000E623E623E623E623E623E623E623E62397
:10012000E623E623E623E623E623E623E623E62387
:10013000E623E623E623E623E623E623E623E62377
:10014000E623E623E623E8211F2257224D237B23C3
:10015000B323E425EA25F025F625FC25022608260A
:100160000E2614261A262026262638263E26442623
:100170005C26622668266E2674267A2680268626C7
:100180008C26922698269E26A426AA26B626C22625
:10019000C826CE26D426EC26F226F826FE260427EC
:1001A0000A27FA270028062818281E282428362877
:1001B0003C28422848284E2854286C2872289C281D
:1001C000A228A828AE28C628CC28D228D8286D294D
:1001D0006D296D296D296D296D296D296D29EE28EF
:1001E000F228F628FC280029042908290C291029BE
:1001F00014291A2938293E294429DA2610271627D6
:100200001C27222728272E27B428BA28C028DE2812
:10021000E428EA284A29502956295A2860283427F0
:100220003A27402746274C2752270C282A28BC2645
:100230002C263226E026E6265C2962296829B0268B
:1002400078287E2884288A289028962858275E2790
:1002500064276A27702776277C27822788278E279E
:1002600094279A27A027A627AC27B227B827BE270E
:10027000CA27D027D627DC27E227E827EE27F4274E
:100280002C29262920293229122830284A265026AE
:1002900056266628C42748302530FE2F6530BC30EE
:1002A0008430B330A2306D3150312931BD318A31C3
:1002B0008A31AC319531513851386B3851387838F2
:1002C0009138AC38C7388442B842ED420D434243BE
:1002D000AA43BA43E4442E4438446C44A144AF4496
:1002E000E444764353496A4981499849AF49DD4915
:1002F000F4490B4A224A414A594A704A8F4AA54A50
:10030000C649395B3C5B2B5B2F5B355B735B405BAA
:10031000445B4A5B4E5B525B585B5C5B605B735B50
:10032000665B6A5B6E5BC960CE60D360DD60E76070
:100330006061F160F96001610B6115611F612E61FF
:100340003861606142614C615661587561756975CB
:100350007D758F75A175AC7505A84CCDB2D44EB91D
:100360003836A9020C50B9918688083CA6AAAA2A58
:10037000BE000000803F3400330032004E6F6E65D7
:100380000053746F70706564004E65757472616CB3
:10039000205475726E004D6F76696E6720526576D7
:1003A00065727365004D6F76696E6720466F727770
:1003B000617264004272616B696E670054414E4B1A
:1003C00020524553544F5245440025004865616C06
:1003D0007468204C6576656C3A2000564548494360
:1003E0004C452052455041495220434F4D504C45B9
:1003F00054450054414E4B2044455354524F5945A7
:10040000440025004865616C7468204C6576656C15
:100410003A2000290056454849434C452052455052
:1004200041495220535441525445442028005245DA
:1004300050414952204F5045524154494F4E20435C
:10044000414E43454C4C45440029004D41434849E9
:100450004E452047554E20484954212028005245FA
:1004600050414952204F5045524154494F4E20432C
:10047000414E43454C4C454400290043414E4E4FAC
:100480004E2048495421202800547572726574200A
:10049000726F746174696F6E206973206E6F74205F
:1004A0006F66207479706520536572766F2E204ECA
:1004B0006F20736574757020617661696C61626C20
:1004C000652E004E6F207374656572696E672073C8
:1004D0006572766F2061737369676E65642C207234
:1004E000652D636865636B2076656869636C65205C
:1004F000747970652E0054757272657420656C6530
:10050000766174696F6E206973206E6F74206F66F8
:10051000207479706520536572766F2E204E6F209F
:10052000736574757020617661696C61626C652EAB
:1005300000546F70204C65667400546F70204365E2
:100540006E74657200546F70205269676874004D54
:100550006964646C65204C656674004D6964646C04
:10056000652043656E746572004D6964646C652036
:10057000526967687400426F74746F6D204C6566D1
:100580007400426F74746F6D2043656E7465720001
:10059000426F74746F6D20526967687400464952E7
:1005A0004D574152452056455253494F4E3A20002F
:1005B0006942757300534275730050504D004E6F81
:1005C0006E6520446574656374656400417A696D85
:1005D0007574682020202000456C65766174696F11
:1005E0006E2020005475726E2020202020202000D4
:1005F0005468726F74746C652020200053746963B2
:100600006B202020202020204D696E2020202043B8
:10061000656E7465722020204D6178202020204472
:1006200065616462616E64202052657665727365EF
:100630006400524144494F20494E464F202D20002E
:100640004E4F542044455445435445440049474E79
:100650004F52454400416E616C6F670044696769A1
:1006600074616C00417578204368616E2E202020F3
:100670004D696E20202020204D61782020202020F0
:1006800054797065004368616E6E656C7320757493
:10069000696C697A65643A20004368616E6E656CC6
:1006A000732064657465637465643A20002028448F
:1006B000697361626C656429002028456E61626C13
:1006C000656429004D656368616E6963616C2072C1
:1006D00065636F696C00416972736F6674004D6584
:1006E0006368616E6963616C2042617272656C3A25
:1006F000200020284D31290020284D3229002028B3
:1007000042290042617272656C20456C65766174A5
:10071000696F6E3A20200020284D30290020284D96
:1007200031290020284129005475727265742052C5
:100730006F746174696F6E3A2020200020416D70E3
:10074000732900202843757272656E74204C696DA0
:1007500069743A20004472697665204D6F746F7237
:10076000733A202020202020004D4F544F52205417
:10077000595045530054616E6B202854616D69795E
:100780006120444D44290054616E6B2028444B4C39
:100790004D2047656172626F78290043617200489D
:1007A000616C66747261636B0054616E6B00554ED0
:1007B0004B4E4F574E00596573004E6F0029002570
:1007C0002C20446563656C65726174696F6E206688
:1007D0006163746F72200020284B69636B626163F0
:1007E0006B2073706565642000547261636B2052E6
:1007F00065636F696C20456E61626C65643A2020A8
:1008000020004E2F4120666F722076656869636C08
:10081000652074797065005475726E204D6F646543
:100820003A202020202020202020202020202000CE
:100830004E2F4120666F722076656869636C652073
:100840007479706500596573202854616D69796108
:1008500029002500202D20004E65757472616C20E2
:100860005475726E20416C6C6F7765643A2020205D
:100870000020736563005472616E736D69737369F0
:100880006F6E2044656C61793A2020202020002082
:1008900073656300456E67696E65205061757365A9
:1008A0002054696D653A20202020202000207365A7
:1008B000630053686966742054696D653A2020208E
:1008C00020202020202020202020004175746F6DE2
:1008D00061746963004D616E75616C005472616E84
:1008E000736D697373696F6E20547970653A202057
:1008F00020202020002500596573202D20005265FE
:100900007665727365205370656564204C696D6906
:100910007465643A2020002500596573202D20005D
:10092000466F7277617264205370656564204C690C
:100930006D697465643A202000206D7329002520BC
:100940007468726F74746C6520666F722000202862
:10095000004D6F746F72204E7564676520456E613F
:10096000626C65643A202020200029004E6F6E657D
:10097000004E6F6E65002C205072657365743A20CE
:10098000002900202841646A757374656420746FBF
:10099000200020284C6576656C3A2000446563652C
:1009A0006C2052616D7020456E61626C65643A2006
:1009B000202020200029004E6F6E65004E6F6E656E
:1009C000002C205072657365743A2000290020289D
:1009D00041646A757374656420746F200020284C2C
:1009E0006576656C3A2000416363656C2052616DE9
:1009F0007020456E61626C65643A202020202000E2
:100A00004163746976652044726976696E67205027
:100A1000726F66696C653A200056656869636C653B
:100A200020547970653A202020202020202020208A
:100A3000200044524956452053455454494E47538B
:100A40000020736563005265636F696C2064656C98
:100A500061793A20202020202020202020202020E2
:100A6000202020202020002500596573202D200003
:100A700042617272656C20456C65766174696F6E57
:100A8000205370656564204C696D697465643A2013
:100A9000002500596573202D20005475727265740D
:100AA00020526F746174696F6E20537065656420A5
:100AB0004C696D697465643A202000545552524562
:100AC000542053455454494E475300556E6B6E6F36
:100AD000776E004578706572696D656E74616C0043
:100AE00053657061726174652048656174202620C9
:100AF00046616E00436F6D62696E65642048656192
:100B00007420262046616E00250044697361626C82
:100B1000656400536D6F6B65207768656E20646552
:100B20007374726F7965643A200046616E206D615E
:100B3000782073706565643A2020202020202020D2
:100B40000046616E20666173742069646C65207371
:100B5000706565643A20200046616E2069646C65AA
:100B60002073706565643A2020202020202000201A
:100B70007365636F6E6473004E2F41005072652D74
:100B8000686561742064656C61793A2020202020BA
:100B9000202000536D6F6B657220547970653A2088
:100BA00020202020202020202000536D6F6B6572B4
:100BB000206F757470757420636F6E74726F6C6CD7
:100BC0006564206D616E75616C6C7900534D4F4B9F
:100BD000455200556E6B6E6F776E00486561767991
:100BE000004D656469756D004C69676874004375F4
:100BF00073746F6D00556E6B6E6F776E004E6F6E17
:100C000065004F70656E2050616E7A6572005461A8
:100C10006D6979612053706563002073656320728C
:100C200065636F766572792900207365632072654C
:100C30006C6F61642C2000204D4720686974732C10
:100C400020002063616E6E6F6E20686974732C20C3
:100C500000280057656967687420436C6173733AB4
:100C600020202020200044616D6167652050726F54
:100C700066696C653A202020005965732028004180
:100C80006363657074204D472044616D6167653A08
:100C9000200059657320280053656E64204D47205D
:100CA000495220436F64653A2020004E2F41005284
:100CB000657061697265642062793A202020202085
:100CC00020004E2F41004869742050726F746F638A
:100CD0006F6C20323A2020200029002028546561C2
:100CE0006D2000466972652050726F746F636F6C7F
:100CF0003A2020202000466972652050726F746F80
:100D0000636F6C3A20202020004973205265706187
:100D100069722054616E6B3F2020200049522026CA
:100D20002054616E6B20426174746C696E6720445C
:100D3000697361626C656400424154544C452049BA
:100D40004E464F00554E4B4E4F574E0042656E6516
:100D500064696E6920544253204D6963726F00428A
:100D6000656965722055534D2D52432D32005461F3
:100D70006967656E20536F756E642043617264000D
:100D80004F70656E2050616E7A657220536F756E7C
:100D90006420436172640042656E6564696E692017
:100DA000544253204D696E6900536F756E64206321
:100DB0006172643A2000534F554E442043415244DF
:100DC00000556E6B6E6F776E0042617272656C20BB
:100DD000456C65766174696F6E20436F6D6D616EF1
:100DE000640054757272657420526F746174696F17
:100DF0006E20436F6D6D616E64005374656572693A
:100E00006E6720436F6D6D616E640056656869633F
:100E10006C6520537065656400456E67696E65207A
:100E20005370656564005468726F74746C65204318
:100E30006F6D6D616E6400537065656420646563F9
:100E40007265617365732062656C6F772000537003
:100E500065656420696E63726561736573206162A4
:100E60006F766520005475726E2053746F707065D4
:100E700064004C656674205475726E205374617200
:100E8000746564005269676874205475726E2053EB
:100E90007461727465640056656869636C6520539B
:100EA000746F70706564004D6F76696E672052656F
:100EB0007665727365004D6F76696E6720466F7256
:100EC0007761726400456E67696E652053746F7058
:100ED00000456E67696E65205374617274004361EA
:100EE0006E6E6F6E2052656C6F616465640056654E
:100EF0006869636C652044657374726F796564001A
:100F000043616E6E6F6E20486974004272616B655A
:100F100073204170706C696564005661726961622A
:100F20006C6500290020286F662000506F73200038
:100F3000417578204368616E6E656C200056617261
:100F40006961626C65004F6E004F66660042004149
:100F50000045787465726E616C20496E70757420FE
:100F600000070809090B0C0C0B0C0C547572726508
:100F70007420537469636B202D200046756E637472
:100F8000696F6E202300202D3E20002073656300D2
:100F9000547572726574206D6F76656D656E742020
:100FA00064656C61793A2020004E6F6E650059656A
:100FB000730054757272657420737469636B206674
:100FC000756E6374696F6E733A200046554E4354D4
:100FD000494F4E20545249474745525300762063AB
:100FE00075746F666629002028004C564320456EB4
:100FF00061626C65643A2020202020200076005633
:101000006F6C746167653A2020202020202020200A
:101010002000596573004E6F0042617474657279E7
:101020002044657465637465643A200042415454F9
:101030004552590053657269616C20332054782001
:10104000426175643A2020004175782053657269C9
:10105000616C20426175643A202020004D6F746FEE
:10106000722053657269616C20426175643A200098
:101070005553422053657269616C20426175643A30
:101080002020200042415544205241544553002124
:101090002000464143544F52592052455345542154
:1010A00020003A200042697420004761703A200015
:1010B000416972736F6674202D20456E61626C65A4
:1010C00064004D656368616E6963616C205265639D
:1010D0006F696C202D20456E61626C65640041690A
:1010E00072736F6674202D2044697361626C65644D
:1010F000004D656368616E6963616C205265636F62
:10110000696C202D2044697361626C656400436FD3
:101110006D6D73206368616E67656420746F205520
:10112000534200436F6D6D73206368616E67656441
:1011300020746F2053657269616C203100447269BC
:1011400076696E672050726F66696C65207365748E
:1011500020746F202300250053706565642072653C
:10116000647563656420746F200053706565642046
:10117000726573746F726564005475726E20456E8B
:1011800067696E65204F6E00207365636F6E6473D0
:1011900000536D6F6B6572207072652D68656174A8
:1011A0002073746172746564202D20656E67696EAA
:1011B000652077696C6C207475726E206F6E206983
:1011C0006E20004D616E75616C207472616E736D7E
:1011D000697373696F6E202D2070757420696E209D
:1011E0006E65757472616C206765617220626566F8
:1011F0006F7265207374617274696E6720656E67C3
:10120000696E6521005475726E20456E67696E6562
:10121000204F666600456E67696E65204175746F84
:101220002053687574646F776E00456E67616765FB
:10123000205472616E736D697373696F6E004469D7
:1012400073656E67616765205472616E736D697353
:1012500073696F6E00536574205475726E204D6F04
:1012600064653A203100536574205475726E204DC8
:101270006F64653A203200536574205475726E2095
:101280004D6F64653A203300456E61626C65204E97
:1012900065757472616C205475726E730044697365
:1012A00061626C65204E65757472616C2054757254
:1012B0006E7300494F20506F72742041204F757437
:1012C000707574202D204F6E00494F20506F72743E
:1012D0002041204F7574707574202D204F66660074
:1012E000401F7017D007A00FA00FDC05D007C4095E
:1012F00010278813983A102758026C0258026C0283
:1013000058026C0258026C0258026C0258026C02BD
:1013100058026C0258026C025802B0366C023A0253
:101320006C023A026C023A026C02B036384A5C1225
:101330001C255C125C121C255C12BC7FC7F2C078B5
:1013400087A5B7C5A00F8813B80B401FB80BB80B03
:101350007017401F00002100240027002A002D00E4
:101360003000330001010000040107010A01000000
:101370002200250028002B002E003100340002013D
:101380000000050108010B010000200023002600D9
:1013900029002C002F00320000010000030106018B
:1013A00009010505050507050808080802020202EB
:1013B0000A0A0808040404040101010101010101F1
:1013C0000303030303030303040707070C0C0C0CBC
:1013D0000C0C0C0C020202020606060606060606A5
:1013E0000B0B0B0B0B0B0B0B010210202008081032
:1013F0002040102040800201020108040201010285
:10140000040810204080804020100804020180045D
:1014100002018040201008040201080402010102B8
:1014200004081020408001020408102040800000C1
:101430000A0B02090C0D0E0807030401000000004E
:10144000000000000000000000000000000000009C
:101450000000000000000000000012111000000059
:10146000000000000000000000000000000000007C
:1014700000000000524144494F204641494C53412D
:10148000464500526164696F205265616479202D80
:10149000200052657665727365643A2020004D61C4
:1014A000782050756C73653A20004D696E20507538
:1014B0006C73653A2000456E642056616C756573E7
:1014C00000456E64205265636F696C2053657276C7
:1014D0006F20536574757000456E6420526F74619F
:1014E00074696F6E20536572766F205365747570E2
:1014F00000456E6420456C65766174696F6E20539B
:101500006572766F20536574757000536572766FDF
:1015100020756E2D72657665727365640053657211
:10152000766F2072657665727365640052657665C4
:10153000727365643A2020004D61782050756C7399
:10154000653A20004D696E2050756C73653A200035
:1015500053746172742056616C75657300494E5600
:10156000414C494420534552564F2E204E4F205354
:10157000455455502E005365747570205265636F45
:10158000696C20536572766F0053657475702054D2
:10159000757272657420526F746174696F6E205039
:1015A000616E20536572766F0053657475702053B9
:1015B00074656572696E6720536572766F20284F77
:1015C00075747075742032290053657475702053DA
:1015D00074656572696E6720536572766F20284F57
:1015E00075747075742034290053657475702054B7
:1015F000757272657420456C65766174696F6E20D2
:10160000536572766F00494F20506F7274204220EC
:101610004F7574707574202D204F6E00494F205007
:101620006F72742042204F7574707574202D204F96
:101630006666004C56432045786974202D20566F0D
:101640006C7461676520526573746F7265640076AF
:1016500029004C5643207468726573686F6C64206F
:1016600072656163686564212028004C696768744D
:101670002031204F6E004C696768742031204F661E
:1016800066004C696768742032204F6E004C6967B1
:1016900068742032204F666600326E64204D472009
:1016A00053746F7000326E64204D47205374617222
:1016B000740052756E6E696E67204C69676874734A
:1016C000204F6E0052756E6E696E67204C696768B8
:1016D0007473204F666600417578204F757470757D
:1016E00074204F6E00417578204F757470757420AA
:1016F0004F66660053746F70205265766F6C766922
:101700006E6720417578204C696768740053746F68
:101710007020417578204F757470757420426C6923
:101720006E6B696E6700417578204F7574707574C3
:10173000205072657365742044696D005374617242
:101740007420417578204F757470757420426C69EF
:101750006E6B696E6700466F7277617264204765D1
:101760006172004E65757472616C2047656172002C
:1017700052657665727365204765617200536574C2
:1017800020416363656C2052616D70204C65766505
:101790006C3A200053657420446563656C20526187
:1017A0006D70204C6576656C3A2000416E616C6FFF
:1017B0006720557365722046756E6374696F6E207D
:1017C00031202D2000416E616C6F6720557365726A
:1017D0002046756E6374696F6E2032202D20002DB7
:1017E00000202D20002000545255450046414C5306
:1017F0004500250057616974696E6720666F722025
:10180000726164696F2E2E2E2000537461727420F1
:101810005265766F6C76696E6720417578204C69E9
:101820006768740054616967656E2056322F5633BD
:1018300000536F6E790052435441204D61636869D3
:101840006E652047756E00436C61726B204D61635D
:1018500068696E652047756E005243544120526599
:101860007061697200494255205265706169720069
:10187000436C61726B20526570616972004F7065D4
:101880006E50616E7A657200567354616E6B0046DD
:101890004F560054616967656E2056310048656E89
:1018A00067204C6F6E670054616D69796120312F3C
:1018B00033350054616D69796120322D53686F743E
:1018C0000054616D69796100556E6B6E6F776E00C3
:1018D000556E6B6E6F776E00446574616368656406
:1018E0002F4E41005265636F696C20536572766FAD
:1018F0000050616E20536572766F00536572766F8B
:101900002F455343004F6E626F617264204D6F74B8
:101910006F7220447269766572004F70656E205058
:10192000616E7A65722053636F75742053657269B6
:10193000616C20455343005361626572746F6F742C
:10194000682053657269616C00506F6C6F6C752014
:1019500053657269616C00536572766F2031005374
:101960006572766F203200536572766F20330053B4
:101970006572766F203400536572766F20350053A0
:101980006572766F203600536572766F203700538C
:101990006572766F20380053657420766F6C756DB4
:1019A000653A2000202D20537461727420526570B6
:1019B000656174696E6700202D2053746F70005547
:1019C00073657220536F756E64200041202D2000D6
:1019D00042202D2000536F756E642042616E6B2093
:1019E00000506C61792F53746F7000506C617920D6
:1019F00052616E646F6D00506C6179205072657633
:101A0000696F757300506C6179204E6578740020A1
:101A10002877697468204952290046697265204315
:101A2000616E6E6F6E004669726520526570616905
:101A300072205369676E616C00416972736F6674DE
:101A4000202D204D616E75616C2054726967676549
:101A500072004D656368616E6963616C20526563F5
:101A60006F696C202D204D616E75616C2054726918
:101A70006767657200536572766F205265636F69A0
:101A80006C202D204D616E75616C20547269676702
:101A90006572004869676820496E74656E73697481
:101AA0007920466C61736820556E6974202D204D35
:101AB000616E75616C2054726967676572004D478D
:101AC000205374617274004D472053746F70004945
:101AD00052204E4F5420656E61626C6564202D204B
:101AE0006E6F2049522070726F746F636F6C732039
:101AF00073656C65637465642E00556E61626C6518
:101B000020746F20656E61626C65204952004952F5
:101B100020656E61626C656400495220646973617E
:101B2000626C656400417578204F7574707574201F
:101B3000466C617368656400417578204F757470F8
:101B4000757420496E766572736520466C617368A2
:101B500065640053746F7020417578204F75747000
:101B6000757420426C696E6B696E670053746F7098
:101B7000205265766F6C76696E6720417578204CCF
:101B8000696768740053746F7020416C6C205573E2
:101B9000657220536F756E647300494F20506F72E9
:101BA000742041202D2050756C73656400494F20CE
:101BB000506F72742041202D205374617274204242
:101BC0006C696E6B696E6700494F20506F727420AC
:101BD00042202D2050756C73656400494F20506F72
:101BE00072742042202D20537461727420426C69FB
:101BF0006E6B696E6700557365722046756E63740F
:101C0000696F6E203100557365722046756E63747E
:101C1000696F6E203200536D6F6B657220656E6167
:101C2000626C656400536D6F6B65722064697361EB
:101C3000626C6564004865617420416D743A2000EF
:101C4000486561743A200053616D652061732066B8
:101C5000616E00002EB111241FBECFEFD1E2DEBFB6
:101C6000CDBF00E00CBF16E0A0E0B2E0E7E6F8EA86
:101C700001E00BBF02C007900D92AE32B107D9F759
:101C800023E1AEE2B6E001C01D92A03DB207E1F74C
:101C90001EE0CBE2DEE000E006C021970109802FC4
:101CA000FE010E94ADC0CA32D10780E00807A9F743
:101CB0000E94009F0C9400C30C9400002F923F924E
:101CC0004F925F926F927F928F929F92AF92BF924C
:101CD000CF92DF92EF92FF920F931F93CF93DF93F8
:101CE000CDB7DEB7E6970FB6F894DEBF0FBECDBF17
:101CF0008091D1069091D2060E941D5E0E94F17FD4
:101D00006DE975E08091D1069091D2060E94BF5C8A
:101D100068EF75E0CE0101960E94805C8091D1064B
:101D20009091D206DC01ED91FC914D815E8169813B
:101D30007A810280F381E02D199560E076E0809150
:101D4000D1069091D2060E94E35C2AE040EE51E079
:101D500060E070E08091D1069091D2060E94F85C1C
:101D600060E176E08091D1069091D2060E94205EDB
:101D7000CE0101960E94505C0E9413998091D10679
:101D80009091D206DC01ED91FC910680F781E02D67
:101D900019958091D1069091D2060E941D5E0E94F5
:101DA000F17F62E376E08091D1069091D2060E94A5
:101DB000BF5CE091170BE4300CF0E0E08EEB95E0B7
:101DC0009A8389838AEB95E09C838B8385EB95E0EE
:101DD0009E838D8380EB95E098878F83EE0FFF0BBA
:101DE00081E090E08C0F9D1FE80FF91F60817181E9
:101DF0008091D1069091D2060E94305E0E94F17FC0
:101E00006CEF75E08091D1069091D2060E94305E11
:101E10000E94F17F60EF75E08091D1069091D2062B
:101E20000E94BF5CE091EF10F091F01081819281EF
:101E3000883E934014F40E94E17FE091EF10F0910E
:101E4000F010618172818091D1069091D2060E943A
:101E5000374684E00E944187E091EF10F091F01046
:101E6000658176818091D1069091D2060E94374695
:101E700085E00E944187E091EF10F091F0106381BE
:101E800074818091D1069091D2060E94374684E0F9
:101E90000E944187E091EF10F091F01067818091EE
:101EA000D1069091D2060E940A4588E00E9441879F
:101EB000E091EF10F091F01080850E94C77F64EEF2
:101EC00075E08091D1069091D2060E94BF5CE091AE
:101ED000F910F091FA1081819281883E934014F4B8
:101EE0000E94E17FE091F910F091FA106181728116
:101EF0008091D1069091D2060E94374684E00E94DC
:101F00004187E091F910F091FA1065817681809116
:101F1000D1069091D2060E94374685E00E94418703
:101F2000E091F910F091FA10638174818091D106EB
:101F30009091D2060E94374684E00E944187E0914A
:101F4000F910F091FA1067818091D1069091D20634
:101F50000E940A4588E00E944187E091F910F091C3
:101F6000FA1080850E94C77F68ED75E08091D106E8
:101F70009091D2060E94BF5CE0910311F091041190
:101F800081819281883E934014F40E94E17FE09128
:101F90000311F0910411618172818091D1069091B9
:101FA000D2060E94374684E00E944187E0910311E7
:101FB000F0910411658176818091D1069091D206CD
:101FC0000E94374685E00E944187E0910311F0911D
:101FD0000411638174818091D1069091D2060E9490
:101FE000374684E00E944187E0910311F09104118B
:101FF00067818091D1069091D2060E940A4588E0BF
:102000000E944187E0910311F091041180850E94A4
:10201000C77F6CEC75E08091D1069091D2060E944A
:10202000BF5CE0910D11F0910E1181819281883E8B
:10203000934014F40E94E17FE0910D11F0910E1194
:10204000618172818091D1069091D2060E943746BB
:1020500084E00E944187E0910D11F0910E1165819D
:1020600076818091D1069091D2060E94374685E014
:102070000E944187E0910D11F0910E1163817481EE
:102080008091D1069091D2060E94374684E00E944A
:102090004187E0910D11F0910E1167818091D10679
:1020A0009091D2060E940A4588E00E944187E09103
:1020B0000D11F0910E1180850E94C77F8091D1068D
:1020C0009091D2060E941D5E0E945B4CC82E64E671
:1020D00076E08091D1069091D2060E94305E0E94F7
:1020E000F17F0EE810E1E12CF12CD12C57012FEFFC
:1020F000A21AB20AB5018091D1069091D2060E942F
:10210000374649E0E416F10410F48BE001C08AE0A0
:102110000E944187D8012C918091D1069091D206DE
:102120002223C9F11596ED91FC9116976181728178
:102130000E943746D8011596ED91FC911697818142
:102140009281883E934014F40E94E17F84E00E94D3
:102150004187D8011596ED91FC91169763817481A2
:102160008091D1069091D2060E94374684E00E9469
:102170004187D8011596ED91FC91169727818091A2
:10218000D1069091D206222319F06CE576E00BC0BF
:1021900065E576E008C0EC14FD041CF46DE476E01F
:1021A00002C060E476E00E94305E095F1F4F750157
:1021B000BCE0AB16B10409F099CF0E94F17F69E948
:1021C00076E08091D1069091D2060E94BF5C0E9479
:1021D0005B4C682F8091D1069091D2060E94F34407
:1021E00065E876E08091D1069091D2060E94BF5CAE
:1021F0006091140B7091150B8091D1069091D206CD
:102200000E946D460E9413998091D1069091D2064A
:10221000DC01ED91FC910680F781E02D199580910C
:10222000D1069091D2060E941D5E0E94F17F69E660
:1022300077E08091D1069091D2060E94305E0E9494
:10224000F17F65E577E08091D1069091D2060E94FA
:10225000BF5C80912B0F0E94E588BC018091D10664
:102260009091D2060E94BF5C80912B0F8A30C1F4FE
:1022700063E477E08091D1069091D2060E94BF5C22
:102280006091E80F8091D1069091D2060E940A4594
:102290006CE377E08091D1069091D2060E94BF5CFA
:1022A0008091D1069091D2060E941D5E68E277E08F
:1022B0008091D1069091D2060E94BF5C80912C0F34
:1022C0000E94E588BC018091D1069091D2060E94BF
:1022D000BF5C20912C0F8091D1069091D2062B30BB
:1022E0003CF4293054F4283069F467E177E007C002
:1022F0002B3041F463E277E002C06DE177E00E94A9
:10230000305E02C00E941D5E63E077E08091D106DE
:102310009091D2060E94BF5C80912D0F0E94E588AB
:10232000BC018091D1069091D2060E94BF5C2091A1
:102330002D0F8091D1069091D2062B303CF429309C
:1023400054F4283069F462EF76E007C02B3041F492
:102350006EEF76E002C068EF76E00E94305E02C069
:102360000E941D5E6EED76E08091D1069091D206BE
:102370000E94BF5C20913F0F8091D1069091D206C0
:10238000222319F066ED76E002C064EC76E00E944C
:10239000BF5C20918C128091D1069091D2062223AD
:1023A00019F069EB76E002C06DEA76E00E94BF5C4E
:1023B0008091D1069091D2060E941D5E0E941399D1
:1023C0008091D1069091D206DC01ED91FC910680BE
:1023D000F781E02D199580910002823011F00C9464
:1023E000731CF090650F0091680F10E08091D1068A
:1023F0009091D2060E941D5E0E94F17F62E37AE016
:102400008091D1069091D2060E94305E0E94F17FA9
:1024100069E17AE08091D1069091D2060E94BF5C7A
:10242000E091750FE6300CF0E0E08EEA97E09A83D9
:10243000898389EA97E09C838B838FE997E09E8369
:102440008D838BE997E098878F8387E897E09A8759
:10245000898785E797E09C878B87EE0FFF0B81E0EC
:1024600090E08C0F9D1FE80FF91F608171818091B2
:10247000D1069091D2060E94305E60E07AE08091B1
:10248000D1069091D2060E94BF5C609100028091BB
:10249000D1069091D2060E94F34467EE79E08091D4
:1024A000D1069091D2060E94BF5C8F2D0E94B27F10
:1024B000FF2009F44BC06DED79E08091D106909139
:1024C000D2060E94BF5C8091D1069091D206112362
:1024D00039F06091600F0E940A459091600F06C02C
:1024E0006091660F0E940A459091660F8091BA1321
:1024F00098130C947A1C61EC79E08091D10690914C
:10250000D2060E94BF5C8091D1069091D206112321
:1025100039F06091610F61110CC06CEB79E006C07D
:102520006091670F611105C067EB79E00E94BF5CA5
:1025300005C0062E000C770B0E94374665EB79E04C
:102540008091D1069091D2060E94BF5C8091D10605
:102550009091D2060E941D5E6CE979E08091D106CF
:102560009091D2060E94BF5C802F0E94B27F002310
:1025700009F44BC062E979E08091D1069091D206CE
:102580000E94BF5C8091D1069091D206112339F050
:102590006091630F0E940A459091630F06C060919D
:1025A000690F0E940A459091690F8091BC1398139E
:1025B0000C94941C66E779E08091D1069091D20644
:1025C0000E94BF5C8091D1069091D206112339F010
:1025D0006091640F61110CC061E779E006C0609101
:1025E0006A0F611105C06CE679E00E94BF5C05C00E
:1025F000062E000C770B0E9437466AE679E0809140
:10260000D1069091D2060E94BF5C8091D106909134
:10261000D2060E941D5E61E579E08091D10690911D
:10262000D2060E94BF5C80917E0F811103C00E9480
:10263000C07F35C066EB77E08091D1069091D206DD
:102640000E94BF5C6EE479E08091D1069091D20641
:102650000E94BF5C60917E0F8091D1069091D2065E
:102660000E940A456EE379E08091D1069091D206EE
:102670000E94BF5C40917F0F5091800F60E070E03E
:102680002AE08091D1069091D2060E94F85C69E31D
:1026900079E08091D1069091D2060E94305E60E28E
:1026A00079E08091D1069091D2060E94BF5C809122
:1026B000760F8436C8F469E179E08091D106909173
:1026C000D2060E94BF5C6091760F8091D1069091F6
:1026D000D2060E940A4567E179E08091D106909187
:1026E000D2060E94305E03C080E00E94C07F6EEF81
:1026F00078E08091D1069091D2060E94BF5C8091D3
:10270000770F8436C8F467EF78E08091D106909116
:10271000D2060E94BF5C6091770F8091D1069091A4
:10272000D2060E940A4565EF78E08091D10690912B
:10273000D2060E94305E03C080E00E94C07F6CED34
:1027400078E08091D1069091D2060E94BF5C2091E2
:10275000CA068091D1069091D206222319F065ED28
:1027600078E002C06BEC78E00E94305E62EB78E0CB
:102770008091D1069091D2060E94BF5C60916C0F4F
:1027800070916D0F072E000C880B990B0E944EBDA7
:1027900020E030E04AE754E40E9453BFAB01BC01A3
:1027A00021E08091D1069091D2060E94405D6DEAB1
:1027B00078E08091D1069091D2060E94305E64E963
:1027C00078E08091D1069091D2060E94BF5C609122
:1027D0006E0F70916F0F072E000C880B990B0E94E3
:1027E0004EBD20E030E04AE754E40E9453BFAB0105
:1027F000BC0121E08091D1069091D2060E94405DFB
:102800006FE878E08091D1069091D2060E94305E08
:1028100066E778E08091D1069091D2060E94BF5C75
:102820006091700F7091710F072E000C880B990B3F
:102830000E944EBD20E030E04AE754E40E9453BFBE
:10284000AB01BC0121E08091D1069091D2060E949B
:10285000405D61E778E08091D1069091D2060E94B8
:10286000305E68E578E08091D1069091D2060E94B2
:10287000BF5C9091750F913011F09430F9F4809114
:10288000720F0E94B27F8091720F882329F164E554
:1028900078E08091D1069091D2060E94BF5C609151
:1028A000730F8091D1069091D2060E940A4562E58D
:1028B00078E08091D1069091D2060CC02091D1068B
:1028C0003091D206953019F465E478E002C060E3F7
:1028D00078E0C9010E94BF5C8091D1069091D20638
:1028E0000E941D5E67E178E08091D1069091D2064A
:1028F0000E94BF5C9091750F2FEF290F8091D10638
:102900009091D206223028F460912E060E94F34462
:1029100004C062E078E00E94305E69EE77E080916A
:10292000D1069091D2060E94BF5C8091820F0E94D6
:10293000B27F8091820F882341F167ED77E080912B
:10294000D1069091D2060E94BF5C6091830F809166
:10295000D1069091D2060E940A456FEB77E08091F4
:10296000D1069091D2060E94BF5C6091840F809145
:10297000D1069091D2060E940A456DEB77E08091D6
:10298000D1069091D2060E94BF5C8091D1069091B1
:10299000D2060E941D5E0E9413998091D1069091EB
:1029A000D206DC01ED91FC910680F781E02D1995AE
:1029B0008091D1069091D2060E941D5E0E94F17F07
:1029C0006BEB7AE08091D1069091D2060E94305E46
:1029D0000E94F17F6AE97AE08091D1069091D20657
:1029E0000E94BF5C8091340F8436C8F463E97AE0BA
:1029F0008091D1069091D2060E94BF5C6091340F05
:102A00008091D1069091D2060E940A4561E97AE050
:102A10008091D1069091D2060E94305E03C080E082
:102A20000E94C07F60E77AE08091D1069091D20643
:102A30000E94BF5C8091330F8436C8F469E67AE067
:102A40008091D1069091D2060E94BF5C6091330FB5
:102A50008091D1069091D2060E940A4567E67AE0FD
:102A60008091D1069091D2060E94305E03C080E032
:102A70000E94C07F66E47AE08091D1069091D206F0
:102A80000E94BF5C6091410F7091420F16161706AD
:102A900014F50091D1061091D206072E000C880B78
:102AA000990B0E944EBD20E030E04AE754E40E94BA
:102AB00053BFAB01BC0122E0C8010E94405DC801C8
:102AC0000E941D5E61E47AE08091D1069091D20669
:102AD0000E94305E03C080E00E94C07F0E94139974
:102AE0008091D1069091D206DC01ED91FC91068097
:102AF000F781E02D19958091D1069091D2060E9420
:102B00001D5E0E94F17F6CEC7BE08091D10690917C
:102B1000D2060E94305E0E94F17F20914E0F80917C
:102B2000D1069091D206211103C06AEA7BE0B9C1B7
:102B300063E97BE00E94BF5CE091570FE3300CF04B
:102B4000E3E084EF9AE09A83898380EE9AE09C83A5
:102B50008B8383ED9AE09E838D838BEC9AE098873C
:102B60008F83EE0FFF0B81E090E08C0F9D1FE80F2D
:102B7000F91F608171818091D1069091D2060E94E7
:102B8000305EFF24F3948091570F811101C0F12C26
:102B90006CE77BE08091D1069091D2060E94BF5CE9
:102BA0006091580F8091D1069091D206611103C0B7
:102BB00068E77BE008C00E940A456FE67BE08091F1
:102BC000D1069091D2060E94305E60914F0F7091B5
:102BD000500F072E000C880B990B0E944EBD20E071
:102BE00030E04FE753E40E9453BF20E030E048EC70
:102BF00052E40E94ADBD20E030E040E05FE30E947F
:102C0000EFBE0E94BBBFE62E262F372F8901C09052
:102C1000590FD0905A0F68E57BE08091D1069091D2
:102C2000D2060E94BF5C8E2D0E94A37F0436110540
:102C30003CF40E94E17F0A30110514F40E94E17F08
:102C400083E00E944187FF2001F10E94F89EB601B7
:102C5000DD0C880B990B0E944EBD20E030E04FE761
:102C600053E40E9453BF20E030E048EC52E40E945D
:102C7000ADBD20E030E040E05FE30E94EFBE0E9487
:102C8000BBBF862F0E94A37F04C00E94F09E0E94BB
:102C9000E89E0E94DB7F6091510F7091520F072ECA
:102CA000000C880B990B0E944EBD20E030E04FE7EE
:102CB00053E40E9453BF20E030E048EC52E40E940D
:102CC000ADBD20E030E040E05FE30E94EFBE0E9437
:102CD000BBBFE62E262F372F8901C0905B0FD09007
:102CE0005C0F61E47BE08091D1069091D2060E9456
:102CF000BF5C8E2D0E94A37F043611053CF40E9418
:102D0000E17F0A30110514F40E94E17F83E00E9404
:102D10004187FF2001F10E94F89EB601DD0C880B6F
:102D2000990B0E944EBD20E030E04FE753E40E9433
:102D300053BF20E030E048EC52E40E94ADBD20E0FB
:102D400030E040E05FE30E94EFBE0E94BBBF862FF1
:102D50000E94A37F04C00E94F09E0E94E89E0E94F1
:102D6000DB7F6091530F7091540F072E000C880B7E
:102D7000990B0E944EBD20E030E04FE753E40E94E3
:102D800053BF20E030E048EC52E40E94ADBD20E0AB
:102D900030E040E05FE30E94EFBE0E94BBBFE62E42
:102DA000262F372F8901C0905D0FD0905E0F6AE209
:102DB0007BE08091D1069091D2060E94BF5C8E2D5F
:102DC0000E94A37F043611053CF40E94E17F0A3083
:102DD000110514F40E94E17F83E00E944187FF20E7
:102DE00001F10E94F89EB601DD0C880B990B0E9440
:102DF0004EBD20E030E04FE753E40E9453BF20E097
:102E000030E048EC52E40E94ADBD20E030E040E00C
:102E10005FE30E94EFBE0E94BBBF862F0E94A37F8C
:102E200004C00E94F09E0E94E89E0E94DB7F63E146
:102E30007BE08091D1069091D2060E94BF5C6091A8
:102E4000550F7091560F0091D1061091D206611561
:102E5000710521F46AE07BE0C80123C0072E000C55
:102E6000880B990B0E944EBD20E030E04FE753E401
:102E70000E9453BF20E030E048EC52E40E94ADBD18
:102E800020E030E040E05FE30E94EFBE0E94BBBF65
:102E9000C8010E94374668E07BE08091D10690919E
:102EA000D2060E94305E0E9413998091D1069091C3
:102EB000D206DC01ED91FC910680F781E02D199599
:102EC0008091D1069091D2060E941D5E0E94F17FF2
:102ED00068E37DE08091D1069091D2060E94305E39
:102EE0000E94F17F209150068091D1069091D206E8
:102EF000222309F4C3C169E07DE00E94BF5C0E9407
:102F00005E620E94C07F0E945E622091D106309175
:102F1000D206882389F066EF7CE0C9010E94BF5C7D
:102F2000809153060E942080BC018091D10690912F
:102F3000D2060E94305E4FC063EE7CE0C9010E9461
:102F4000BF5C809150060E942080BC018091D10618
:102F50009091D2060E94BF5C809151068823A9F10E
:102F60006BED7CE08091D1069091D2060E94BF5C0F
:102F7000E0915106E4300CF0E0E08CE793E09A83B6
:102F800089838AE793E09C838B8388E793E09E8321
:102F90008D8386E793E098878F83EE0FFF0B81E0A8
:102FA00090E08C0F9D1FE80FF91F60817181809167
:102FB000D1069091D2060E94BF5C69ED7CE08091C1
:102FC000D1069091D2060E94BF5C8091D10690916B
:102FD000D2060E941D5E66EC7CE08091D106909145
:102FE000D2060E94BF5C809152060091D1061091DA
:102FF000D206882321F00E942080BC0102C062EC2E
:103000007CE0C8010E94305E6FEA7CE08091D106CE
:103010009091D2060E94BF5C809153060091D10628
:103020001091D206882321F00E942080BC0102C0AA
:103030006BEA7CE0C8010E94305E68E97CE0809128
:10304000D1069091D2060E94BF5C809155068823DC
:10305000E1F062E97CE08091D1069091D2060E9475
:10306000BF5C809154060E942080BC018091D106F3
:103070009091D2060E94BF5C60E176E08091D1061B
:103080009091D2060E94205E03C080E00E94C07F23
:103090006FE77CE08091D1069091D2060E94BF5CE0
:1030A000809156068823E1F069E77CE08091D106A3
:1030B0009091D2060E94BF5C809154060E942080AD
:1030C000BC018091D1069091D2060E94BF5C60E164
:1030D00076E08091D1069091D2060E94205E03C0D6
:1030E00080E00E94C07F66E67CE08091D1069091EE
:1030F000D2060E94BF5CE0915706E3300CF0E3E09B
:103100008EE09CE09A83898382E09CE09C838B83A1
:103110008DEF9BE09E838D8385EF9BE098878F8367
:10312000EE0FFF0BA1E0B0E0AC0FBD1FEA0FFB1FDD
:10313000608171818091D1069091D2060E94305EAB
:1031400063E57CE08091D1069091D2060E94BF5C3D
:10315000E0914906E4300CF0E4E08EEE9BE09A83C7
:10316000898388EE9BE09C838B8381EE9BE09E832A
:103170008D838BED9BE098878F8383ED9BE09A870F
:103180008987EE0FFF0B81E090E08C0F9D1FE80F09
:10319000F91F608171818091D1069091D2060E94C1
:1031A000305E61E57CE08091D1069091D2060E946C
:1031B000BF5C60914E068091D1069091D2060E942C
:1031C0000A4562E47CE08091D1069091D2060E948B
:1031D000BF5C80914906811110C060914F068091BB
:1031E000D1069091D2060E940A4567E37CE0809167
:1031F000D1069091D2060E94BF5C60914A06709100
:103200004B06072E000C880B990B0E944EBD20E048
:1032100030E04AE754E40E9453BFAB01BC0121E017
:103220008091D1069091D2060E94405D69E27CE0D7
:103230008091D1069091D2060E94BF5C60914C06AD
:1032400070914D06072E000C880B990B0E944EBD05
:1032500020E030E04AE754E40E9453BFAB01BC01D8
:1032600021E08091D1069091D2060E94405D6AE1F2
:103270007CE08091D1069091D20602C06CE17DE0A5
:103280000E94305E0E9413998091D1069091D206DF
:10329000DC01ED91FC910680F781E02D199580917C
:1032A000D1069091D2060E941D5E0E94F17F66EBCE
:1032B0007DE08091D1069091D2060E94305E0E94FE
:1032C000F17F69EA7DE08091D1069091D2060E945B
:1032D000BF5CE0918B0FE5300CF0E5E087E99DE005
:1032E0009A83898380E89DE09C838B838EE69DE0B2
:1032F0009E838D838FE59DE098878F838CE49DE08E
:103300009A87898784E49DE09C878B87EE0FFF0B6B
:1033100081E090E08C0F9D1FE80FF91F60817181A3
:103320008091D1069091D2060E94305E0E9413993E
:103330008091D1069091D206DC01ED91FC9106803E
:10334000F781E02D199583EA96E8A1E0BB278BABC6
:103350009CABADABBEAB8091D1069091D2060E94E2
:103360001D5E0E94F17F6BEC7FE08091D106909111
:10337000D2060E94305E0E94F17F62EB7FE0809176
:10338000D1069091D2060E94BF5C2091120B8091D1
:10339000D1069091D206222319F06EEA7FE002C096
:1033A00069EA7FE00E94305E8091120B882349F128
:1033B00060E97FE08091D1069091D2060E94BF5CC7
:1033C0006091890F70918A0F072E000C880B990B62
:1033D0000E944EBD20E030E04AE754E40E9453BF13
:1033E000AB01BC0122E08091D1069091D2060E94EF
:1033F000405D6BE87FE08091D1069091D2060E94FB
:10340000305E95EBE92E9EE0F92E29E2622E38E13E
:10341000232E3CEF332E4AE0A42EB12C54E6C52EC9
:10342000D12CD7012C91222309F400C2F701329745
:10343000008111810115110509F4F8C180E096E8B9
:10344000A1E0BB27820F911DA11DB11DABBFFC01E7
:10345000879177247394811101C0712C2091D1063A
:103460003091D206C8010197849790F56BE67FE012
:10347000C9010E94BF5C09500C3148F4E02FF0E014
:10348000EE0FFF1FE25EFD4F6081718102C061ECB3
:103490007DE08091D1069091D2060E94BF5C0C31F4
:1034A00030F4E02FF0E0EA5AFD4F808101C080E067
:1034B00090E08F59904F092E000CAA0BBB0BABBFAD
:1034C000FC0187919EE0981B892F09F051C152C1E0
:1034D000C801845691098438934008F03FC061E5E3
:1034E0007FE0C9010E94BF5CC801B6010E9486C08E
:1034F0006130710531F06230710559F46DE47FE09F
:1035000002C06FE47FE08091D1069091D2060E94C4
:10351000BF5C0E94E97F8090D1069090D206772010
:10352000B1F0C8010E945D8F811107C069E47FE09E
:10353000C4010E94BF5C87E01BC1813009F01AC141
:1035400066E47FE0C4010E94BF5C88E011C16DE3C6
:103550007FE0C4010E94BF5C82E00AC1C801885EAE
:1035600093408035964408F05AC0C80168EE73E075
:103570000E9486C04B0160E37FE0C9010E94BF5CEE
:10358000FAE08F16910410F40E94E17FB40180915B
:10359000D1069091D2060E9437460E94E97F409062
:1035A000D1065090D2067720A1F1C8010E945D8F0C
:1035B000782E6BE27FE0C2010E94BF5C672D809194
:1035C000D1069091D2060E940A4565E27FE0809183
:1035D000D1069091D2060E94BF5C829CC001839C60
:1035E000900D929C900D1124800F911FB5010E94A7
:1035F0009AC077278091D1069091D2060E943746D3
:1036000063E27FE08091D1069091D2060E94BF5C78
:10361000B1C06AE17FE0C2010E94BF5C61C0F801F5
:10362000E853FA44E83E43E0F40708F046C0EC30C3
:10363000F10508F09FC08827EE58FF4F8F4F0C947C
:10364000ADC06BE07FE019C060E07FE0C9010E947F
:10365000BF5C83E18DC06EEE7EE027C06EED7EE044
:1036600016C061ED7EE055C065EC7EE0C9010E94A8
:10367000BF5C82E17DC066EB7EE0C9010E94BF5C59
:103680008FE076C067EA7EE0F8CF67E97EE0C901A7
:103690000E94BF5C8EE06CC064E87EE0C9010E94BD
:1036A000BF5C8BE065C062E77EE0C9010E94BF5C41
:1036B0008CE05EC065E67EE02CC0C80180529E446E
:1036C000883E934078F400526EE47EE0C9010E9487
:1036D000BF5C0A3010F40E94E17F802F0E94A37F1C
:1036E00084E046C0C80188509245883E934020F44B
:1036F000085067E37EE0EACF013FE5E51E0719F4D5
:1037000066E27EE01CC0023FF5E51F0739F469E17F
:103710007EE0C9010E94BF5C81E12AC0033F45E50C
:10372000140739F46BE07EE0C9010E94BF5C80E1C0
:103730001FC0043F85E5180739F46AEF7DE0C90131
:103740000E94BF5C8DE014C0053F95E5190739F470
:1037500062EE7DE0C9010E94BF5C86E009C0063FC1
:10376000154541F469EC7DE0C9010E94BF5C85E02C
:103770000E94418766E87FE08091D1069091D20651
:103780000E94BF5C6BE77FE08091D1069091D206EA
:103790000E94BF5CF701608170E08091D10690913A
:1037A000D2060E943746D7018C918A3020F482E0FD
:1037B0000E94418704C0843610F40E94E17F0E9479
:1037C000E97FF7014081649EA0011124052E000CC1
:1037D000660B770B8BA99CA9ADA9BEA9480F591FF1
:1037E0006A1F7B1FDE0111968A019B010F5F1F4F2D
:1037F0002F4F3F4F6BBFFA0187918D93B901A801FD
:103800008111F2CFBE016F5F7F4F8091D106909101
:10381000D2060E94205E8091D1069091D206DC01F2
:10382000ED91FC910680F781E02D1995B3E0EB0E48
:10383000F11CEDE2EE16EFE0FE0609F0F2CD0E947B
:1038400013998091D1069091D206DC01ED91FC9103
:103850000680F781E02D19958091D1069091D206CE
:103860000E941D5E0E94F17F6CE270E18091D106A2
:103870009091D2060E94305E0E94F17F69E170E172
:103880008091D1069091D2060E94BF5C0E94A17BDC
:1038900020E030E040E050E40E9448BD2091D10695
:1038A0003091D20687FD5AC062E170E1C9010E94E1
:1038B000305E6FEF7FE08091D1069091D2060E943A
:1038C000BF5C0E94A17BAB01BC0122E08091D106CC
:1038D0009091D2060E94405D6DEF7FE08091D1060D
:1038E0009091D2063EC0F0905F0F0091620F11E000
:1038F0000C94F6116EEC79E08091D1069091D2068D
:103900000E94BF5C6091BA138091D1069091D2065B
:103910000E940A456CEC79E08091D1069091D20624
:103920000E94BF5C0C947B1263E879E08091D10621
:103930009091D2060E94BF5C6091BC138091D10629
:103940009091D2060E940A4561E879E08091D10603
:103950009091D2060E94BF5C0C94DA1266E170E18D
:10396000C9010E94305E6AEE7FE08091D10690919D
:10397000D2060E94BF5C8091D50F0E94B27F209139
:10398000D50F8091D1069091D206222379F067EE6F
:103990007FE00E94BF5C0E947F876DED7FE0809199
:1039A000D1069091D2060E94305E02C00E941D5E38
:1039B0000E9413998091D1069091D206DC01ED917D
:1039C000FC910680F781E02D19958091D1069091A8
:1039D000D2060E941D5E0E94F17F64E870E1809132
:1039E000D1069091D2060E94305E0E94F17F60E77E
:1039F00070E18091D1069091D2060E94BF5C409107
:103A0000C50F5091C60F6091C70F7091C80F80917C
:103A1000D1069091D2060E9424466CE570E1809117
:103A2000D1069091D2060E94BF5C4091CD0F50917B
:103A3000CE0F6091CF0F7091D00F8091D1069091F1
:103A4000D2060E94244668E470E18091D1069091EC
:103A5000D2060E94BF5C4091C90F5091CA0F60917D
:103A6000CB0F7091CC0F8091D1069091D2060E941D
:103A7000244664E370E18091D1069091D2060E94C1
:103A8000BF5C4091D10F5091D20F6091D30F7091D4
:103A9000D40F8091D1069091D2060E9424460E94B4
:103AA00013998091D1069091D206DC01ED91FC91A1
:103AB0000680F781E02D19958091D1069091D2066C
:103AC0000E941D5E0E94F17FE6960FB6F894DEBF5D
:103AD0000FBECDBFDF91CF911F910F91FF90EF905F
:103AE000DF90CF90BF90AF909F908F907F906F901E
:103AF0005F904F903F902F9008952F923F924F925A
:103B00005F926F927F928F929F92AF92BF92CF926D
:103B1000DF92EF92FF920F931F93CF93DF93CDB776
:103B2000DEB7AB970FB6F894DEBF0FBECDBF8CEDFE
:103B300091E00E9479BE6C347D458105910519F0B4
:103B40000E945D8108C040EE51E060E070E08EE0D0
:103B50009EE00E9461BE40E052EC61E070E086EFC2
:103B600098E00E943A734091C90F5091CA0F60913A
:103B7000CB0F7091CC0F89E598E00E943A73409189
:103B8000CD0F5091CE0F6091CF0F7091D00F8CEB75
:103B900097E00E943A734091D10F5091D20F6091FB
:103BA000D30F7091D40F8FE197E00E943A738CECA1
:103BB0009DE090931D0780931C078DE89BE09093F8
:103BC0001B0780931A0786EF98E09093A3138093C6
:103BD000A2131092A4131092D10D1092CE0D109238
:103BE000D00D1092CF0D11E0109393120E94C84097
:103BF0008091E90F8093D4061092D3061092800032
:103C000082E0809381008FE286BB10926F00109259
:103C10008500109284009BE29093A00099E090931D
:103C2000A10089BB109272001092A5001092A4000E
:103C30001092A9001092A8001092AB001092AA0056
:103C40001092AD001092AC0099EA9093200110936D
:103C500021018ABB10927300109225011092240159
:103C6000109229011092280110922B0110922A0122
:103C700010922D0110922C018091AB0E9091AC0E00
:103C80008093650690936606813001F58FE38093FB
:103C9000350B1092360B61E00E9466608BE29BE070
:103CA0000E945B851092370B10923A0B1092390BE1
:103CB00080916606882329F08BE29BE00E942E8784
:103CC00011C08BE29BE00E9407870CC080916606C2
:103CD000882311F062E001C060E08FE30E9466601B
:103CE0000E94353D8091AD0E9091AE0E80936B0693
:103CF00090936C06813001F58EE38093660B1092F1
:103D0000670B61E00E9466608CE59BE00E945B852A
:103D10001092680B10926B0B10926A0B80916C06DC
:103D2000882329F08CE59BE00E942E8711C08CE54A
:103D30009BE00E9407870CC080916C06882311F0DD
:103D400062E001C060E08EE30E9466600E94747CC5
:103D500060E085E40E94666062E08CE30E94666039
:103D600062E08BE30E94666062E080E40E9466602D
:103D700062E081E40E94666062E082E40E94666024
:103D800062E081E20E94666062E084E40E94666014
:103D900061E089E30E94666061E08AE30E946660F8
:103DA0000E94567A0E948D7A61E085E30E946660E7
:103DB00061E085E00E94666061E070E085E00E945D
:103DC000A26061E084E00E94666061E087E00E949A
:103DD000666061E089E20E94376061E089E20E94EA
:103DE0006660519A60E085E30E94376060E085E09C
:103DF0000E94376060E084E00E94376060E087E006
:103E00000E943760599861E088E00E94666080E017
:103E100090E09C01225F314FF901E955FF4F40814D
:103E20004F3629F4329720813181232B31F40396C8
:103E30008837910571F760E001C061E088E00E9479
:103E4000376061E08DE20E94666061E08EE20E9470
:103E5000666061E08CE20E94666061E08BE20E9435
:103E6000666060E08BE20E9437600E948D7A0E945B
:103E7000B54580911B0B813009F058C080911E0B15
:103E800090911F0BA091200BB091210B4091220B20
:103E90005091230B6091240B7091250B841B950B83
:103EA000A60BB70B84379E40A105B10500F30E9415
:103EB0005D810E94DB7F0E94DB7F0E94F17F62E9CF
:103EC00070E18091D1069091D2060E94BF5C01E022
:103ED00010E00E945A7A0E948D7A6EEE72E080E0C5
:103EE00090E00E9450936FE870E18091D10690912C
:103EF000D2060E94BF5C0E94567A0E94897A0530E1
:103F0000110531F064EF71E080E090E00E94509381
:103F10000F5F1F4F06301105E1F60E94DB7F0E9404
:103F2000F17F0E94DB7F0E94DB7F02C081119FCF67
:103F300080916F00826080936F00809184009091E7
:103F400085008056904F90938900809388000E944E
:103F5000CF2B8EE89BE0909309128093081210916A
:103F6000840F2091830F8091720F9091740F309184
:103F7000750F30931E0790932E0680932F0630E026
:103F8000AFEFB0E00E94DFBE24E630E040E050E05A
:103F90000E9491BE2093C313612F70E080E090E0F7
:103FA0000E944CBD23EC34E64AEA5AE30E94ADBDC0
:103FB0002AE939E949E55FE30E94EFBE6093BD134A
:103FC0007093BE138093BF139093C013109295000B
:103FD00010929400109290008CE08093910084EFF6
:103FE00090E0909399008093980011E018BB82E0D4
:103FF00080937100809100020E9464408091D106FC
:104000009091D2062091D40640916E0F50916F0F7F
:1040100050934B1340934A132093DF0D9093DE0D82
:104020008093DD0D1092300610934C1380918B0F0E
:10403000853040F010928B0F60E070E08DE791E0EA
:104040000E94464510918B0F123009F444C008F5C8
:10405000112309F466C0113009F05BC08CE090E0D8
:104060000E94C1C02AE433E0DC0111963C932E93F8
:104070002CEB37E01B963C932E931A979093CE0629
:104080008093CD0610933313109336131093391386
:1040900067C0133009F45EC01430D9F586E090E0B3
:1040A0000E94C1C08C0124EB33E0DC012D933D93D1
:1040B000CD0141E06EE87BE00E94BA7486E792E0B1
:1040C000F801918380831093CE060093CD0681E0A2
:1040D0008093331341C086E090E00E94C1C020EE7F
:1040E00032E0FC01318320839093CE068093CD068D
:1040F0008FB7F8942CED35E0309311112093101107
:10410000109216118FBF81E0809333138093361382
:1041100025C010928B0F60E070E08DE791E00E9467
:10412000464586E090E00E94C1C08C0124EB33E05C
:10413000DC012D933D93CD0140E06EE87BE00E94D1
:10414000BA7486E792E0F801918380831093CE06DB
:104150000093CD0610923313109236131092391338
:104160008091CD069091CE06DC01ED91FC910190FD
:10417000F081E02D19958091271381111FC0809146
:104180002A1381111BC080912D13811117C08091BA
:104190003013811113C08091331381110FC08091AE
:1041A000361381110BC080913913811107C081E052
:1041B0000E94C440882309F419C311C3A12CB12C57
:1041C000912C1DA2412C512C612C712C812C00EFC3
:1041D00015E0EE24EA94A3E0FA2ECC24CA94DD2460
:1041E000D39484EE282E85E0382EC501825F914F4E
:1041F000FC01E955FF4FE081EE2309F4E7C2DC0141
:10420000AB55BF4F8D919C91892B09F4DFC28E2F46
:1042100090E0FC01F797EB32F10508F0D7C2882750
:10422000E258FF4F8F4F0C94ADC080912713882325
:1042300009F4CCC28110CAC289E190E00E94C1C0D9
:104240009C01FC011183008387E090E093838283CB
:1042500015821482F782E682D186C086108EC9014B
:104260002AA73BA70E94AE572AA53BA5E6E3F4E0A8
:10427000D901ED93FC933093181320931713C901C0
:104280000E949D6C7DC180912A13882309F49EC2EF
:1042900071109CC289E190E00E94C1C09C01DC01C8
:1042A00011961C930E93E6E0F0E01396FC93EE93C8
:1042B000129715961C921E9214971796FC92EE92E6
:1042C00016971996DC92CE92189758961C922AA7A8
:1042D0003BA70E94AE572AA53BA5E6E3F4E0D9012F
:1042E000ED93FC9330931A1320931913C9010E9484
:1042F0009D6C74C180912D13882309F467C26110ED
:1043000065C289E190E00E94C1C09C01DC01119668
:104310001C930E93E5E0F0E01396FC93EE93129756
:1043200015961C921E9214971796FC92EE92169771
:104330001996DC92CE92189758961C922AA73BA702
:104340000E94AE572AA53BA5E6E3F4E0D901ED9320
:10435000FC9330931C1320931B13C9010E949D6C86
:104360006BC180913013882309F430C251102EC2E2
:1043700089E190E00E94C1C09C01DC0111961C9370
:104380000E93E4E0F0E01396FC93EE9312971596EB
:104390001C921E9214971796FC92EE9216971996FD
:1043A000DC92CE92189758961C922AA73BA70E949F
:1043B000AE572AA53BA5E6E3F4E0D901ED93FC93C3
:1043C00030931E1320931D13C9010E949D6C62C17E
:1043D00080913313882309F4F9C14110F7C189E1B1
:1043E00090E00E94C1C09C01DC0111961C930E93C9
:1043F000E2E0F0E01396FC93EE93129715961C9270
:104400001E9214971796FC92EE9216971996DC92CC
:10441000CE92189758961C922AA73BA70E94AE5797
:104420002AA53BA5E6E3F4E0D901ED93FC93309394
:10443000201320931F13C9010E949D6C59C18091C4
:104440003613882309F4C2C12DA12111BFC189E10E
:1044500090E00E94C1C09C01DC0111961C930E9358
:10446000E1E0F0E01396FC93EE93129715961C9200
:104470001E9214971796FC92EE9216971996DC925C
:10448000CE92189758961C922AA73BA70E94AE5727
:104490002AA53BA5E6E3F4E0D901ED93FC93309324
:1044A000221320932113C9010E949D6C59C1809150
:1044B0003913882309F48AC1911088C189E190E0F9
:1044C0000E94C1C09C01DC0111961C930E931396AF
:1044D0001C921E92129715961C921E921497179674
:1044E000FC92EE9216971996DC92CE9218975896F7
:1044F0001C922AA73BA70E94AE572AA53BA586E39C
:1045000094E0F90191838083309324132093231343
:10451000C9010E949D6C58C180912713882309F41A
:1045200055C1811053C18CE190E00E94C1C09C0133
:10453000DC0111961C930E93E7E0F0E01396FC93D8
:10454000EE93129715961C921E9214971796FC9252
:10455000EE9216971996DC92CE92189758961C9266
:104560002AA73BA70E94AE572AA53BA5D9012D92A9
:104570003C923093261320932513C9010E943D6D70
:104580008824839423C180912A13882309F41EC1AF
:1045900071101CC18CE190E00E94C1C09C01FC0123
:1045A0001183008386E090E09383828315821482D6
:1045B000F782E682D186C086108EC9012AA73BA762
:1045C0000E94AE572AA53BA5D9012D923C9230936B
:1045D000291320932813C9010E943D6D77247394F9
:1045E000F5C080912D13882309F4F0C06110EEC04E
:1045F0008CE190E00E94C1C09C01FC01118300830A
:1046000085E090E09383828315821482F782E682AC
:10461000D186C086108EC9012AA73BA70E94AE573B
:104620002AA53BA5D9012D923C9230932C132093BF
:104630002B13C9010E943D6D66246394C7C080910D
:104640003013882309F4C2C05110C0C08CE190E03F
:104650000E94C1C09C01FC011183008384E090E0B2
:104660009383828315821482F782E682D186C08684
:10467000108EC9012AA73BA70E94AE572AA53BA5C9
:10468000D9012D923C9230932F1320932E13C90100
:104690000E943D6D5524539499C080913313882313
:1046A00009F494C0411092C08CE190E00E94C1C016
:1046B0009C01FC011183008382E090E0938382835C
:1046C00015821482F782E682D186C086108EC901D7
:1046D0002AA73BA70E94AE572AA53BA5D9012D9238
:1046E0003C923093321320933113C9010E943D6DE7
:1046F000442443946BC080913613882309F466C028
:104700002DA1211163C08CE190E00E94C1C09C01E9
:10471000DC0111961C930E93E1E0F0E01396FC93FC
:10472000EE93129715961C921E9214971796FC9270
:10473000EE9216971996DC92CE92189758961C9284
:104740002AA73BA70E94AE572AA53BA5D9012D92C7
:104750003C923093351320933413C9010E943D6D70
:1047600021E02DA333C080913913882379F1911072
:104770002DC08CE190E00E94C1C09C01DC0111962B
:104780001C930E9313961C921E92129715961C92D0
:104790001E9214971796FC92EE9216971996DC9239
:1047A000CE92189758961C922AA73BA70E94AE5704
:1047B0002AA53BA5F901318220823093381320933A
:1047C0003713C9010E943D6D99249394F3E0AF0E15
:1047D000B11C28E7A216B10409F007CDE8CC82E0AD
:1047E0000E94C440882311F01FA216C081E00E94DD
:1047F000C440882329F082E00E94A84081118AC722
:104800008CE30E940F60892B09F075C78CE30E942E
:104810000F60892B09F075C786E0EBEBFFE0DE0146
:10482000549601900D928A95E1F78091B40F909182
:10483000C40FB090B50F0091B60F1091B70F7091E3
:10484000B80F6091B90F5091BA0F4091C10F2091EC
:10485000C20F3091C30FE091CD06F091CE06FEA3BA
:10486000EDA3A0917613B0917713B9A7A8A7909064
:10487000E70F6090E20FE090DB0FF090DC0F80908C
:10488000E50F7090E40FC090410FD090420F509010
:10489000440F40903F0F3090400FBFA1BB8B8A8FD9
:1048A0009B8FBC8E0D8F1E8F7F8F68A359A34AA349
:1048B0003CA32BA3F2E1AF2EFE017396DE0111960D
:1048C00001900D92AA94E1F7EEE8FBE0F09339062F
:1048D000E0933806EFA1E98388879987BA860B872A
:1048E0001C877D876E875F87488B3A8B298B22E1F7
:1048F000FE013196A9E4B6E001900D922A95E1F708
:10490000992321F0863011F01092510630928C12CA
:1049100040928D1250928A12D0928312C0928212CB
:10492000609278137092871280928612F0928512AC
:10493000E092841290928B1288A599A59093891287
:10494000809388128DA19EA190933B0680933A0696
:1049500087E08093170A1092180A61E00E9466604F
:104960008DE09AE00E945B851092190A10921C0A51
:1049700010921B0A80915406811102C010925506B4
:1049800090915006911105C0811103C01092020B45
:1049900098C08091FD0A9091FE0A0E94EF3B81E051
:1049A0008093020B80914906882359F1813071F080
:1049B0008330C1F488E293E290934B0680934A06D9
:1049C00089E080934E0680E197E217C088EB9BE078
:1049D00090934B0680934A0683E080934E0688E9C5
:1049E0009AE30BC088E893E190934B0680934A06C4
:1049F00086E080934E0680EE9EE290934D06809373
:104A00004C06809150068823E9F18091540660910C
:104A10004E0670E08823C9F0809156068823A9F0DD
:104A200080E090E00E944CBD9B01AC0160E070E032
:104A300088EC92E40E9453BF60933C0670933D065D
:104A400080933E0690933F0625C080E090E00E9450
:104A50004CBD9B01AC0160E070E088EC92E40E94E8
:104A600053BF60933C0670933D0680933E0690933F
:104A70003F061092330610923406109235061092BB
:104A800036061FC010923C0610923D0610923E065C
:104A900010923F0660914F0670E080E090E00E9427
:104AA0004CBD9B01AC0160E070E088EC92E40E9498
:104AB00053BF60933306709334068093350690930A
:104AC0003606109246061092400610923706109253
:104AD00041061092420610924306109244060E942C
:104AE00083905098589AE898809169008C7F8093C1
:104AF000690080918D12882321F080916900826085
:104B000003C080916900836080936900E8980E94E7
:104B1000A96180E090E040E09C01225F314FF90103
:104B2000E955FF4F5081552331F032972081318173
:104B3000232B09F04F5F03968837910569F740935F
:104B40005E06ADE6B6E020E030E082EC282E85E996
:104B5000382E9CE4492E9CE3592E41E2642E4CE30E
:104B6000742E54E3852E5CE3952E65ECA62E65E944
:104B7000B62E46EF5DE707EC15E974EDE72E75E913
:104B8000F72EE0E4CE2EEDE7DE2EC901825F914FD5
:104B9000FC01E955FF4F6081662309F49EC38B55E4
:104BA0009F4FFC0180819181892B09F496C370E0AD
:104BB000FB013197E23AF10508F08FC38827E755EA
:104BC000FF4F8F4F0C94ADC084EF9EE811969C93DD
:104BD0008E9383C382EF9EE811969C938E937DC340
:104BE00080EF9EE811969C938E9377C389EE9EE8A2
:104BF00011969C938E9371C387EE9EE811969C93B9
:104C00008E936BC385E59EE811969C938E9365C346
:104C10008FE59EE811969C938E935FC388E39EE890
:104C200011969C938E9359C384E29EE811969C93AF
:104C30008E9353C385E19EE811969C938E934DC34A
:104C400089EB9DE811969C938E9347C380E79DE87E
:104C500011969C938E9341C383E69DE811969C9395
:104C60008E933BC386E59DE811969C938E9335C346
:104C70008BE49DE811969C938E932FC384E59DE869
:104C800011969C938E9329C38DE49DE811969C9375
:104C90008E9323C38AE29DE811969C938E931DC345
:104CA0008BE19DE811969C938E9317C384E19DE858
:104CB00011969C938E9311C384E09DE811969C936A
:104CC0008E930BC382E09DE811969C938E9305C34F
:104CD00080E498E911969C938E93FFC280E398E953
:104CE00011969C938E93F9C28EE298E911969C934B
:104CF0008E93F3C28CE298E911969C938E93EDC249
:104D00008CE198E911969C938E93E7C28AE198E929
:104D100011969C938E93E1C288E198E911969C9339
:104D20008E93DBC280EA95E911969C938E93D5C24F
:104D30008EE995E911969C938E93CFC28CE995E903
:104D400011969C938E93C9C28AED98E711969C9315
:104D50008E93C3C286E198E911969C938E93BDC24F
:104D600086E098E911969C938E93B7C28EEB96E9F4
:104D700011969C938E93B1C28FE996E911969C93FC
:104D80008E93ABC284E098E911969C938E93A5C252
:104D900085ED97E911969C938E939FC28EEC97E9CF
:104DA00011969C938E9399C28DE997E911969C93E5
:104DB0008E9393C28DEF9EE811969C938E938DC235
:104DC0008CE997E911969C938E9387C28BE997E9BA
:104DD00011969C938E9381C289E997E911969C93D1
:104DE0008E937BC281E897E911969C938E9375C24E
:104DF00089E697E911969C938E936FC287E997E9AC
:104E000011969C938E9369C28FE797E911969C93B4
:104E10008E9363C287E697E911969C938E935DC249
:104E200085E997E911969C938E9357C28DE797E990
:104E300011969C938E9351C285E697E911969C93A7
:104E40008E934BC283E997E911969C938E9345C24A
:104E50008BE797E911969C938E933FC283E697E97F
:104E600011969C938E9339C281E997E911969C9390
:104E70008E9333C289E797E911969C938E932DC246
:104E800081E697E911969C938E9327C28FE897E964
:104E900011969C938E9321C287E797E911969C9374
:104EA0008E931BC28FE597E911969C938E9315C242
:104EB0008DE897E911969C938E930FC285E797E949
:104EC00011969C938E9309C28DE597E911969C9358
:104ED0008E9303C28BE897E911969C938E93FDC144
:104EE00083E797E911969C938E93F7C18BE597E939
:104EF00011969C938E93F1C189E897E911969C9342
:104F00008E93EBC181E797E911969C938E93E5C14F
:104F100089E597E911969C938E93DFC187E897E91D
:104F200011969C938E93D9C18FE697E911969C9325
:104F30008E93D3C187E597E911969C938E93CDC14B
:104F400085E897E911969C938E93C7C18DE697E902
:104F500011969C938E93C1C185E597E911969C9318
:104F60008E93BBC183E897E911969C938E93B5C14C
:104F70008BE697E911969C938E93AFC183E597E9F1
:104F800011969C938E93A9C181EE95E911969C93FD
:104F90008E93A3C180E597E911969C938E939DC152
:104FA0008DE497E911969C938E9397C18AE497E9D3
:104FB00011969C938E9391C187E497E911969C93E7
:104FC0008E938BC184E497E911969C938E9385C14F
:104FD00081E497E911969C938E937FC18EE397E9C4
:104FE00011969C938E9379C18BE397E911969C93CC
:104FF0008E9373C182E397E911969C938E936DC152
:105000008AE995E911969C938E9367C188E995E9A1
:1050100011969C938E9361C183E097E911969C93BE
:105020008E935BC18BEF95E911969C938E9355C13E
:1050300089E297E911969C938E934FC186E995E991
:1050400011969C938E9349C184E995E911969C939E
:105050008E9343C18DED96E911969C938E933DC13D
:105060008DE496E911969C938E9337C181EE9EE76D
:1050700011969C938E9331C186E99EE711969C937D
:105080008E932BC18EE79CE311969C938E9325C142
:105090008AE69CE311969C938E931FC186E59CE360
:1050A00011969C938E9319C186E49FE811969C9368
:1050B0008E9313C185E89FE711969C938E930DC143
:1050C00088E79FE711969C938E9307C182E69FE73E
:1050D00011969C938E9301C18EE29DE711969C934D
:1050E0008E93FBC084EE9CE711969C938E93F5C043
:1050F00086E09DE711969C938E93EFC086EF9CE728
:1051000011969C938E93E9C088E19DE711969C933C
:105110008E93E3C08CEB9CE711969C938E93DDC03D
:105120008CEA9CE711969C938E93D7C08EEC9CE7FB
:1051300011969C938E93D1C08AE89EE711969C931A
:105140008E93CBC08EE79EE711969C938E93C5C03D
:1051500082E79EE711969C938E93BFC086E69EE7FA
:1051600011969C938E93B9C08AE59EE711969C9305
:105170008E93B3C08EE49EE711969C938E93ADC040
:1051800082E49EE711969C938E93A7C08CEA9DE7DC
:1051900011969C938E93A1C08AE99DE711969C93EA
:1051A0008E939BC088E89DE711969C938E9395C043
:1051B00086E79DE711969C938E938FC084E69DE7CA
:1051C00011969C938E9389C082E59DE711969C93DE
:1051D0008E9383C01196DC92CE927FC01196FC9282
:1051E000EE927BC011961C930E9377C08CE19EE7E4
:1051F00011969C938E9371C011965C934E936DC0E3
:105200001196BC92AE9269C011969C928E9265C026
:1052100011967C926E9261C011965C924E925DC026
:1052200011963C922E9259C0EFEBF5E91196FC9342
:10523000EE9353C086EB95E911969C938E934DC0E7
:10524000E3EBF5E91196FC93EE9347C080EB95E90B
:1052500011969C938E9341C0E0EAFFE71196FC9370
:10526000EE933BC08DE99FE711969C938E9335C0DA
:10527000E2E9FFE71196FC93EE932FC08BE99FE7DD
:1052800011969C938E9329C0E4E9FFE71196FC9355
:10529000EE9323C088ED9DE711969C938E931DC0DD
:1052A000EBECFDE71196FC93EE9317C08EEB9DE7B8
:1052B00011969C938E9311C0E0E5FFE71196FC9345
:1052C000EE930BC08EE39FE711969C938E9305C0DF
:1052D000ECE2FFE71196FC93EE932D5F3F4F1296A1
:1052E0002837310509F051CC10926106809165068E
:1052F000811114C080E090E0FC01ED54F14F208159
:105300003181245631092436310528F00396883737
:10531000910591F703C081E08093610610926706C2
:1053200080916B06811114C080E090E0FC01ED5487
:10533000F14F20813181285C31092436310528F074
:1053400003968837910591F703C081E08093670643
:105350008091CD069091CE06DC01ED91FC91EE5A44
:10536000FF4F20918E0F30918F0F40918C0F5091F5
:105370008D0F0190F081E02D61E019958091CD06AF
:105380009091CE06DC01ED91FC91EE5AFF4F2091F9
:10539000920F3091930F4091900F5091910F019087
:1053A000F081E02D62E019958091CD069091CE06B6
:1053B000DC01ED91FC91EE5AFF4F2091960F309158
:1053C000970F4091940F5091950F0190F081E02D2F
:1053D00063E019958091CD069091CE06DC01ED91A8
:1053E000FC91EE5AFF4F2091A10F3091A20F4091F6
:1053F0009F0F5091A00F0190F081E02D64E019956E
:105400008091CD069091CE06DC01ED91FC91EE5A93
:10541000FF4F2091A50F3091A60F4091A30F5091FF
:10542000A40F0190F081E02D65E019958091CD06E3
:105430009091CE06DC01ED91FC91EE5AFF4F209148
:10544000A90F3091AA0F4091A70F5091A80F01907A
:10545000F081E02D66E019958091CD069091CE0601
:10546000DC01ED91FC91EC5AFF4F0190F081E02DB1
:105470004091980F61E019958091CD069091CE06EC
:10548000DC01ED91FC91EC5AFF4F0190F081E02D91
:105490004091990F62E019958091CD069091CE06CA
:1054A000DC01ED91FC91EC5AFF4F0190F081E02D71
:1054B00040919A0F63E019958091CD069091CE06A8
:1054C000DC01ED91FC91EC5AFF4F0190F081E02D51
:1054D0004091AB0F64E019958091CD069091CE0676
:1054E000DC01ED91FC91EC5AFF4F0190F081E02D31
:1054F0004091AC0F65E019958091CD069091CE0654
:10550000DC01ED91FC91EC5AFF4F0190F081E02D10
:105510004091AD0F66E019958091CD069091CE0631
:10552000DC01ED91FC9102ACF3ADE02D60919C0F9C
:1055300019958091CD069091CE06DC01ED91FC91FC
:1055400006ACF7ADE02D6091B10F19958091CD06B5
:105550009091CE06DC01ED91FC9100A8F1A9E02D1F
:1055600060919D0F19958091CD069091CE06DC013A
:10557000ED91FC9106A8F7A9E02D60919E0F199579
:105580008091CD069091CE06DC01ED91FC91E65B19
:10559000FF4F0190F081E02D4091B20F60E019952E
:1055A0008091CD069091CE06DC01ED91FC91E65BF9
:1055B000FF4F0190F081E02D4091B30F61E019950C
:1055C00080E090E09C01225F314FF901E955FF4FE7
:1055D0004081423731F4329720813181232B09F009
:1055E0009FC003968837910569F70E945890809173
:1055F000CD069091CE06DC01ED91FC91EC59FF4F68
:105600000190F081E02D40E06091AE0F19958091FE
:10561000CD069091CE06DC01ED91FC91EC59FF4F47
:105620000190F081E02D41E06091B00F19958091DB
:10563000CD069091CE06DC01ED91FC91EC59FF4F27
:105640000190F081E02D42E06091AF0F199520911B
:10565000D90F30E0AFEFB0E00E94DFBE24E630E0CB
:1056600040E050E00E9491BE209301138091D80F3A
:1056700081110E94E67A0E94866B0E9488936B01DA
:105680007C0110E011110FC08091D406882359F0DD
:1056900025EE3DE740ED57E060E070E08EE89BE0EE
:1056A0000E94F35411E00E94F86F882351F00E9489
:1056B000017A0E94843F0E948D7A0E94856F0E9429
:1056C0001D7A0E94884C029711F00E94584F0E9448
:1056D00013990E94884C0297A9F60E948893DC01D6
:1056E000CB018C199D09AE09BF098C3B9240A105E5
:1056F000B10540F218C082E00E94C44081110DC083
:1057000085C882E00E94A840882309F485C8A3E0E8
:10571000AFA382C881E08FA37FC892E09FA37CC81B
:105720000E944C9064CF0E94336B0E948D7A8091CE
:10573000160B811102C00E94BC460E945B4C86E39E
:105740000E946961BC01990F880B990B6115710565
:105750008105910511F00E94D3BC27EA3CE748EE91
:1057600053E060E070E08EE89BE0AB960FB6F894F3
:10577000DEBF0FBECDBFDF91CF911F910F91FF9084
:10578000EF90DF90CF90BF90AF909F908F907F90E1
:105790006F905F904F903F902F900C94F3545F92D6
:1057A0006F927F928F929F92AF92BF92CF92DF9231
:1057B000EF92FF920F931F93CF93DF9381E080933B
:1057C000271380932A1380932D1380933013809393
:1057D0003C1380933F139091750F9150953040F09A
:1057E0008093750F61E070E087E691E00E94464586
:1057F0009091750F2DEF290F80912B0F233008F01A
:1058000011C28A3079F03CF4883009F463C08930E1
:1058100009F4C0C1B6C18B3009F4A4C08C3009F4BE
:10582000E6C0AFC184E290E00E94C1C0FC0180915B
:10583000E80F28E030E0338322838824839499247E
:105840009A9495828482AA24AA94B12CB782A682C3
:1058500011861086108ED3E87D2E718E9CEBC92E9A
:1058600097E0D92ED38EC28E26E6E22E24E0F22EC9
:10587000F182E082CDECDFE0D1A3C0A312A283A32A
:10588000F093C306E093C206CF010E940E8884E223
:1058900090E00E94C1C0FC018091E80F29E030E057
:1058A0003383228395828482B782A68211861086F2
:1058B000108E718ED38EC28EF182E082D1A3C0A3EE
:1058C00012A283A3F093C106E093C006CF010E9409
:1058D0000E880EC380E290E00E94C1C0FC0188E007
:1058E00090E0938382838824839499249A94958268
:1058F0008482AA24AA94B12CB782A682118610862B
:10590000108E7AE0D72ED18EACEBEA2EA7E0FA2EDD
:10591000F38EE28ECEE4D4E0D183C083F093C3064D
:10592000E093C206CF010E94636E80E290E00E9485
:10593000C1C0FC0189E090E09383828395828482D8
:10594000B782A68211861086108ED18EF38EE28EDB
:10595000D183C083F093C106E093C006CF010E94BB
:10596000636EC6C289E190E00E94C1C0FC0188E07C
:1059700090E093838283CC24C394DD24DA94D5828F
:10598000C482EE24EA94F12CF782E6821186108616
:10599000108EC2E4D4E0D183C083F093C306E093B9
:1059A000C206CF010E94676D10923C138091750F63
:1059B000843009F09DC289E190E00E94C1C0FC01E1
:1059C00089E090E093838283D582C482F782E68265
:1059D00011861086108ED183C083F093C106E093A8
:1059E000C006CF010E94676D10923F1381C29430B0
:1059F00009F04BC089E190E00E94C1C0EC01B0EF1A
:105A00008B2EB5E09B2E9982888287E090E09B8365
:105A10008A83AA24A394BB24BA94BD82AC82CC24EA
:105A2000CA94D12CDF82CE8219861886188ECE01B8
:105A30000E94AE5726E3E22E24E0F22EF982E8829D
:105A4000D093C306C093C206CE010E949D6C1092F3
:105A5000271389E190E00E94C1C0EC0199828882FD
:105A600086E090E09B838A83BD82AC82DF82CE8217
:105A700019861886188ECE010E94AE57F982E882E8
:105A8000D093C106C093C0064DC0953009F050C0F8
:105A900089E190E00E94C1C0EC0170EF872E75E0B3
:105AA000972E9982888287E090E09B838A83AA243C
:105AB000A394BB24BA94BD82AC82CC24CA94D12CCA
:105AC000DF82CE8219861886188ECE010E94AE57CC
:105AD000A6E3EA2EA4E0FA2EF982E882D093C1066A
:105AE000C093C006CE010E949D6C1092271389E1DD
:105AF00090E00E94C1C0EC019982888286E090E02B
:105B00009B838A83BD82AC82DF82CE82198618860F
:105B1000188ECE010E94AE57F982E882D093C30658
:105B2000C093C206CE010E949D6C10922A13E0C160
:105B300089E190E00E94C1C0EC0180EF95E099837B
:105B4000888387E090E09B838A8381E09FEF9D8339
:105B50008C838FEF90E09F838E8319861886188E32
:105B6000CE010E94AE5786E394E099838883D09358
:105B7000C306C093C206CE010E949D6C10922713EB
:105B8000B7C189E080932B0F69E070E08DE191E06F
:105B90000E94464580E290E00E94C1C0FC0188E07E
:105BA00090E0938382838824839499249A949582A5
:105BB0008482AA24AA94B12CB782A6821186108668
:105BC000108E50E8D52ED18E6CEBE62E67E0F62EC7
:105BD000F38EE28ECAE5D4E0D183C083F093C3068E
:105BE000E093C206CF010E94B98780E290E00E9454
:105BF000C1C0FC0189E090E0938382839582848216
:105C0000B782A68211861086108ED18EF38EE28E18
:105C1000D183C083F093C106E093C006CF010E94F8
:105C2000B98766C18A3009F458C03CF4883009F459
:105C3000A2C0893009F405C1FBC08B3009F4BEC095
:105C40008C3009F0F5C089E190E00E94C1C0EC0100
:105C500080EF882E85E0982E9982888287E090E0F8
:105C60009B838A83AA24A394BB24BA94BD82AC826A
:105C7000CC24CA94D12CDF82CE8219861886188E45
:105C8000CE010E94AE5736E3E32E34E0F32EF982C4
:105C9000E882D093C506C093C40689E190E00E94D3
:105CA000C1C0EC019982888286E090E09B838A8360
:105CB000BD82AC82DF82CE8219861886188ECE0114
:105CC0000E94AE57F982E882D093C706C093C606F9
:105CD0001092271310922A13F5C084E290E00E94DC
:105CE000C1C0FC017090E80F6090810F88E090E0E7
:105CF000938382838824839499249A9495828482BE
:105D0000AA24AA94B12CB782A68211861086108E7E
:105D100083E8582E518E9CEBC92E97E0D92ED38E56
:105D2000C28E26E6E22E24E0F22EF182E082CDEC55
:105D3000DFE0D1A3C0A362A273A2F093C506E093F3
:105D4000C40684E290E00E94C1C0FC0189E090E0BA
:105D50009383828395828482B782A682118610867D
:105D6000108E518ED38EC28EF182E082D1A3C0A359
:105D700062A273A2A3C080E290E00E94C1C0FC01B5
:105D800088E090E0938382838824839499249A9472
:105D900095828482AA24AA94B12CB782A682118605
:105DA0001086108EAAE0DA2ED18EBCEBEB2EB7E077
:105DB000FB2EF38EE28ECEE4D4E065C089E190E064
:105DC0000E94C1C0FC0188E090E093838283CC24D0
:105DD000C394DD24DA94D582C482EE24EA94F12CB3
:105DE000F782E68211861086108EC2E4D4E0D18359
:105DF000C083F093C506E093C40689E190E00E9459
:105E0000C1C0FC0189E090E093838283D582C48283
:105E1000F782E68211861086108ED183C083F093BC
:105E2000C706E093C60610923C1310923F134AC077
:105E300089E080932B0F69E070E08DE191E00E9492
:105E4000464580E290E00E94C1C0FC0188E090E0FD
:105E5000938382838824839499249A94958284825C
:105E6000AA24AA94B12CB782A68211861086108E1D
:105E7000A0E8DA2ED18EBCEBEB2EB7E0FB2EF38E32
:105E8000E28ECAE5D4E0D183C083F093C506E093E7
:105E9000C40680E290E00E94C1C0FC0189E090E06D
:105EA0009383828395828482B782A682118610862C
:105EB000108ED18EF38EE28ED183C083F093C7060D
:105EC000E093C6068091C6069091C706DC01ED916D
:105ED000FC910280F381E02D19958091C406909188
:105EE000C506DC01ED91FC910280F381E02D19954E
:105EF0008091750F833039F0823009F06CC0809149
:105F00002B0F8C3051F189E190E00E94C1C0EC016F
:105F100080EF95E09983888386E090E09B838A8375
:105F200081E09FEF9D838C838FEF90E09F838E8332
:105F300019861886188ECE010E94AE5786E394E02B
:105F400099838883D093BE06C093BD06CE010E947C
:105F50009D6C10922A13C6E029C089E190E00E944E
:105F6000C1C0EC0180EF95E09983888384E090E0E4
:105F70009B838A8381E09FEF9D838C838FEF90E0EA
:105F80009F838E8319861886188ECE010E94AE5785
:105F900086E394E099838883D093BE06C093BD06C0
:105FA000CE010E949D6C10923013C4E060913A0FB4
:105FB00070913B0F8C2F0E94C75660913C0F7091DF
:105FC0003D0F8C2F0E94C35680913E0FE091BD067D
:105FD000F091BE06808FE0912C0F8E2FEE0F990B63
:105FE000AA0BBB0BFC013897E830F10508F0BBC0E9
:105FF0008827E55BFE4F8F4F0C94ADC084E290E0A4
:106000000E94C1C0FC018091E80F28E030E033839A
:10601000228321E03FEF358324832FEF30E0378365
:10602000268311861086108E94E8918F2CEB37E032
:10603000338F228F26E634E0318320832DEC3FE03E
:1060400031A320A312A283A31EC080E290E00E948D
:10605000C1C0FC0188E090E09383828381E09FEFE0
:10606000958384838FEF90E09783868311861086D3
:10607000108E87E8818F8CEB97E0938F828F8AE573
:1060800094E091838083F093CC06E093CB0699C093
:1060900080E290E00E94C1C0FC0188E090E0938320
:1060A000828381E09FEF958384838FEF90E09783D5
:1060B000868311861086108E8DE0818F8CEB97E0A1
:1060C000938F828F8EE494E0DCCF89E190E00E9490
:1060D000C1C0FC0188E090E09383828381E09FEF60
:1060E000958384838FEF90E0978386831186108653
:1060F000108E82E494E091838083F093CC06E09349
:10610000CB0610923C135DC08CE190E00E94C1C0B0
:10611000EC0180EF95E09983888385E090E09B8394
:106120008A8381E09FEF9D838C838FEF90E09F8334
:106130008E8319861886188ECE010E94AE5784EE83
:1061400095E037C089E190E00E94C1C0FC01138254
:106150001282158214821782168211861086108E82
:106160008EE194E08ECF8CE080932C0F6CE070E099
:106170008EE191E00E94464589E190E00E94C1C015
:10618000EC0180EF95E09983888385E090E09B8324
:106190008A8381E09FEF9D838C838FEF90E09F83C4
:1061A0008E8319861886188ECE010E94AE5786E31C
:1061B00094E099838883D093CC06C093CB06109249
:1061C0002D138091CB069091CC06DC01ED91FC91D2
:1061D0000280F381E02D19958091340F843658F4B4
:1061E000853608F084E664E6681B8091CB069091C2
:1061F000CC060E94B98880912C0F8C508230A8F474
:106200006091350F7091360F85E00E94F9556091CD
:10621000370F7091380F85E00E94DE558091390F5D
:10622000E091CB06F091CC06808F20912D0F822F2C
:10623000022E000C990BAA0BBB0BFC013897E8301F
:10624000F10508F089C08827ED5AFE4F8F4F0C9456
:10625000ADC084E290E00E94C1C0FC018091E80FD3
:1062600029E030E03383228321E03FEF358324832C
:106270002FEF30E03783268311861086108E94E846
:10628000918F2CEB37E0338F228F26E634E0318379
:1062900020832DEC3FE031A320A312A283A357C09B
:1062A00080E290E00E94C1C0FC0189E090E093830D
:1062B000828381E09FEF958384838FEF90E09783C3
:1062C000868311861086108E87E8818F8CEB97E08D
:1062D000938F828F8AE594E038C080E290E00E943C
:1062E000C1C0FC0189E090E09383828381E09FEF4D
:1062F000958384838FEF90E0978386831186108641
:10630000108E8DE0818F8CEB97E0938F828F8EE4DF
:1063100094E01BC08091750F823009F0C5C2809156
:106320002B0F8C3009F0C0C21FC089E190E00E94A1
:10633000C1C0FC0113821282158214821782168258
:1063400011861086108E8EE194E091838083F09305
:10635000D006E093CF065EC08091750F823061F564
:1063600080912B0F8C3041F58BE080932D0F6BE0EB
:1063700070E08FE191E00E94464589E190E00E9443
:10638000C1C0FC0189E090E09383828381E09FEFAC
:10639000958384838FEF90E09783868311861086A0
:1063A000108E82E494E091838083F093D006E09392
:1063B000CF0610923F132EC08CE080932D0F6CE01F
:1063C00070E08FE191E00E94464589E190E00E94F3
:1063D000C1C0EC0180EF95E09983888384E090E070
:1063E0009B838A8381E09FEF9D838C838FEF90E076
:1063F0009F838E8319861886188ECE010E94AE5711
:1064000086E394E099838883D093D006C093CF0627
:10641000109230138091CF069091D006DC01ED915F
:10642000FC910280F381E02D19958091330F843621
:1064300058F4853608F084E664E6681B8091CF0640
:106440009091D0060E94B98880912D0F8C50823097
:1064500000F560912E0F70912F0F84E00E94F95586
:106460006091300F7091310F84E00E94DE55809171
:10647000320FE091CF06F091D006808F80912D0FE2
:106480008D3039F48091320FE0919112F091921297
:10649000808F8EE190E00E94C1C0EC01D090430F4C
:1064A000A090470FB090480F8090450F9090460FF6
:1064B00080EF95E09983888383E090E09B838A83D3
:1064C00081E09FEF9D838C83EE24EA94F12CFF8280
:1064D000EE8219861886188ECE010E94AE578AE287
:1064E00094E0998388839A8E898EBC8EAB8EDD8EE4
:1064F000D0937713C09376136091490F70914A0F30
:1065000083E00E94F95560914B0F70914C0F83E02E
:106510000E94DE558091430FE0917613F09177133E
:10652000808F8091430F0E94114580917613909146
:106530007713DC01ED91FC910280F381E02D199538
:1065400080914E0F8823A1F18BE390E00E94C1C09F
:10655000FC018091580F9091570F20915D0F309161
:106560005E0F40915B0F50915C0F6091590F7091DD
:106570005A0FA091530FB091540FC091510FD09169
:10658000520FC0904F0FD090500F11821082F382A3
:10659000E28215821482D4A2C3A2D6A3C5A3B0A757
:1065A000A7A372A761A754A743A736A725A72FC003
:1065B0008BE390E00E94C1C0FC018091580F909144
:1065C000570F20915D0F30915E0F40915B0F5091FE
:1065D0005C0F6091590F70915A0FA091510FB091BB
:1065E000520FC0914F0FD091500F11821082F38241
:1065F000E28215821482D4A3C3A3B6A3A5A370A775
:1066000067A352A741A734A723A7F6A6E5A62CEBBC
:1066100037E030AB27A72DEC3FE032AB21AB93AB9B
:1066200084ABF0934806E0934706C0914706D091AB
:1066300048062FA138A54BA15CA18DA19EA14217B0
:1066400053071CF4821793077CF0281739071CF4B2
:106650004817590764F0241735075CF48417950729
:1066600044F4142F052F05C0122F032F02C0182F3A
:10667000092F1F821E82188709871B861A861D868E
:106680001C861E870F87198A188A2DA53EA549A545
:106690005AA58BA59CA5421753071CF48217930794
:1066A0007CF0281739071CF44817590764F02417A1
:1066B00035075CF48417950744F4142F052F05C0A3
:1066C000122F032F02C0182F092F1B8A1A8A1C8B26
:1066D0000D8B1F8A1E8A198E188E1A8F0B8F1D8E96
:1066E0001C8E1AAE19AE18A28BA9813069F08230C7
:1066F000E9F0811183C061E08CE20E946660109233
:106700002D0110922C017AC061E08CE20E9466603B
:1067100010922D0110922C0161E088E00E946660C9
:1067200060E070E088E00E94A26068C0E9A9FAA970
:1067300080819181A281B38181159649A105B1051E
:1067400009F457C040E056E960E070E08FA598A9D1
:106750000E943A7364E170E080E090E00E94509300
:10676000E9A9FAA980819181A281B38181152BE4E5
:106770009207A105B105E9F068F4803629E0920797
:10678000A105B105A1F080389542A105B105C1F47C
:1067900042E012C0811521EE9207A105B10559F022
:1067A0008115924CA140B10559F445E005C041E086
:1067B00003C043E001C046E06FE0CE010E94B55245
:1067C0008FA598A9DC01ED91FC910680F781E02D61
:1067D0001995E9A9FAA940815181628173818FA538
:1067E00098A90E943A7364E170E080E090E00E9412
:1067F00050934AE06EE0CE010E94B55280913C1366
:106800008823F9F089E190E00E94C1C0FC0188E092
:1068100090E093838283158214828FEF93E09783B5
:1068200086838FEF91E091878087108E82E494E0D9
:1068300091838083F0933B13E0933A13CF010E943E
:10684000676D80913F13882309F478C089E190E057
:106850000E94C1C0FC0189E090E09383828315828D
:1068600014828FEF93E0978386838FEF91E0918777
:106870008087108E82E494E091838083F0933E13AE
:10688000E0933D13CF01DF91CF911F910F91FF90C6
:10689000EF90DF90CF90BF90AF909F908F907F90C0
:1068A0006F905F900C94676D2C3009F48ECD8CE165
:1068B00090E00E94C1C0EC0190EF692E95E0792E26
:1068C0007982688224E0822E912C9B828A82AA247B
:1068D000A394BB24BA94BD82AC82CC24CA94D12C9C
:1068E000DF82CE8219861886188ECE010E94AE579E
:1068F00054EEE52E55E0F52EF982E882D093D006CD
:10690000C093CF068CE190E00E94C1C0EC01798277
:1069100068829B828A82BD82AC82DF82CE821986A7
:106920001886188E0E94AE57F982E882D093921290
:10693000C0939112CE010E943D6D6ACDDF91CF913F
:106940001F910F91FF90EF90DF90CF90BF90AF908D
:106950009F908F907F906F905F9008952F923F92BD
:106960004F925F926F927F928F929F92AF92BF925F
:10697000CF92DF92EF92FF920F931F93CF93DF930B
:10698000CDB7DEB7C65AD1090FB6F894DEBF0FBE39
:10699000CDBFCDB6DEB6CC55DF4F1882C45AD0403D
:1069A000CD55DF4F1882C35AD0408091D20D8A371F
:1069B00009F447C0C0F4873709F4D9C238F48F31DD
:1069C00009F435C5863709F4E2C1F7C5883709F4FB
:1069D000DDC2893709F0F1C50E94C1590E94889330
:1069E0002B013C0129C08E3709F42EC338F48B37B4
:1069F00009F4CAC18C3709F4D8C2DFC5813809F45B
:106A000007C5823809F4EDC4803809F0D6C565C4DD
:106A10000E948893DC01CB0184199509A609B70966
:106A200080329340A105B10508F00CC50E94584F73
:106A30000E94C1590E94569B0E94884C029741F7C0
:106A400001C50E94884C029729F060E084E80E940A
:106A5000189C8BC18091170B823031F0833039F450
:106A600082E08093D31103C081E080933F1281E0E4
:106A70008093DC0D8E010C551F4F2BE0AE01445767
:106A80005F4F68E871E90E94929B0E945B4C8930DD
:106A900058F0015011092BE0AE014F575F4F68E8E5
:106AA00072E981E00E94929B1092DB0D772473942F
:106AB0000E94714C882309F43DC1198222961FAEB1
:106AC00022971091DB0D11110EC0BE0164577F4F4C
:106AD000CE018F5B9F4F0E94DFC2CC55DF4F0881F4
:106AE000C45AD04011C0113071F4BE016F577F4FAE
:106AF000CE018F5B9F4F0E94DFC2CD55DF4F0881D3
:106B0000C35AD04001C000E0ADB6BEB68091130BB1
:106B1000EDB7FEB722E0829FE019F10911240FB60C
:106B2000F894FEBF0FBEEDBF8DB79EB701967C01F6
:106B300068E276E0CE0183569F4F0E94805C809190
:106B4000170B823089F0833061F1813009F0A1C0E8
:106B50004091130B50E0B7018091111290911212E5
:106B60000E944E9A10E039C02091130B30E05FB7BD
:106B7000F89440E0842F90E08217930774F4880F14
:106B8000991FF701E80FF91FDC01A25EBD4E8D9140
:106B90009C91918380834F5FEDCF5FBF10923E1237
:106BA0001CC02091130B30E05FB7F89440E0842FB5
:106BB00090E08217930774F4880F991FF701E80F8C
:106BC000F91FDC01A451BE4E8D919C91918380836D
:106BD0004F5FEDCF5FBF10920E126DE270E0CE01FD
:106BE00083569F4F0E94AF5B2091130B293048F0D2
:106BF000112321F0113021F418E004C028E001C075
:106C000020E010E0121758F5F701E10FF11DE10F38
:106C1000F11D608171814AE0CE0189569F4FCB55AD
:106C2000DF4F2883C55AD0400E94555CBE0169568B
:106C30007F4FCE0183569F4F0E94D65BCE0189566F
:106C40009F4F0E94505CCE0183569F4F0E9469481F
:106C50001F5FCB55DF4F2881C55AD040D3CF40E4CA
:106C600050E0BE016F5F7F4FCE0183569F4F0E9461
:106C70006148CF55DF4F1881C15AD040CE018356AD
:106C80009F4F0E94505C0FB6F894BEBE0FBEADBEC3
:106C90000BC0CE0183569F4F0E94505C0FB6F894F4
:106CA000BEBE0FBEADBE10E0BE016F5F7F4FCE0116
:106CB0008F5B9F4F0E94DFC2010F10E0E1E4F0E024
:106CC000EC0FFD1FE00FF11F1082BE016F5B7F4FC5
:106CD0008091A2139091A3130E94E35CB801CE01AE
:106CE0008F5B9F4F0E94729BBC018091A213909179
:106CF000A3130E9437466AE08091A2139091A313D8
:106D00000E94B85C8091A2139091A313DC01ED91D5
:106D1000FC910680F781E02D19950E945B4C89302B
:106D200048F08091DB0D811103C07092DB0D02C031
:106D30001092DB0D0E94C1590E94569B0E94866EE4
:106D400081110CDE8091D10D81110FC08091DC0D7D
:106D5000882359F08091A413811107C08091CF0D31
:106D60009091D00D0A970CF4A3CE8091170B82302E
:106D700039F0833009F021C481E08093D3111DC420
:106D800081E080933F1219C41092DC0D4DC3109125
:106D9000D50D8FEF810F853028F060E089E80E94E3
:106DA000189C0BC4133079F018F41230F9F004C0B9
:106DB000143079F0153099F040E6442E49E0542E15
:106DC000612C712C19C0412C3BE4532E612C712C89
:106DD00013C0412C26E9522E612C712C0DC0412C80
:106DE00092EC592E66246394712C06C080E8482EDC
:106DF00085E2582E612C712C00E0E12EF12C570118
:106E0000BFE8AB0EB11C1501E89427F83324E6E97E
:106E1000EE0EF11CE894E7F8FF24023091F018F42C
:106E2000013051F004C0033089F00430A1F040E695
:106E300059E060E070E013C040E855E260E070E0C7
:106E40000EC040E05BE460E070E009C040E056E95D
:106E500060E070E004C040E052EC61E070E08CEB78
:106E600097E00E943A738CEB97E00E94D45A0E94FC
:106E700088934B015C01F2E38F0E911CA11CB11CA5
:106E80000E94199B0E948893681579058A059B05C5
:106E9000B8F360E870E08CEB97E00E9477706FE0E9
:106EA00070E08CEB97E00E947770612F8CEB97E09D
:106EB0000E948E5AB1018CEB97E00E9477700E947D
:106EC00088934B015C012AE0820E911CA11CB11C2D
:106ED0000E94199B0E948893681579058A059B0575
:106EE000B8F367E870E08CEB97E00E9477706FE092
:106EF00070E08CEB97E00E947770612F8CEB97E04D
:106F00000E948E5AB7018CEB97E00E9477708CEB51
:106F100097E00E94D45A0E9488934B015C013EE5A1
:106F2000830E31E0931EA11CB11C0E94199B0E948C
:106F30008893681579058A059B05B8F30F5F0530BE
:106F400009F06BCFB301A2018CEB97E00E943A737A
:106F50004092CD0F5092CE0F6092CF0F7092D00F13
:106F6000B301A2018FEB91E00E949C485DC283E0D7
:106F700090E00E94C1C02AE0DC012C932CEB37E0AA
:106F800012963C932E9311976AE00CC083E090E038
:106F90000E94C1C02DE0FC0120832CEB37E032833E
:106FA00021836DE00E9412513FC24091D50D509156
:106FB000D60D0091D70D1091D80D6091D30D709121
:106FC000D40DCE010196CB55DF4F4883C55AD04032
:106FD000CA55DF4F5883C65AD0400E94FF83CB5515
:106FE000DF4F4881C55AD040CA55DF4F5881C65A35
:106FF000D040892BE9F08D81873050F4853080F4C2
:107000008130B0F0642F8B819C810E94A2460DC01C
:10701000893070F4B8018B819C810E949C4805C026
:10702000BA018B819C810E9446450E94939C04C0BA
:1070300061E085E80E94189C8091CE0D8111BDC24F
:1070400081E08093CE0DB9C2B090D30DE090D40D05
:10705000C956DF4F1882C759D04068E276E0CE01AA
:107060008F579F4F0E94805C6B2D7E2DCE018457E1
:107070009F4F0E94FF83892B09F4C9C0C057DF4F7F
:10708000E881C059D0404E2F50E0FA013197E830E6
:10709000F10508F0BCC08827E55AFE4F8F4F0C94CD
:1070A000ADC0C257DF4F88819981CE58D0400E9431
:1070B00071BE23961FAE1EAE239725961FAE1EAE41
:1070C000259727961FAE1EAE27974AE0BE016F5F39
:1070D0007F4F90E03EC0C257DF4F88819981CE58E4
:1070E000D0400E9471BE682F880F770B4AE00AC01B
:1070F000C257DF4F88819981CE58D0400E947EBE12
:107100004AE0BC01CE0101960E94555CBE016F5F52
:107110007F4FCE018F579F4F0E94765BCE01019625
:1071200063C0C257DF4F88819981CE58D0400E94FA
:107130007EBE23961FAE1EAE239725961FAE1EAEB3
:10714000259727961FAE1EAE27974AE0BE016F5FB8
:107150007F4F0E941FBD35C0C257DF4F8881998184
:10716000CE58D0400E9479BE23961FAE1EAE239704
:1071700025961FAE1EAE259727961FAE1EAE2797EB
:107180002AE0AE014F5F5F4F0E94F0BC1AC0C257A9
:10719000DF4F88819981CE58D0400E9479BE2396D6
:1071A0001FAE1EAE239725961FAE1EAE25972796BF
:1071B0001FAE1EAE27972AE0AE014F5F5F4F0E94C1
:1071C000FEBCBE016F5F7F4FCE018F5B9F4F0E9461
:1071D000305CBE016F5B7F4FCE018F579F4F0E9487
:1071E000765BCE018F5B9F4F0E94505C4BE050E07E
:1071F000BE016F5B7F4FCE018F579F4F0E9461484A
:10720000CB57DF4FF880C558D04011E002C0F12CB9
:1072100010E0CE018F579F4F0E94505C112309F45C
:10722000BCCD8E0109561F4F20E4AE014F5F5F4F6A
:1072300068E87B2D8E2D0E94929BBE016F5B7F4F75
:10724000CE0101960E94DFC2C956DF4F8881C7591F
:10725000D040F80E81E08F0DC956DF4F8883C759A3
:10726000D040E1E0F0E0EC0FFD1FEF0DF11D9CE7D9
:107270009083E1E0F0E0EC0FFD1FE80FF11D1082BC
:10728000BE016F5F7F4F8091A2139091A3130E9464
:10729000E35CC956DF4F6881C759D04070E0CE012A
:1072A00001960E94729BBC018091A2139091A3133E
:1072B0000E9437466AE08091A2139091A3130E9426
:1072C000B85C8091A2139091A313DC01ED91FC9125
:1072D0000680F781E02D199570C18091D30D9091B2
:1072E000D40D8038910509F068C18E0104571F4FF5
:1072F00020E4AE014F5F5F4F68E870E880E00E94D5
:10730000929B68EF75E0CE018F579F4F0E94805C83
:10731000CE018F579F4F0E946948C457DF4F288185
:10732000CC58D040CB57DF4F88819981C558D04089
:10733000820F911DC457DF4F8883CC58D0402296CE
:107340001FAE22974BE050E0BE016F5B7F4FCE0136
:107350008F579F4F0E943E48BE016F5B7F4FCE010B
:1073600001960E94DFC2C457DF4F8881CC58D040BD
:10737000E1E0F0E0EC0FFD1FE80FF11D1082BE010F
:107380006F5F7F4F8091A2139091A3130E94E35CE3
:10739000C457DF4F6881CC58D04070E0CE010196D1
:1073A0000E94729BBC018091A2139091A3130E9432
:1073B00037466AE08091A2139091A3130E94B85CB3
:1073C0008091A2139091A313DC01ED91FC910680B2
:1073D000F781E02D1995CE018F579F4F0E94505C89
:1073E000ECC08091D30D9091D40D8238910509F0B5
:1073F000E4C08E0104571F4F20E4AE014F5F5F4F82
:1074000068E872E880E00E94929B62E176E07BCFC0
:107410008091D30D9091D40D8138910509F0CDC0A4
:107420008091DC0D8111C9C00E94939CC6C08091DF
:10743000D30D9091D40D4F9709F0BFC081E0809398
:10744000D10DBBC00E94884C029719F060E084E81F
:10745000A6CC8091160B811102C00E94BC460E94EE
:107460005B4CF82E68E276E0CE0184579F4F0E9475
:10747000805CC956DF4F1882C759D0408E0109562B
:107480001F4F20E4AE014F5F5F4F68E879E780E06F
:107490000E94929BCF57DF4F19821882C158D0406B
:1074A000CD57DF4F19821882C358D040CB57DF4FDA
:1074B00019821882C558D0406F2D70E080E090E0AE
:1074C0002AE0AE014F5B5F4F0E94F0BCBE016F5BD4
:1074D0007F4FCE018F579F4F0E94305CBE016F5788
:1074E0007F4FCE0184579F4F0E94765BCE018F570E
:1074F0009F4F0E94505C4BE050E0BE016F5B7F4F9E
:10750000CE0184579F4F0E943E48C057DF4F1881DD
:10751000C059D040BE016F5B7F4FCE0101960E94E3
:10752000DFC2C956DF4F8881C759D040810F91E033
:10753000980FC956DF4F9883C759D040E1E0F0E07B
:10754000EC0FFD1FE80FF11D8CE78083E1E0F0E018
:10755000EC0FFD1FE90FF11D1082BE016F5F7F4F21
:107560008091A2139091A3130E94E35CC956DF4F50
:107570006881C759D04070E0CE0101960E94729B8D
:10758000BC018091A2139091A3130E9437466AE038
:107590008091A2139091A3130E94B85C8091A213D2
:1075A0009091A313DC01ED91FC910680F781E02D11
:1075B0001995CE0184579F4F11CF0FB6F894DEBEB8
:1075C0000FBECDBECA55DF4F0FB6F894DEBF0FBE5B
:1075D000CDBFDF91CF911F910F91FF90EF90DF9082
:1075E000CF90BF90AF909F908F907F906F905F9063
:1075F0004F903F902F9008951092FB0A0895FC0140
:1076000012821382148215821682178212860895BE
:1076100080E008950F931F93CF938C016AEA70E185
:1076200086EF98E00E94BF5CD8011896ED91FC911E
:1076300019976081718186EF98E02FD7C1E0D8015A
:107640001A968C91C81708F565EA70E186EF98E004
:107650000E94BF5C6C2F86EF98E00E940A4562EAA8
:1076600070E186EF98E00E94BF5CF801908581850B
:10767000E92FF82FEC0FF11DEC0FF11D60817181E6
:1076800086EF98E00AD7CF5FDACFCF911F910F91A5
:1076900008951F920F920FB60F9211240BB60F92FE
:1076A0001F932F933F934F935F936F937F938F938A
:1076B0009F93AF93BF93EF93FF93CF93DF9300D04C
:1076C0001F92CDB7DEB780918D0A0E940F6011E046
:1076D000892B09F010E00E942B9369837A838B83B6
:1076E0009C8389819A81AB81BC814091910A5091A0
:1076F000920A6091930A7091940A841B950BA60BD1
:10770000B70B20918E0A30918F0A2430310509F48D
:107710004CC02530310521F021303105E9F414C089
:107720002091900A222339F02091FB0A20FF02C009
:10773000289A01C02898112379F0813E2EE2920701
:10774000A105B10548F02BC0112379F125E030E007
:1077500030938F0A20938E0A20918E0A30918F0ADF
:107760002530310511F5E091FB0AF0E0EE0FFF1F27
:10777000EB56F54F9183808389819A81AB81BC81DF
:107780008093910A9093920AA093930AB093940ADB
:107790008091FB0A8F5F8093FB0A833330F084E093
:1077A00090E090938F0A80938E0A0F900F900F9025
:1077B0000F90DF91CF91FF91EF91BF91AF919F918A
:1077C0008F917F916F915F914F913F912F911F9179
:1077D0000F900BBE0F900FBE0F901F901895CF9378
:1077E000DF93EC0180918D0A62E00E946660E8817F
:1077F000F9810190F081E02DCE01DF91CF911994B4
:107800008091CD069091CE06DC01ED91FC91008433
:10781000F185E02D19958091CD069091CE06DC0181
:10782000ED91FC910480F581E02D1994809107027F
:10783000813019F485E08093070208951092C806FC
:10784000089580912F06882371F010922F06809161
:10785000D306882341F06DE972E18091D1069091C1
:10786000D2060C94305E08958091750F833099F0A4
:1078700080912F0681110FC081E080932F068091A7
:10788000D306882341F068E872E18091D106909197
:10789000D2060C94305E089580912F06882319F04B
:1078A00080E090E0CECF80E090E0DECF80912E06A9
:1078B000833079F083E080932E068091D30688236D
:1078C00041F067E772E18091D1069091D2060C9465
:1078D000305E089580912E06823079F082E08093A8
:1078E0002E068091D306882341F066E672E18091EE
:1078F000D1069091D2060C94305E089580912E06A8
:10790000813079F081E080932E068091D306882320
:1079100041F065E572E18091D1069091D2060C9418
:10792000305E08958091070181FF1BC08091D306CE
:10793000882351F08BE29BE00E941A87811108C0D6
:107940008091370B811104C08BE29BE00C94078778
:1079500069EC72E18091D1069091D2060E94305E6E
:10796000F3CF08958091070181FF17C08091D3065E
:10797000882331F08BE29BE00E941A87882321F054
:107980008BE29BE00C942E8763EB72E18091D10631
:107990009091D2060E94305EF3CF08950E94AF848A
:1079A00080913006882361F18091010B811128C0FC
:1079B0008091C906811124C081E08093C9060E948C
:1079C0007B9880915B06882319F010925B060CC0AF
:1079D0008091CD069091CE06DC01ED91FC9102885C
:1079E000F389E02D61E019958091D306882341F059
:1079F0006AE272E18091D1069091D2060C94305ED9
:107A000008958091FC0A8823C1F0609174137091ED
:107A100075138EE89BE00E94A45410927513109287
:107A200074131092FC0A809107028130D9F480917E
:107A3000820F8823B9F0FADE15C08091E00D8F5FC8
:107A40008093E00D803580F0609174137091751310
:107A50008EE89BE00E94A454109275131092741348
:107A60001092FC0A1092E00D0895CF93DF9380915D
:107A7000070181FD2AC0C0916206D0916306809102
:107A80006606882371F08FE30E946961813092401D
:107A90002CF010926306109262060AC081E090E01A
:107AA00003C08FE30E94696190936306809362062E
:107AB00080916206909163068C179D0719F41092CD
:107AC000640603C081E080936406DF91CF9108953E
:107AD0008091750F833041F12CF48130A9F0823010
:107AE00099F02DC086305CF58091C2069091C30656
:107AF000DC01ED91FC910480F581E02D19958091D8
:107B0000C0069091C10614C08091C6069091C70628
:107B1000DC01ED91FC910480F581E02D19958091B7
:107B2000C4069091C50604C08091C2069091C30618
:107B3000DC01ED91FC910480F581E02D1995809197
:107B4000CD069091CE06DC01ED91FC91E25BFF4FFA
:107B50000190F081E02D19958091CD069091CE068F
:107B6000DC01ED91FC910484F585E02D60E070E08E
:107B700019940E94AF84809130068823D1F08091BF
:107B8000C9068823B1F01092C9060E9442988091DC
:107B90005B06882389F010925B068091D3068823C8
:107BA00041F06EE372E18091D1069091D2060E947D
:107BB000305E1092C90608958091CD069091CE0650
:107BC000DC01ED91FC910288F389E02D60E01995CC
:107BD000E4CFCF93DF93C091010ED091020EBE018E
:107BE0008EE89BE00E948C54882329F0BE018EE829
:107BF0009BE00E94A4541092020E1092010EDF919D
:107C0000CF9108950F931F93CF93DF9380917A0FB5
:107C100090917B0FA0917C0FB0917D0F18161906E3
:107C20001A061B060CF044C00E94AF8480913006F7
:107C30008823C9F10091010E1091020EB8018EE85F
:107C40009BE00E948C548823D9F0ECE8FDE0C0E072
:107C5000D0E0819191918017910769F40E948893F7
:107C6000CC0FDD1FCC0FDD1FC257D44F6883798343
:107C70008A839B831DC02196CE31D10551F718C050
:107C800040917A0F50917B0F60917C0F70917D0F26
:107C90002EEA3FE38EE89BE00E94F3549093020E9D
:107CA0008093010E05C0DF91CF911F910F9191CF6D
:107CB000DF91CF911F910F910895CF93DF93809122
:107CC000010B8111CFC08091CA06823040F08091B3
:107CD000D306882309F4C6C063EC71E16AC08091C1
:107CE000570F882309F46DC08091580F882309F439
:107CF00068C080915D06811164C0C0914706D09133
:107D0000480689AD9AAD892B11F01AAE19AE8BA930
:107D1000813051F0823081F44FEF60E0CE010E945B
:107D2000B5528FEF90E006C08FEF90E090932D0159
:107D300080932C019F8F8E8F0E9488936DAB7EABBA
:107D40008FAB98AF8091CD069091CE06DC01ED917E
:107D5000FC910284F385E02D199581E080935D0606
:107D60002091580F88EE93E0289FA001299F500D85
:107D70001124052E000C660B770B2DE53EE38EE8F3
:107D80009BE00E94F3548091D306882309F46AC0D3
:107D900061E971E18091D1069091D2060E94BF5CA9
:107DA0006091580F8091D1069091D20633D668E841
:107DB00071E18091D1069091D206DF91CF910C9420
:107DC000305E0E94AF8480914C13882309F44AC02E
:107DD00080913006811146C081E080933006109278
:107DE0004C130E94D6848091DF0D882341F069E70F
:107DF00071E18091DD0D9091DE0D0E94305E109258
:107E00005D0680915F0690916006806190936006A8
:107E100080935F068091CD069091CE06DC01ED91B6
:107E2000FC910280F381E02D19958091CA068111A1
:107E300016C04091700F5091710F81E080935B06E6
:107E40004115510559F060E070E02EEC3CE38EE8FE
:107E50009BE00E94F3540E94429801C09FDDDF9195
:107E6000CF91D0CEDF91CF9108958091010B8111F8
:107E70004AC010925D060E94AF8480914C13882303
:107E8000B1F080913006882391F010923006109264
:107E90004C130E94D6848091DF0D882341F065E069
:107EA00072E18091DD0D9091DE0D0E94305E809137
:107EB0005F069091600680629093600680935F06F3
:107EC0008091C906882311F081E001C080E00E9402
:107ED000B49881E080935B064CDE80918B0F81111A
:107EE0000FC080914606882359F020E03CE344E629
:107EF00050E060E070E08EE89BE00E94F35401C027
:107F00007FDCE6DD7FCE0895E3DD0E9450950E9480
:107F1000AF84809130068111A8DF8091CF069091C7
:107F2000D006DC01ED91FC910480F581E02D1995DE
:107F30008091CB069091CC06DC01ED91FC91048000
:107F4000F581E02D199580914E0F882331F08091B5
:107F50004706909148060C94055308950E94AF84FB
:107F600080913006882369F080DF8091D3068823D2
:107F700041F065E172E18091D1069091D2060C94B6
:107F8000305E0895AF92BF92CF92DF92EF92FF9250
:107F90000F931F93CF93DF939091F90D91110BC025
:107FA0002091D9063091DA063093F80D2093F70D21
:107FB00091E09093F90D9091EF0D91110BC02091EC
:107FC000D7063091D8063093EE0D2093ED0D91E059
:107FD0009093EF0DA090F70DB090F80D0091ED0D7E
:107FE0001091EE0DD091D306843608F046C0C82F0C
:107FF000682F70E080E090E00E944CBD20E030E00F
:1080000048EC52E40E9453BF6B017C01B501BB0CEC
:10801000880B990B0E944EBD9B01AC01C701B601B4
:108020000E94ADBD0E94BBBF7093DA066093D90673
:10803000B801110F880B990B0E944EBD9B01AC013A
:10804000C701B6010E94ADBD0E94BBBF7093D806A8
:108050006093D706DD2369F168E571E18091D1066F
:108060009091D2060E94BF5C6C2F8091D1069091B6
:10807000D206D0D466E571E10CC0B092DA06A092C7
:10808000D9061093D8060093D706DD2391F06AE64F
:1080900071E18091D1069091D206DF91CF911F912D
:1080A0000F91FF90EF90DF90CF90BF90AF900C9426
:1080B000305EDF91CF911F910F91FF90EF90DF9095
:1080C000CF90BF90AF900895CF93823069F4909194
:1080D000690F2091660F30916A0F4091670F5091A0
:1080E000680F6091650F0CC09091630F2091600F35
:1080F0003091640F4091610F5091620F60915F0F5A
:108100006093BB135093B8134093B9133093B713D4
:108110002093BA139093BC13909100028917B1F089
:10812000809300029091D306992381F0C82F6DE3CC
:1081300071E18091D1069091D2060E94BF5C6C2FB4
:108140008091D1069091D206CF914DC4CF910895E0
:10815000833079F030F4813051F0823091F48BE348
:108160000BC0843041F0853061F482E405C08CE3BB
:1081700003C080E401C081E40E940F6021E0892BEC
:1081800009F420E0822F0895E3DF91E08927089524
:108190000F931F938091E50D81110DC00E9488936C
:1081A0006093E10D7093E20D8093E30D9093E40DE5
:1081B00081E08093E50D80910A028A3AF1F485E02E
:1081C000C7DF882371F089E598E09093A31380932B
:1081D000A2139093D2068093D1068FEF80930A0268
:1081E0000CC086EF98E09093A3138093A213909312
:1081F000D2068093D10610920A020E9488930091C1
:10820000E10D1091E20D2091E30D3091E40DDC01C0
:10821000CB01801B910BA20BB30BC397A105B1053A
:1082200008F449C00E9488936093E10D7093E20DB9
:108230008093E30D9093E40D85E08ADF882321F09D
:1082400080910A02882349F085E082DF811133C0E2
:1082500080910A028F3F79F518C089E598E09093E4
:10826000A3138093A2139093D2068093D10680919A
:10827000D306882331F063E271E189E598E00E943A
:10828000305E8FEF80930A0216C086EF98E09093DD
:10829000A3138093A2139093D2068093D10680916A
:1082A000D306882331F06EE071E186EF98E00E94FA
:1082B000305E10920A021F910F91089510928C1255
:1082C0008091D306882379F020913F0F8091D106C9
:1082D0009091D206222319F06EED70E102C061EF99
:1082E00070E10C94305E089581E080938C1280914F
:1082F000D306882379F020913F0F8091D106909189
:10830000D206222319F060EB70E102C062EC70E14A
:108310000C94305E0895CF93DF93EC010E94889314
:10832000688379838A839B83CE01DF91CF910895FF
:10833000EF92FF921F93CF93DF93CDB7DEB7659790
:108340000FB6F894DEBF0FBECDBF182F7B018DE0B6
:108350009AE00E94498581E080933B0A84E690E0A0
:1083600090931E0A80931D0A84E6E816F10418F41F
:1083700084E6E82EF12CC70164E670E00E9486C016
:1083800070933D0A60933C0A7093200A60931F0A21
:1083900010931A0A8FEF810F823010F41230D1F04F
:1083A0008DE09AE00E945B858091180A882329F06D
:1083B00083EC95EFA8ECBFE304C084EB98ECA6E94E
:1083C000B0E48093370A9093380AA093390AB093A7
:1083D0003A0A55C08091180A882329F084EB98EC5A
:1083E000A6E9B0E404C083EC95EFA8ECBFE380936A
:1083F000370A9093380AA093390AB0933A0A8DE06D
:108400009AE00E94658580913B0A8823C1F1109211
:108410001A0A8EE690E09A83898388E290E09C8332
:108420008B838CE390E09E838D831D8A83E08F9302
:108430008DB79EB745970FB6F8949EBF0FBE8DBF00
:10844000ADB7BEB7119685E1FE01319601900D9250
:108450008A95E1F78DE09AE00E946F850FB6F89457
:10846000DEBF0FBECDBF65960FB6F894DEBF0FBE60
:10847000CDBFDF91CF911F91FF90EF9008958DE0D8
:108480009AE065960FB6F894DEBF0FBECDBFDF91C0
:10849000CF911F91FF90EF903ECF0F931F93CF93FB
:1084A000DF93EC01AB0160E070E02AE00E94F85C31
:1084B0008C01CE010E941D5E800F911FDF91CF9134
:1084C0001F910F9108958F929F92AF92BF92CF927A
:1084D000DF92EF92FF920F931F93CF93DF931F9240
:1084E0001F92CDB7DEB7082E000C990BAA0BBB0B61
:1084F000FC013197EF30F10508F066C28827ED598D
:10850000FE4F8F4F0C94ADC084E08093FC098AE04D
:108510008093FD0986E28093FF0981E08093020A3F
:108520008093030A8093010A4CE453E120E030E099
:108530008091FC0990E0281739070CF08CC1FA01F2
:1085400085919491A0E0B0E0880F991FAA1FBB1FEE
:10855000F901EE0FFF1FEE0FFF1FED56F64F808360
:108560009183A283B3832F5F3F4F4E5F5F4FE0CF76
:1085700084E08093FC098AE08093FD0986E2809381
:10858000FF0981E08093020A8093030A82E08093CE
:10859000010A44E453E120E030E08091FC0990E0DE
:1085A000281739070CF057C1FA0185919491A0E082
:1085B000B0E0880F991FAA1FBB1FF901EE0FFF1F24
:1085C000EE0FFF1FED56F64F80839183A283B38396
:1085D0002F5F3F4F4E5F5F4FE0CF84E08093FD09F8
:1085E00085E28093FF0981E08093020A88E080930E
:1085F000030A83E08093010A80E090E0FC01E45CE0
:10860000FC4EE491DC01AC5FB54FEC9301968830F1
:108610009105A1F70E94B18A1EC188E08093FC09F0
:1086200086E08093FD0986E28093FF0981E08093D4
:10863000020A8093030A84E08093010A4CE253E12A
:1086400020E030E08091FC0990E0281739070CF019
:1086500002C1FA0185919491A0E0B0E0880F991FC2
:10866000AA1FBB1FF901EE0FFF1FEE0FFF1FED56F4
:10867000F64F80839183A283B3832F5F3F4F4E5F7A
:108680005F4FE0CF88E08093FC0981E08093FD0993
:1086900097E29093FF098093020A8093030A85E092
:1086A0008093010A4CE153E120E030E08091FC0925
:1086B00090E0281739070CF0CEC0FA01859194910B
:1086C000A0E0B0E0880F991FAA1FBB1FF901EE0FB1
:1086D000FF1FEE0FFF1FED56F64F80839183A2839D
:1086E000B3832F5F3F4F4E5F5F4FE0CF82E18093B8
:1086F000FC0981E08093FD0997E29093FF09809344
:10870000020A8093030A8FE08093010A48EF52E146
:1087100020E030E08091FC0990E0281739070CF048
:108720009AC0FA0185919491A0E0B0E0880F991F5A
:10873000AA1FBB1FF901EE0FFF1FEE0FFF1FED5623
:10874000F64F80839183A283B3832F5F3F4F4E5FA9
:108750005F4FE0CFE091670AF091680A74978081DB
:10876000918140E550E060E070E08959954F0E94AA
:10877000088C2AC182E18093FC0985E08093FD0981
:1087800082E28093FF0981E08093020A8093030ACA
:1087900087E08093010A80E993E3A0E0B0E0809352
:1087A000930990939409A0939509B0939609F2E0E8
:1087B0008F2E912C01E010E080E090E0A0E0BBE57E
:1087C0004CE454E060E070E024EEC22E2CE0D22EA7
:1087D000E12CF12C9801220F331F220F331F54017B
:1087E000AA0CBB1CAA0CBB1C2D56364FF901B7FFB7
:1087F0000DC0C082D182E282F38295012D56364FA0
:10880000F90140835183628373830CC04083518399
:108810006283738395012D56364FF901C082D18250
:10882000E282F382880F991FAA1FBB1F0E5F1F4FA2
:10883000F2E08F0E911C22E18216910459F688E72E
:108840009FEFA0E0B0E08093D7099093D809A09360
:10885000D909B093DA090E94208BB6C0CE010196E7
:108860000E949D8A23E040E150E060E070E072C029
:1088700084E08093FC0982E38093FD0986E2809383
:10888000FF0981E08093020A8093030A8AE08093C3
:10889000010A40EF52E120E030E08091FC0990E0D5
:1088A00028173907C4F6FA0185919491A0E0B0E049
:1088B000880F991FAA1FBB1FF901EE0FFF1FEE0FB4
:1088C000FF1FED56F64F80839183A283B3832F5F02
:1088D0003F4F4E5F5F4FE1CF84E08093FC0980E221
:1088E0008093FD0986E28093FF0981E08093020A6C
:1088F0008093030A8BE08093010A48EE52E120E066
:1089000030E08091FC0990E0281739070CF0A3CFE4
:10891000FA0185919491A0E0B0E0880F991FAA1FF9
:10892000BB1FF901EE0FFF1FEE0FFF1FED56F64FB5
:1089300080839183A283B3832F5F3F4F4E5F5F4F4E
:10894000E0CFCE0101960E949D8A21E040E154E0F3
:1089500060E070E0CE0101960E947C8B35C084E01F
:108960008093FC0983E08093FD0986E28093FF09F0
:1089700081E08093020A8093030A8DE08093010ACC
:1089800040EE52E120E030E08091FC0990E02817B1
:1089900039070CF060CFFA0185919491A0E0B0E026
:1089A000880F991FAA1FBB1FF901EE0FFF1FEE0FC3
:1089B000FF1FED56F64F80839183A283B3832F5F11
:1089C0003F4F4E5F5F4FE0CF0F900F90DF91CF9101
:1089D0001F910F91FF90EF90DF90CF90BF90AF90DD
:1089E0009F908F9008950F931F93CF93DF93EC0187
:1089F000462F50E060E070E02AE00E94F85C8C01B5
:108A0000CE010E941D5E800F911FDF91CF911F91BB
:108A10000F910895462F50E060E070E02AE00C943A
:108A2000F85C2FB7F894882381F0809151119091D0
:108A300052119093601180935F1180916111909118
:108A4000621118161906ACF00FC080915311909165
:108A500054119093601180935F11809161119091F6
:108A60006211181619062CF480916111909162110F
:108A700007C0809161119091621191958195910942
:108A800090936211809361112FBF0895AF92BF92AE
:108A9000CF92DF92EF92FF920F931F93CF93DF93CA
:108AA0001F921F92CDB7DEB78C017A836983CE0106
:108AB00001966C01580192E0A90EB11CE12CF12C39
:108AC000C8010E9471BEF60161916F01861731F0F5
:108AD000C8010E9483BEFFEFEF1AFF0A0F5F1F4F0E
:108AE0000A151B0569F781E0EF2809F480E00F9073
:108AF0000F90DF91CF911F910F91FF90EF90DF903A
:108B0000CF90BF90AF900895EF92FF920F931F9375
:108B1000CF93DF931F921F92CDB7DEB78C017B01FD
:108B20008AEA8A8341E050E0BE016E5F7F4FC80150
:108B30000E94F099D701ED91FC910680F781E02D1C
:108B4000C701199582E8898341E050E0BE016F5F5B
:108B50007F4FC8010E94F0990F900F90DF91CF9145
:108B60001F910F91FF90EF900895CF92DF92EF92B7
:108B7000FF920F931F930E9488936B017C01609377
:108B8000CD117093CE118093CF119093D01180911D
:108B9000180B0E940F608093CC1190911A0B9923AF
:108BA00029F091E0811190E09093CC118091220BFB
:108BB0009091230BA091240BB091250B9701860176
:108BC000081B190B2A0B3B0B4091260B5091270BCE
:108BD0006091280B7091290B90911B0B04171507BE
:108BE0002607370760F4C0921E0BD0921F0BE0924D
:108BF000200BF092210B10921D0B892F1EC0909319
:108C00001C0B8091CC1180931B0BC0921E0BD09239
:108C10001F0BE092200BF092210B891761F0C0929C
:108C2000220BD092230BE092240BF092250B91E0C3
:108C300090931D0B02C010921D0B1F910F91FF907E
:108C4000EF90DF90CF9008950F931F93CF93DF9312
:108C5000EC012AE00E94F85C8C01CE010E941D5EAE
:108C6000800F911FDF91CF911F910F910895CF92A7
:108C7000DF92EF92FF920F931F93CF93DF936B01DD
:108C8000770FEE08FF08F7FE1BC0EC016DE20E94B3
:108C9000B85C8C0144275527BA014C195D096E094F
:108CA0007F092AE0CE010E94F85C800F911FDF91BE
:108CB000CF911F910F91FF90EF90DF90CF9008958B
:108CC0002AE0B701A601DF91CF911F910F91FF908C
:108CD000EF90DF90CF900C94F85CCF92DF92EF9200
:108CE000FF920F931F93CF93DF938C016B01770F4C
:108CF000EE08FF08F7FE12C06DE20E94B85CEC01BE
:108D000044275527BA014C195D096E097F092AE0ED
:108D1000C8010E94F85CC80FD91F06C02AE0B7013D
:108D2000A6010E94F85CEC01C8010E941D5E8C0F38
:108D30009D1FDF91CF911F910F91FF90EF90DF90DA
:108D4000CF9008950F931F93CF93DF931F92CDB7CA
:108D5000DEB78C0169830E9471BE6981861729F094
:108D6000C8010E9483BE81E001C080E00F90DF91C6
:108D7000CF911F910F910895CF939DD584E090E0FE
:108D80009093150B8093140B8FE09EE09093F0105E
:108D90008093EF101092EA108091130B90910F0EB8
:108DA000891718F091E09093E71028E13EE03093A6
:108DB000FA102093F9101092F4109091180E891760
:108DC00018F091E09093F11021E23EE0309304110D
:108DD000209303111092FE109091210E891718F024
:108DE00091E09093FB102AE23EE030930E11209325
:108DF0000D111092081190912A0E891718F091E028
:108E0000909305111092120B20E030E0F901ED541F
:108E1000F14F40815181415051094432510520F4B4
:108E200091E09093120B05C02D5F3F4F283731051D
:108E300069F79091120B992341F12091220E309104
:108E4000230E2D5D3F4F3093230E2093220E209151
:108E5000240E3091250E235231093093250E209394
:108E6000240E20912B0E30912C0E2D5D3F4F309310
:108E70002C0E20932B0E20912D0E30912E0E23526E
:108E8000310930932E0E20932D0E90912C0F9F3090
:108E900049F490912D0F9F3029F41092E610109212
:108EA000E51008C02091890F30918A0F3093E610A9
:108EB0002093E51022E130E03093E3102093E2109C
:108EC0002091140B3091150BA3E3BEE0EEE8F0E126
:108ED00041E0B683A5839C91992329F0891718F066
:108EE00040832F5F3F4F1A96379690E1E23EF90795
:108EF00081F73093150B2093140B2131310534F099
:108F000080E190E09093150B8093140BBFD48BEE0F
:108F100090E19093F10F8093F00F8091EF1090917A
:108F2000F0109093EF0F8093EE0F88EE90E1909306
:108F3000F30F8093F20F89EE90E19093F50F8093F9
:108F4000F40F87EE90E19093F70F8093F60F85EF83
:108F500090E19093FB0F8093FA0F8091F91090911C
:108F6000FA109093F90F8093F80F82EF90E19093AD
:108F7000FD0F8093FC0F83EF90E19093FF0F8093A0
:108F8000FE0F81EF90E190930110809300108FEF1E
:108F900090E19093051080930410809103119091BB
:108FA000041190930310809302108CEF90E1909342
:108FB0000710809306108DEF90E190930910809335
:108FC00008108BEF90E190930B1080930A1089E0CA
:108FD00091E190930F1080930E1080910D1190915C
:108FE0000E1190930D1080930C1086E091E19093F8
:108FF00011108093101087E091E1909313108093EB
:10900000121085E091E19093151080931410209137
:10901000140B3091150B2450310960E07AE0C7E061
:10902000462F50E04217530724F5CA010496789F53
:10903000F001799FF00D1124E251F04FC49FC0015F
:10904000C59F900D1124AC0140575F4E538342835E
:10905000DC01A257BF4E15964D915C911697518336
:10906000408381579F4E95838483B187A0876F5F2C
:10907000D7CF81E08093160BCF9108950F931F9364
:10908000CF93DF93FC01248135812115310519F43B
:10909000FB01108211C0EA0121972C173D0708F44B
:1090A000E9018B01FC0160817181AE01C8010E9460
:1090B000F1C2C00FD11F1882DF91CF911F910F9184
:1090C00008954115510521F06115710509F0D6CFBC
:1090D0000895EF92FF920F931F93CF93DF931F9208
:1090E0001F92CDB7DEB78C018CE789831A82F80115
:1090F000E480F580FFEFEF1AFF0AB701C8010E9474
:10910000AF5B882381F0F8012081318184819581D2
:10911000BE016F5F7F4F820F931F0E94EAC2F8016A
:10912000F582E48281E00F900F90DF91CF911F9143
:109130000F91FF90EF900895AF92BF92CF92DF9280
:10914000EF92FF920F931F93CF93DF9300D01F9264
:10915000CDB7DEB78C0149835A836B837C83CE0104
:1091600001966C01580194E0A90EB11CE12CF12C80
:10917000C8010E9471BEF60161916F01861731F03E
:10918000C8010E9483BEFFEFEF1AFF0A0F5F1F4F57
:109190000A151B0569F781E0EF2809F480E00F90BC
:1091A0000F900F900F90DF91CF911F910F91FF9033
:1091B000EF90DF90CF90BF90AF900895CF92DF9265
:1091C000EF92FF920F931F93CF93DF93EC010091E7
:1091D000030EE0E0F0E020E030E0A90110E0CE175F
:1091E000DF071CF1309711F40D32E1F0DF01AD5FC4
:1091F000B14FFC9080ED8F0D8A30A8F4AAE0B0E06A
:109200000E94ADBE2F2DFF0C330B20533109690195
:10921000330FEE08FF089B01AC012C0D3D1D4E1DC8
:109220005F1D01C011E03196DACFCA01B9011123E7
:1092300039F090958095709561957F4F8F4F9F4F36
:10924000DF91CF911F910F91FF90EF90DF90CF9022
:10925000089580911B0B811105C081E090911D0B39
:10926000911101C080E00895CF93DF9320913E0AD1
:1092700030913F0AE9012697A881B981A25CB54FD8
:1092800012961C92082E000C990BAA0BBB0BFC012A
:109290003197EF30F10508F06EC18827EE58FE4F88
:1092A0008F4F0C94ADC0F9013A9780819181825C17
:1092B000954F0E9488BA882309F462C1E0913E0A62
:1092C000F0913F0A36970190F081E02DE25CF54F76
:1092D00081E0EDC0F9013C9780819181825C954FDE
:1092E0000E94C5B9882309F44BC1E0913E0AF09170
:1092F0003F0A36970190F081E02DE25CF54F82E065
:10930000D6C0F9013E9780819181825C954F0E9481
:1093100008B9882309F434C1E0913E0AF0913F0A6C
:1093200036970190F081E02DE25CF54F83E0BFC0FD
:10933000F901709780819181825C954F0E948EB86F
:10934000882309F41DC1E0913E0AF0913F0A369747
:109350000190F081E02DE25CF54F84E0A8C0F901B6
:10936000729780819181825C954F0E9449B88823D1
:1093700009F406C1E0913E0AF0913F0A3697019048
:10938000F081E02DE25CF54F85E091C0F901749722
:1093900080819181825C954F0E9404B8882309F4F2
:1093A000EFC0E0913E0AF0913F0A36970190F081BC
:1093B000E02DE25CF54F8FE07AC0F901769780816D
:1093C0009181825C954F0E948BB7882309F4D8C0A5
:1093D000E0913E0AF0913F0A36970190F081E02D2E
:1093E000E25CF54F86E063C0F90178978081918156
:1093F000825C954F0E9405B7882309F4C1C0E091B3
:109400003E0AF0913F0A36970190F081E02DE25C30
:10941000F54F87E04CC0F9017A9780819181825C99
:10942000954F0E94F7B6882309F4AAC0E0913E0A3E
:10943000F0913F0A36970190F081E02DE25CF54F04
:1094400088E035C0F901B29780819181825C954FA7
:109450000E941AB4882309F493C0E0913E0AF09167
:109460003F0A36970190F081E02DE25CF54F838151
:109470009481A581B6814097A105B10509F080C00E
:109480008FC0F9017C9780819181825C954F0E9409
:109490002EB6882309F474C0E0913E0AF0913F0A89
:1094A00036970190F081E02DE25CF54F8AE08283EF
:1094B00067C0F9017E9780819181825C954F0E94FF
:1094C00064B5882309F45CC0E0913E0AF0913F0A3C
:1094D00036970190F081E02DE25CF54F8BE0E7CF0D
:1094E000F901B29780819181825C954F0E941AB4F4
:1094F000882309F445C0E0913E0AF0913F0A36976F
:109500000190F081E02DE25CF54F83819481A5818B
:10951000B68180319440A105B10591F543C0F901B0
:10952000B09780819181825C954F0E9493B488238B
:1095300039F1E0913E0AF0913F0A36970190F081AF
:10954000E02DE25CF54F8DE0B2CFF901B29780815A
:109550009181825C954F0E941AB4882389F0E09132
:109560003E0AF0913F0A36970190F081E02DE25CCF
:10957000F54F8EE09CCFE881F981E25CF54F1282D5
:10958000E0913E0AF0913F0A36970190F081E02D7C
:10959000E25CF54F81E09281911106C080E004C049
:1095A00089E085CF8CE083CFDF91CF9108958091C2
:1095B000110B811157C0E091EF10F091F0108581EF
:1095C00096819093EC108093EB101092EE10109215
:1095D000ED10E091F910F091FA1085819681909349
:1095E000F6108093F5101092F8101092F710E09199
:1095F0000311F0910411858196819093001180935D
:10960000FF101092021110920111E0910D11F091D2
:109610000E118581968190930A1180930911109201
:109620000C1110920B1182E190E09093E310809363
:10963000E21081E08093E8108093F2108093FC1098
:10964000809306118093E41080E090E021E0FC011B
:10965000E257FF4E2183079684359105C1F781E0DB
:109660008093110B08951092081108951092FE1026
:1096700008958F929F92AF92BF92CF92DF92EF9216
:10968000FF921F93CF93DF93EC0111E08E819F81B6
:10969000892B09F410E02C813D81E885F985C5808E
:1096A000D680878190E0A601480F591F24173507FF
:1096B00064F180850D2C000CEE08FF08A901330F22
:1096C000660B770B0380F481E02D9A01AB012C1916
:1096D0003D094E095F09882329F0A1E0BFEF0E94F0
:1096E000B9BE04C0AFEFB0E00E94ADBE4F01FF0FA6
:1096F000AA08BB08A50194012C193D094E095F0970
:109700000E9491BE3F832E834BC0A601481B590B7C
:10971000421753070CF43FC080850D2C000CEE0857
:10972000FF08A901330F660B770B81809280092C0B
:10973000000CAA08BB089A01AB01281939094A098B
:109740005B09882399F0A1E0BFEF0E94B9BEA70191
:109750009601281939094A095B090E9491BEDA016C
:10976000C90181509F4FAF4FBF4F12C0AFEFB0E064
:109770000E94ADBEA7019601281939094A095B0963
:109780000E9491BEDA01C9018F5F9109A109B10957
:109790009F838E8305C01F821E82111101C0198212
:1097A0008E819F81009789F08F3F910519F014F009
:1097B0008FEF90E081305FEF950714F481E09FEF29
:1097C0009F838E8381E018271A83DF91CF911F91A9
:1097D000FF90EF90DF90CF90BF90AF909F908F90D1
:1097E000089581E080930E0B089581E080930F0B24
:1097F000089581E08093100B0895CF93DF93C0917B
:109800000812D09109126091181270911912CE01AC
:109810000E948C5481110DC027ED3AE444EF51E0D1
:1098200060E070E0CE010E94F3549093191280938F
:109830001812DF91CF910895CF93DF9300D01F923C
:109840001F92CDB7DEB7FE01319625E0DF011D92F4
:109850002A95E9F724E8298325E52C832AE22D833C
:109860006A834B8345E050E0BF010E94F09965E0B8
:1098700070E080E090E00E94509380E00F900F90A5
:109880000F900F900F90DF91CF9108951092E810F4
:109890001092F2101092FC10109206111092E41027
:1098A00080E090E0FC01E257FF4E1182079684357C
:1098B0009105C1F708958091170B823039F08330FC
:1098C00049F0813049F48091101201C080E1809309
:1098D000130B04C08EE0FBCF1092130B8091130B7F
:1098E00008958091170B823039F0833051F0813028
:1098F00069F480910F1208950E94B75980913E1229
:1099000008950E94AC5980910E12089580E0089548
:109910008091170B823049F0833071F0813099F4D7
:1099200080910A1290910B1208950E94B75980916C
:1099300042129091431208950E94AC5980910C12EA
:1099400090910D12089581E090E008952F923F923A
:109950005F926F927F928F929F92AF92CF92DF929F
:10996000EF92FF920F931F93CF93DF931F921F925B
:10997000CDB7DEB76DB67EB60E94B7590E94AC591E
:10998000C7DF029709F01DC2ACDF882309F415C2B6
:10999000C0901812D0901912E0900812F09009129D
:1099A000B601C701B9D78823F1F0F701E250FE4FA5
:1099B00000E010E0819191918C159D0571F40E9459
:1099C0008893000F111F000F111FF701E00FF11F07
:1099D000608371838283938307C00F5F1F4F0E31B3
:1099E000110541F701C009DF1092110BEDB6FEB66B
:1099F0004091140B5091150BCA01880F991F2DB778
:109A00003EB7281B390B0FB6F8943EBF0FBE2DBFD3
:109A10000DB71EB70F5F1F4F8091170B823069F093
:109A2000833029F1813009F071C0B80180911112A1
:109A3000909112120E944E9A33C03FB7F89420E0E2
:109A4000822F90E08417950774F4880F991FF8010E
:109A5000E80FF91FDC01A25EBD4E8D919C919183B0
:109A600080832F5FEDCF3FBF10923E1219C03FB7EA
:109A7000F89420E0822F90E08417950774F4880F03
:109A8000991FF801E80FF91FDC01A451BE4E8D911A
:109A90009C91918380832F5FEDCF3FBF10920E1278
:109AA00020E06AE071E0822F90E04091140B509129
:109AB000150B8417950754F5689FF001699FF00D09
:109AC0001124E251F04FA085B1858C918823E1F0FB
:109AD000A081B1813C91C801830F911D830F911D1D
:109AE000DC0112978D919C91A281B3814D915C9183
:109AF00011970480F581E02D4817590711F4108261
:109B000003C070838D939C932F5FCDCF0FB6F894D5
:109B1000FEBE0FBEEDBE8091E810882319F087EEDF
:109B200090E1A7DD8091F210882319F081EF90E198
:109B3000A0DD8091FC10882319F08BEF90E199DD76
:109B400080910611882319F085E091E192DD8091E2
:109B5000120B882309F465C08091FC10811105C0A7
:109B600080910611882309F450C08091FF109091D4
:109B70000011E0910311F091041123813481281721
:109B8000390724F48085811109C00EC021813281FA
:109B90008217930734F48085811106C088E090E035
:109BA00005C080E190E002C080E290E020910911C0
:109BB00030910A11E0910D11F0910E114381548101
:109BC0004217530724F42085222349F00AC041811B
:109BD0005281241735073CF42085222311F081603F
:109BE00003C0846001C082602091E2103091E310D4
:109BF0002817390719F41092E41007C09093E31066
:109C00008093E21081E08093E4108091E2109091C3
:109C1000E310429709F4D8C081E080930811809343
:109C2000FE10EFE8F0E182E990E19A83898398EEF3
:109C3000892E93E0992E55245394CF010197DC018E
:109C40008C91882309F4ACC0E480F580D701179685
:109C50008C911797882309F4A3C08081882309F485
:109C60009FC04181528118966C918401041B150B91
:109C7000101611061CF08A01085E134020E030E047
:109C800022242394312C8FE097E2A12CC62ED12CD4
:109C90002C143D04ACF56430A9F040F4623071F04E
:109CA000633019F5C9018A529A4F13C0653071F0BB
:109CB0006630D9F4C90188549A4F0BC0C901845247
:109CC0009A4F07C0C90182539A4F03C0C9018C53F0
:109CD0009A4FDC0112968D919C911397841B950BE2
:109CE00097FF03C09195819591098017910714F40E
:109CF000A22C8C01BFEF2B1A3B0A2E5F3F4FC8CF1F
:109D000081E08A0DD70119969C919923F1F1643075
:109D100099F028F4623041F0633049F036C0653084
:109D2000A1F06630D9F031C0813021F52DC08130ED
:109D300049F1833051F51EC0813011F1823011F1AB
:109D4000833011F1843009F515C08130B9F08230CB
:109D5000B9F08430C9F08530C1F40CC0813061F0B5
:109D6000823061F0833061F0843061F0853061F0E1
:109D7000863059F481E009C086E007C085E005C05F
:109D800084E003C083E001C082E0A981BA819C9194
:109D9000981302C0108204C05082A981BA818C93AA
:109DA000379629813A81295F3F4F3A83298330E1F1
:109DB000E33EF30709F041CF02C068DD1EDD81E01C
:109DC0005FC064DD80E05CC0E090E510F090E610DC
:109DD0001E141F040CF04FC08091FD10009108125A
:109DE0001091091260911612709117128823A1F038
:109DF00081E08093FE10C8018FD5811113C0A701A7
:109E0000FF0C660B770B26E33BE4C801ECD590937F
:109E100017128093161206C0C8017ED5811102C0A8
:109E20001092FE10809107110091081210910912F2
:109E300060911412709115128823C1F081E0809313
:109E40000811C80169D58111ECCE4091E5105091FF
:109E5000E610052E000C660B770B23E33BE4C801EC
:109E6000C2D59093151280931412DBCEC80154D53D
:109E70008111D7CE02C01092FE1010920811D1CEDF
:109E80000FB6F8947EBE0FBE6DBE0F900F90DF919F
:109E9000CF911F910F91FF90EF90DF90CF90AF90F7
:109EA0009F908F907F906F905F903F902F9008953C
:109EB000CF9380911312C0910B028111FFC0C23069
:109EC00009F44FC0C33009F49CC0C13009F026C169
:109ED0008091100B811122C181E090E00E94C1C0ED
:109EE000909312128093111262E083E00E946660E8
:109EF0001092E91110920B1210920A1210920F1286
:109F000080E090E0FC01EE0FFF1FE952FE4E11824F
:109F10001082019688309105A9F71092E8111092ED
:109F2000E71180916A008C6080936A00ED9A8FB788
:109F3000F89420918400309185003093D2112093C1
:109F4000D1118FBF29EF3BE44AEF50E060E070E0B1
:109F5000809108129091091246D581E080931312E6
:109F6000DDC080910F0B8111D9C081E090E00E948B
:109F7000C1C090931B1280931A12809104018E7FAE
:109F800080930401809105018160809305018FE138
:109F900097E090934512809344122EE240EA56E8EF
:109FA00061E070E00E94AA5F809165008B7F8093E2
:109FB00065001092350189E0809334018EE2809330
:109FC00032018CEF8093300180E98093310110924F
:109FD00043121092421210924112109240121092AB
:109FE0003E12EEE1F2E18CED95E08193919322E156
:109FF000EE33F207D1F7C1E0C0933F1225EF3BE407
:10A0000051C080910E0B811189C081E090E00E94C7
:10A01000C1C090931D1280931C12809104018E7F09
:10A0200080930401809105018160809305018FE197
:10A0300097E09093EB118093EA1126E040E052EC18
:10A0400061E070E00E94AA5F809165008B7F809341
:10A0500065001092350180E18093340186E08093A1
:10A0600032018EEF8093300180E9809331011092AC
:10A070000D1210920C121092D6111092D51110924E
:10A080000E12ECEEF1E18CED95E08193919322E1DB
:10A09000E830F207D1F71092D411C1E0C093D31188
:10A0A00021EF3BE44AEF50E060E070E0809108125D
:10A0B0009091091298D4C093131230C0C23069F045
:10A0C000C330D1F0C13051F58091100B811126C001
:10A0D00080910A1290910B121DC080910F0B81117B
:10A0E0001DC080911A1290911B120E94A658809157
:10A0F0004212909143120EC080910E0B81110EC03E
:10A1000080911C1290911D120E947D8080910C12F2
:10A1100090910D12029711F4C093170B80910B02CE
:10A120008230A1F1833009F454C0813009F074C049
:10A130008091100B882309F46FC0ED98E59A109276
:10A14000E9111092101210920B1210920A12109232
:10A150000F1280E090E0FC01EE0FFF1FE952FE4E6F
:10A1600011821082019688309105A9F71092E811AA
:10A170001092E71180911112909112120E9456C113
:10A180001092131210920F0B82E044C080910F0BBB
:10A19000882309F441C080914412909145120E9495
:10A1A000885F809131018F778093310180913101F7
:10A1B0008F7E809331011092300180911A1290911C
:10A1C0001B120E9456C11092131210920E0B83E0C4
:10A1D00021C080910E0B8823F9F08091EA119091B3
:10A1E000EB110E94885F809131018F77809331015C
:10A1F000809131018F7E80933101109230018091E6
:10A200001C1290911D120E9456C1109213121092AE
:10A21000100B81E080930B0280910812909109123B
:10A22000CF91F1C3EF92FF921F93CF93DF931F92D1
:10A23000CDB7DEB77C01162FFC01618172810E94CF
:10A24000844565E070E080E090E00E94509342E435
:10A2500062E4C701F1DA412F60E0C701EDDA811154
:10A2600064C040E061E0C701E7DA81115EC040E010
:10A2700062E0C701E1DA811158C046E062E0C7013F
:10A28000DBDA811152C040E063E0C701D5DA811109
:10A290004CC040E064E0C701CFDA11E0811110E06A
:10A2A00040E065E0C701C8DA811101C01F5F40E0EE
:10A2B00066E0C701C1DA811101C01F5F40E067E0BD
:10A2C000C701BADA811101C01F5F40E068E0C70131
:10A2D000B3DA811101C01F5F40E069E0C701ACDA69
:10A2E000811101C01F5F44E06AE0C701A5DA811156
:10A2F00001C01F5F44E06AE0C7019EDA811101C01E
:10A300001F5F62E370E080E090E00E94509382E87B
:10A31000898341E050E0BE016F5F7F4FC7010E941B
:10A32000F09981E0183011F0111180E00F90DF9169
:10A33000CF911F91FF90EF900895FC0182810895C5
:10A34000482F50E095E1899FF0011124E15FFE4E16
:10A350002181328180859185280F391F83819481E5
:10A360008217930728F08581968128173907E8F42A
:10A3700085E1849FF001859FF00D1124E15FFE4E81
:10A38000858196812817390728F52581368185E151
:10A39000849FF001859FF00D1124E15FFE4E8285C0
:10A3A000823019F411861086128685E1849FF001AF
:10A3B000859FF00D1124E15FFE4E32832183809151
:10A3C000840090918500280F391F309389002093D5
:10A3D000880008958381948182179307C0F62381B2
:10A3E0003481D5CF62E30C94D27661E30C94D276BB
:10A3F00060E30C94D27664E50C94D2766FE20C9410
:10A40000D2766DE20C94D2766CE20C94D27677FF21
:10A4100003C071956195710920E0462F6EE20C949E
:10A420008C76462F20E06DE40C948C76FC016283E0
:10A43000611105C020E040E06BE40C948C76089537
:10A4400077FF03C071956195710920E0462F6BE499
:10A450000C948C764F925F926F927F928F929F9224
:10A46000AF92BF92CF92DF92EF92FF920F931F9322
:10A47000CF93DF936C01A4ECCA1AADEFDA0AD601D0
:10A48000ED91FC917E970CF05DC0FC01E858FF4F08
:10A49000812C912CA191B191AB2B21F42115310587
:10A4A00049F450C0BFEF8B1A9B0AAEE18A169104A3
:10A4B00089F748C0EC015401AA0CBB1CAA0CBB1CB8
:10A4C000AC0EBD1EF501EC54FF4F408351836283F7
:10A4D00073837401EE0CFF1CEC0EFD1EF701E858AF
:10A4E000FF4F31832083EC54FF4F11830083BE0163
:10A4F000680D791DFB01EC55FE4F81E080830E94C1
:10A500008893F5016083718382839383C65CDD4FFA
:10A5100088819981F701E250FE4F91838083D601B3
:10A520002D913C9111972F5F3F4F2D933C939C01B0
:10A530002F5F3F4F1216130614F021E030E03983ED
:10A54000288302C08FEF9FEFDF91CF911F910F9172
:10A55000FF90EF90DF90CF90BF90AF909F908F9043
:10A560007F906F905F904F9008950F931F93CF93BC
:10A57000DF938C01C62FD42F65E870E0DC019F9635
:10A580008D919C91D0970E947770F80187A590A932
:10A59000DC01ED91FC910190F081E02D6C2F19957B
:10A5A000F80187A590A9DC01ED91FC910190F08163
:10A5B000E02D6D2F19952C2F30E0B9016B577F4F8F
:10A5C0006D0F711D6F777727F80187A590A9DF912F
:10A5D000CF911F910F910C947770262F2B7FA1F4B0
:10A5E0009A014F3F510519F014F02FEF30E0A90107
:10A5F00041302FEF520714F441E05FEF57FF03C0E3
:10A60000519541955109B1CF0895CF93DF93EC0156
:10A6100089AD9AAD892B11F01AAE19AECE010E9408
:10A6200012738BA9813029F0823069F0811117C033
:10A6300005C060E070E088E00E94A26010922D01E9
:10A6400010922C0108C040E064E0CE018EDF40E0B3
:10A6500060E0CE018ADF1AA219A21F8E1E8E0E9410
:10A6600088936DAB7EAB8FAB98AFDF91CF910895A0
:10A670008F929F92AF92BF92CF92DF92EF92FF9212
:10A680000F931F93DC0114968D919C91159756960C
:10A69000CD90DC9057976817790709F455C09096CC
:10A6A000FC9090974C01092E000CAA08BB088B0166
:10A6B000072E000C220B330B861797073CF41296DB
:10A6C000ED91FC911397FF2031F014C0ED91FC91B6
:10A6D0001197FF2079F00D2C000CEE08FF08A9015E
:10A6E0009801281939094A095B0954966D917C91A2
:10A6F00055970EC00D2C000CEE08FF08A90198011B
:10A70000281939094A095B0952966D917C91539732
:10A71000CB01770FAA0BBB0BBC01CD016C197D09D6
:10A720008E099F090E9477C08F01FF0F220B330B08
:10A73000A9019801281939094A095B090E9491BEAB
:10A74000C20ED31EE41EF51EC6011F910F91FF908D
:10A75000EF90DF90CF90BF90AF909F908F90089533
:10A760008F929F92AF92BF92CF92DF92EF92FF9221
:10A770000F931F93DC0114968D919C9115971A9657
:10A78000CD90DC901B976817790709F455C0909617
:10A79000FC9090974C01092E000CAA08BB088B0175
:10A7A000072E000C220B330B861797073CF41296EA
:10A7B000ED91FC911397FF2031F014C0ED91FC91C5
:10A7C0001197FF2079F00D2C000CEE08FF08A9016D
:10A7D0009801281939094A095B0918966D917C91ED
:10A7E00019970EC00D2C000CEE08FF08A901980166
:10A7F000281939094A095B0916966D917C911797BA
:10A80000CB01770FAA0BBB0BBC01CD016C197D09E5
:10A810008E099F090E9477C08F01FF0F220B330B17
:10A82000A9019801281939094A095B090E9491BEBA
:10A83000C20ED31EE41EF51EC6011F910F91FF909C
:10A84000EF90DF90CF90BF90AF909F908F90089542
:10A85000EF92FF920F931F93CF93DF93EC0189AD9B
:10A860009AAD892B11F01AAE19AE8BA98130B1F0D7
:10A87000823059F1811143C0CB0177FF03C091951C
:10A8800081959109BC01CE016BDF90932D018093DE
:10A890002C019AA389A39F8F8E8F31C08B0177FFE4
:10A8A00003C0119501951109B801CE0159DF7C0152
:10A8B000B801CE01DDDE8C01B70188E00E94A26004
:10A8C00010932D0100932C0116C08B0177FF03C05C
:10A8D000119501951109B801CE0142DF7C01B80143
:10A8E000CE01C6DE8C01A70164E0CE0176DEA801B0
:10A8F00060E0CE0172DEFAA2E9A21F8F0E8F0E94E5
:10A9000088936DAB7EAB8FAB98AFDF91CF911F91EA
:10A910000F91FF90EF900895DC01A250BE4F20E010
:10A9200030E04D915D914617570739F4280F391FD4
:10A93000F901EC55FE4F808108952F5F3F4F2E3176
:10A94000310579F780E00895CF93DF93EC01C45C83
:10A95000DD4FA881B981109709F442C0FC01E25093
:10A96000FE4F20E030E0419151914617570799F58D
:10A97000A901440F551F480F591FFA01E858FF4F0E
:10A9800060817181672B61F111821082FC01E20FFD
:10A99000F31FEC55FE4F1082FA01EE53FE4F118269
:10A9A0001082235D3F4F220F331F220F331FFC0104
:10A9B000E20FF31F1082118212821382FA01E8590A
:10A9C000FE4F11821082EA56FF4F118210821197BA
:10A9D000B983A88305C02F5F3F4F2E31310519F68B
:10A9E000DF91CF9108950F931F9301E010E032DDC6
:10A9F0001F910F9108950F931F9300E010E02ADD3F
:10AA00001F910F9108952F923F924F925F926F92F4
:10AA10007F928F929F92AF92BF92CF92DF92EF92EE
:10AA2000FF920F931F93CF93DF9300D000D0CDB749
:10AA3000DEB78C010E94889398012E533E4F3C83D1
:10AA40002B831E830D83D801AC55BE4FBA83A983D7
:10AA50001801B2E02B1ABEEF3B0AF901AA24A39415
:10AA6000B12C32E0832E912C118210829F012A5446
:10AA70003140D9012D913C91232B09F44DC0AD817A
:10AA8000BE812D913D914D915C9113977D01B4EB69
:10AA9000EB0EF11CD701CD90DD90ED90FC902B01D9
:10AAA0003C01421A530A640A750A4C145D046E0490
:10AAB0007F0490F1C20ED31EE41EF51EAD81BE814F
:10AAC000CD92DD92ED92FC921397A981BA812C91DF
:10AAD000222311F19F0126593109D9012D913C9171
:10AAE0002115310519F4B182A08216C07F01BAE5A3
:10AAF000EB1AF108D7014D915C911197421753075A
:10AB00005CF4B182A0824F5F5F4F4D935C9342171C
:10AB1000530714F09182808232962D813E812C5F02
:10AB20003F4F3E832D83A981BA811196BA83A983B1
:10AB3000E215F30509F098CFEB81FC8181919191A9
:10AB4000FC83EB838130910599F00297C9F4EB8186
:10AB5000FC81EC54F1400190F081E02D1995AB811E
:10AB6000BC81DA966D917C91DB97C801EDDE08C05F
:10AB7000EB81FC81EC54F1400190F081E02D1995BE
:10AB80002B813C8122153305B9F626960FB6F89431
:10AB9000DEBF0FBECDBFDF91CF911F910F91FF9010
:10ABA000EF90DF90CF90BF90AF909F908F907F906D
:10ABB0006F905F904F903F902F9008956E3E22E0EF
:10ABC000720738F06B3C98E0790728F06AEC78E07F
:10ABD00002C06EEE72E0660F771F9FB7F89425E112
:10ABE000829FF0011124E15FFE4E748363839FBF57
:10ABF00008956E3E22E0720738F06B3C98E07907CA
:10AC000028F06AEC78E002C06EEE72E0660F771F03
:10AC10009FB7F89425E1829FF0011124E15FFE4E79
:10AC2000768365839FBF0895660F771F282F30E0D6
:10AC300095E1899FF0011124E15FFE4E85819681A7
:10AC40006817790718F46581768107C0838194813C
:10AC50008617970710F4638174818FB7F89495E194
:10AC6000929FF001939FF00D1124E15FFE4E7283DD
:10AC700061838FBF0895982F8FB7F89425E1929F35
:10AC8000F0011124E15FFE4E21E027838FBF41B127
:10AC900021E030E0B90102C0660F771F9A95E2F714
:10ACA000CB01842B81B908958A3058F49FB7F8946A
:10ACB00025E1829FF0011124E15FFE4E118610868E
:10ACC0009FBF08951F93CF93DF9325E1829FC0011B
:10ACD0001124EC01C15FDE4E8A8581110FC01FB7C0
:10ACE000F89481E08A8789899A899A8389830E9466
:10ACF00088936B877C878D879E871FBFDF91CF915D
:10AD00001F910895CF93DF938A30D0F56233710598
:10AD100038F061369DE6790728F060E67DE602C0EE
:10AD200062E370E0D42FC82F80E090E00E944CBD19
:10AD300020E030E04AE754E40E9453BF20E030E0D6
:10AD40004CE852E40E94ADBD9B01AC0160E070E0B4
:10AD50008AEF94E40E9453BF0E94BBBF9B01DD2396
:10AD600021F022273327261B370B8FB7F89495E164
:10AD7000C99FF0011124E15FFE4E318720878FBF0C
:10AD8000DF91CF9108958A3008F418CF08958A3062
:10AD900008F42FCF08958A3058F495E1899FF00187
:10ADA0001124E15FFE4E81819281969587950895E9
:10ADB00080E090E008958A3008F436CF08951F921D
:10ADC0000F920FB60F9211240BB60F920F931F9391
:10ADD0002F933F934F935F936F937F938F939F93A3
:10ADE000AF93BF93CF93EF93FF938091611289301C
:10ADF00048F0109261128091BE11882399F08091E1
:10AE0000B7110DC0E0916112E15025E1E29FF00120
:10AE10001124E15FFE4E8781882321F0808192B169
:10AE2000892782B9E091611285E1E89FF001112440
:10AE3000E15FFE4E8781882321F0808192B1892BCA
:10AE400082B9E0916112C5E1CE9FF0011124E15F6A
:10AE5000FE4E80859185892B09F04DC0E0916112ED
:10AE6000CE9FF0011124E15FFE4E8285813009F012
:10AE700060C00E948893E0916112CE9FF00111247E
:10AE8000E15FFE4E0385148525853685E0916112CC
:10AE9000CE9FF0011124E15FFE4E0784F089E02D82
:10AEA000AB01BC01401B510B620B730BCF01A0E047
:10AEB000B0E084179507A607B707D8F5E0916112AF
:10AEC000A0916112CA9FD0011124A15FBE4E53967A
:10AED0008D919C915497CE9FF0011124E15FFE4E1D
:10AEE00091878087E0916112CE9FF0011124E15F8C
:10AEF000FE4E82E082878091611222DA8091611297
:10AF00008F5F80936112FF91EF91CF91BF91AF91CD
:10AF10009F918F917F916F915F914F913F912F9171
:10AF20001F910F910F900BBE0F900FBE0F901F90AF
:10AF30001895E0916112809184009091850025E13F
:10AF4000E29FF0011124E15FFE4E21813281820FE8
:10AF5000931F9093890080938800D0CF1F93CF9345
:10AF6000DF9380916012811173C0109261129FB7BC
:10AF7000F89485E128EB3BE04CED55E064E971E1A4
:10AF8000A1E0B0E0E0916112E93008F052C0E09138
:10AF900061128E9FF0011124E15FFE4E3283218306
:10AFA000E09161128E9FF0011124E15FFE4E568305
:10AFB0004583E09161128E9FF0011124E15FFE4E06
:10AFC00074836383E0916112F0916112ED0101C01D
:10AFD000CC0FFA95EAF78E9FF0011124E15FFE4E47
:10AFE000C083E09161128E9FF0011124E15FFE4E5B
:10AFF0001782E09161128E9FF0011124E15FFE4EF5
:10B0000011861086E09161128E9FF0011124E15F9C
:10B01000FE4E1286E09161128E9FF0011124E15FD5
:10B02000FE4E148A138AE0916112EF5FE093611281
:10B03000A9CF9FBF8FB7F89420EA3FE03093B911B2
:10B040002093B8111092B7118FBF81E080936012E6
:10B05000DF91CF911F9108950F931F93CF93DF93AB
:10B060008C01C62FD42FDC0111968D919C911297E3
:10B07000DC01ED91FC910190F081E02DD8016C9103
:10B080001995F80181819281DC01ED91FC9101908B
:10B09000F081E02D6C2F1995F80181819281DC01FE
:10B0A000ED91FC910190F081E02D6D2F1995F80143
:10B0B00080816C2F70E0680F711D6D0F711D6F77AF
:10B0C000772781819281DF91CF911F910F910C940D
:10B0D00077700F931F93CF93DF938C01C62FD42FDC
:10B0E000DC0111968D919C911297DC01ED91FC9100
:10B0F0000190F081E02DD8016C911995F8018181C2
:10B100009281DC01ED91FC910190F081E02D6C2F9A
:10B110001995F80181819281DC01ED91FC910190FA
:10B12000F081E02D6D2F1995F80180816C2F70E072
:10B13000680F711D6D0F711D6F7777278181928167
:10B14000DF91CF911F910F910C9477704F925F9286
:10B150006F927F92AF92BF92CF92DF92EF92FF9267
:10B160001F93CF93DF93DD24D39445E0C42EC2E038
:10B17000D0E053E0E52EF12CAA24A394B12C8091C9
:10B18000441290914512DC01ED91FC910084F1850F
:10B19000E02D1995892B09F4D1C0109130018091CF
:10B1A000441290914512DC01ED91FC910284F385EB
:10B1B000E02D199596B3B39A2091840030918500C3
:10B1C0002059384E30938D0020938C00212F2C7104
:10B1D00019F010925F122AC093FB992790F9E09121
:10B1E0005F12E11116C0992351F28F3041F6D092CF
:10B1F0005F12809346128091421290914312892BE4
:10B2000009F0BDCFB0924312A092421210924112A7
:10B21000B6CF992381F010925F1210924112809163
:10B22000421290914312029709F0A9CFF092431273
:10B23000E0924212A4CF91E09E0F90935F12F0E053
:10B24000EA5BFD4E8083993109F099CF811173C07B
:10B2500080915D1282FF05C0F0924312E09242128B
:10B260006AC083FDF9CF80914212909143120197F9
:10B2700061F4809141128F5F80934112843058F0C5
:10B28000D0934312C093421206C0D0934312C0938E
:10B29000421210924112809140128F5F80934012AF
:10B2A00090913F12981708F044C0D0923E12AEE140
:10B2B000B2E1E7E4F2E140E050E0BA0110E0CF0192
:10B2C000FC011B3098F401964080512C612C712CAC
:10B2D000012E04C0440C551C661C771C0A94D2F73E
:10B2E0004429552966297729185FEACF9A013770D2
:10B2F000205E3340C29EC001C39E900D112497FD75
:10B30000079623E0959587952A95E1F784529A4F01
:10B310008D939D931B503BE0769567955795479588
:10B320003A95D1F782E1AE33B80749F61092401250
:10B3300002C010923E1210925F1221CFDF91CF9186
:10B340001F91FF90EF90DF90CF90BF90AF907F90D4
:10B350006F905F904F9008958091170B833031F478
:10B3600080911C1290911D120C947D800895809103
:10B37000170B823029F480911A1290911B12E6CE9D
:10B380000895F5DFE9CF0895CF92DF92EF92FF9213
:10B390000F931F93CF93DF936C017A018B01C0E071
:10B3A000D0E0CE15DF0589F0D8016D918D01D60171
:10B3B000ED91FC910190F081E02DC6011995892B4A
:10B3C00011F47E0102C02196ECCFC701DF91CF912D
:10B3D0001F910F91FF90EF90DF90CF900895FC01A7
:10B3E000A089B1898C91A689B78982FD0FC09C91F3
:10B3F000818D8F5F8F73228D821749F0218DDF0140
:10B40000A20FB11D5D969C93818F08958C91089534
:10B41000089580E090E00895FC01538D448D252F20
:10B4200030E0842F90E0821B930B541710F0CF96DE
:10B43000089501970895FC01918D828D981761F010
:10B44000828DDF01A80FB11D5D968C91928D9F5F5B
:10B450009F73928F90E008958FEF9FEF0895FC0106
:10B46000918D828D981731F0828DE80FF11D858DB9
:10B4700090E008958FEF9FEF0895FC01918D228D4C
:10B48000892F90E0805C9F4F821B91098F739927D1
:10B4900008958FE197E0F1DF21E0892B09F420E0A6
:10B4A000822F08958CEB97E0E8DF21E0892B09F4E7
:10B4B00020E0822F089589E598E0DFDF21E0892BE5
:10B4C00009F420E0822F089586EF98E0D6DF21E08E
:10B4D000892B09F420E0822F0895FC01848DDF017F
:10B4E000A80FB11DA35ABF4F2C91848D90E00196F7
:10B4F0008F739927848FA689B7892C93A089B189E6
:10B500008C9180648C93938D848D981306C00288EF
:10B51000F389E02D80818F7D80830895EF92FF92E3
:10B520000F931F93CF93DF93EC0181E0888F9B8D66
:10B530008C8D981305C0E889F989808185FD23C029
:10B54000F62E0B8D10E00F5F1F4F0F731127E02EAB
:10B550008C8DE8120BC00FB607FCFACFE889F98989
:10B56000808185FFF5CFCE01B8DFF2CF8B8DFE0154
:10B57000E80FF11DE35AFF4FF0820B8FEA89FB8938
:10B580008081806207C0EE89FF896083E889F9893C
:10B5900080818064808381E090E0DF91CF911F9172
:10B5A0000F91FF90EF900895CF93DF93EC01888D7A
:10B5B0008823C1F0EA89FB89808185FD05C0A889BF
:10B5C000B9898C9186FD0EC00FB607FCF5CF80813E
:10B5D00085FFF2CFA889B9898C9185FFEDCFCE0187
:10B5E0007CDFE8CFDF91CF91089580E090E0892B58
:10B5F00019F06ADF811116C080E090E0892B19F004
:10B600005ADF811112C080E090E0892B19F04ADFE7
:10B6100081110EC080E090E0892B79F03ADF811132
:10B620000AC008950E940000E7CF0E940000EBCFFF
:10B630000E940000EFCF0C940000089590E0FC0100
:10B640003197E231F10508F04EC08827EF57FE4FE1
:10B650008F4F0C94ADC0809180008F7703C0809194
:10B6600080008F7D80938000089580918000877F87
:10B67000F9CF84B58F7702C084B58F7D84BD0895DE
:10B680008091B0008F7703C08091B0008F7D809350
:10B69000B0000895809190008F7707C0809190004E
:10B6A0008F7D03C080919000877F809390000895E4
:10B6B0008091A0008F7707C08091A0008F7D03C08C
:10B6C0008091A000877F8093A00008958091200141
:10B6D0008F7707C0809120018F7D03C0809120016A
:10B6E000877F8093200108950E94D2C20F931F93F9
:10B6F000CF93DF938C01EB01FC0180819181009756
:10B70000B1F0688179816115710579F042815381C9
:10B710002C813D814217530740F00E94EAC28C8180
:10B720009D81F8019583848313C00E9456C188814E
:10B730009981F801918380838A819B81938382839D
:10B740008C819D8195838483198218821B821A8241
:10B750001D821C82DF91CF911F910F9108950F934D
:10B760001F93CF93DF93EC0188819981009729F093
:10B770002A813B812617370788F48B016F5F7F4F43
:10B780000E94EEC1009761F0998388831B830A832E
:10B790002C813D81232B11F4FC01108281E001C03A
:10B7A00080E0DF91CF911F910F910895EF92FF926A
:10B7B0000F931F93CF93DF93FB0124813581E080AA
:10B7C000F180FC0104811581E114F10411F480E0A1
:10B7D00016C02115310591F0EC01020F131FB801BD
:10B7E000BEDF8823A1F3288139818C819D81B70137
:10B7F000820F931F0E94EAC21D830C8381E0DF91B8
:10B80000CF911F910F91FF90EF900895EF92FF92CB
:10B810000F931F93CF93DF93EC017B018A01BA0151
:10B820009EDF2881398181110DC02115310519F064
:10B83000C9010E9456C1198218821D821C821B8276
:10B840001A8206C01D830C83B701C9010E94EAC297
:10B85000CE01DF91CF911F910F91FF90EF9008954E
:10B86000CF93DF93EC016115710551F0FB0101905D
:10B870000020E9F73197AF01461B570BC7DF0CC01B
:10B8800088819981009711F00E9456C1198218820F
:10B890001D821C821B821A82CE01DF91CF910895F6
:10B8A000FC01808191810C9456C10F931F93CF931B
:10B8B000DF93CDB7DEB762970FB6F894DEBF0FBE49
:10B8C000CDBF8C01CB01F80111821082138212824C
:10B8D0001582148250E0BE016F5F7F4F0E94DCBC76
:10B8E000BE016F5F7F4FC801BBDF62960FB6F89451
:10B8F000DEBF0FBECDBFDF91CF911F910F91089595
:10B90000FC01118210821382128215821482611549
:10B91000710549F0FB0101900020E9F73197AF0173
:10B92000461B570B73CF0895CF93DF9300D01F9220
:10B93000CDB7DEB7611571058105910579F09B01E1
:10B94000AC0169833A834B835C830E94D0BC29811C
:10B950003A814B815C810E9491BE03C060E070E03F
:10B96000CB010F900F900F900F90DF91CF91089522
:10B97000DC01ED91FC910190F081E02D1994EF92A2
:10B98000FF920F931F93CF93DF938C017B01C0E055
:10B99000D0E0F701EC0FFD1F6491662361F0D80140
:10B9A000ED91FC910190F081E02DC8011995892B52
:10B9B00011F02196EECFCE01DF91CF911F910F9123
:10B9C000FF90EF9008956115710579F0FB010190EA
:10B9D0000020E9F73197AF01461B570BDC01ED91D1
:10B9E000FC910280F381E02D199480E090E00895AD
:10B9F0004F925F926F927F92EF92FF920F931F93FD
:10BA0000CF93DF93CDB7DEB7A1970FB6F894DEBF23
:10BA10000FBECDBF7C01FA01CB0119A2223008F480
:10BA20002AE08E010F5D1F4F422E512C612C712C8C
:10BA3000BF01A30192010E94BDBEF901CA010150DC
:10BA400011096A3014F4605D01C0695CD8016C931F
:10BA5000232B242B252B61F7B801C701B4DFA19656
:10BA60000FB6F894DEBF0FBECDBFDF91CF911F910F
:10BA70000F91FF90EF907F906F905F904F9008959F
:10BA80004F925F926F927F928F929F92AF92BF92EE
:10BA9000CF92DF92EF92FF92CF93DF93EC016A0196
:10BAA0007B01B22E9A01AB01C701B6010E94F6BF1D
:10BAB000882319F06AE176E027C026013701E8946F
:10BAC00077F82FEF3FEF4FE75FE7C301B2010E9426
:10BAD000F6BF81110DC02FEF3FEF4FE75FE7C301C6
:10BAE000B2010E9448BD18161CF46EE176E00CC04D
:10BAF0002FEF3FEF4FE75FE4C701B6010E94ECBFB5
:10BB0000181694F462E276E0CE01DF91CF91FF90B7
:10BB1000EF90DF90CF90BF90AF909F908F907F90ED
:10BB20006F905F904F904FCF2FEF3FEF4FE75FEC5D
:10BB3000C701B6010E9448BD87FDE4CF20E030E098
:10BB4000A901C701B6010E9448BD87FF09C06DE287
:10BB5000CE010EDF4C01F7FAF094F7F8F09402C032
:10BB6000812C912CA12C60E070E080E09FE3AB146D
:10BB700041F020E030E040E251E40E9453BFA39442
:10BB8000F6CF9B01AC01C701B6010E94EFBE2B01AD
:10BB90003C010E94C0BF6B017C010E944CBD9B0117
:10BBA000AC01C301B2010E94EEBE2B013C012AE0B0
:10BBB000B701A601CE011CDF7C01E80CF91CBB20FB
:10BBC00029F06EE2CE01D4DEE80EF91EDB2CDD207A
:10BBD00021F120E030E040E251E4C301B2010E94D3
:10BBE000ADBD2B013C010E94C0BF4B01A12CB12C6B
:10BBF0002AE0B501A401CE01FBDEE80EF91EC50165
:10BC0000B4010E944CBD9B01AC01C301B2010E9472
:10BC1000EEBE2B013C01DA94DACFC701DF91CF9160
:10BC2000FF90EF90DF90CF90BF90AF909F908F905C
:10BC30007F906F905F904F90089566E276E0C3CE5C
:10BC40000F931F93CF93DF93EC01BDDE8C01CE01E8
:10BC5000F4DF800F911FDF91CF911F910F91089515
:10BC60000F931F93CF93DF93EC0189DE8C01CE01FC
:10BC7000E4DF800F911FDF91CF911F910F91089505
:10BC80001F920F920FB60F9211240BB60F922F93A3
:10BC90003F934F935F936F937F938F939F93AF9354
:10BCA000BF93EF93FF938FE197E017DCFF91EF9144
:10BCB000BF91AF919F918F917F916F915F914F91C4
:10BCC0003F912F910F900BBE0F900FBE0F901F90C2
:10BCD00018951F920F920FB60F9211240BB60F9268
:10BCE0002F933F934F935F936F937F938F939F9384
:10BCF000AF93BF93EF93FF938FE197E070DBFF91DA
:10BD0000EF91BF91AF919F918F917F916F915F91D3
:10BD10004F913F912F910F900BBE0F900FBE0F9040
:10BD20001F9018951F920F920FB60F9211240BB609
:10BD30000F922F933F934F935F936F937F938F93C4
:10BD40009F93AF93BF93EF93FF938CEB97E0C5DB8B
:10BD5000FF91EF91BF91AF919F918F917F916F91E3
:10BD60005F914F913F912F910F900BBE0F900FBE9F
:10BD70000F901F9018951F920F920FB60F921124DB
:10BD80000BB60F922F933F934F935F936F937F93D5
:10BD90008F939F93AF93BF93EF93FF938CEB97E0B9
:10BDA0001EDBFF91EF91BF91AF919F918F917F919A
:10BDB0006F915F914F913F912F910F900BBE0F901C
:10BDC0000FBE0F901F9018951F920F920FB60F92F3
:10BDD00011240BB60F922F933F934F935F936F9362
:10BDE0007F938F939F93AF93BF93EF93FF9389E5D7
:10BDF00098E073DBFF91EF91BF91AF919F918F918D
:10BE00007F916F915F914F913F912F910F900BBE5A
:10BE10000F900FBE0F901F9018951F920F920FB6A4
:10BE20000F9211240BB60F922F933F934F935F9372
:10BE30006F937F938F939F93AF93BF93EF93FF93F2
:10BE400089E598E0CCDAFF91EF91BF91AF919F9196
:10BE50008F917F916F915F914F913F912F910F90B3
:10BE60000BBE0F900FBE0F901F9018951F920F9250
:10BE70000FB60F9211240BB60F922F933F934F934F
:10BE80005F936F937F938F939F93AF93BF93EF9342
:10BE9000FF9386EF98E021DBFF91EF91BF91AF9187
:10BEA0009F918F917F916F915F914F913F912F91D2
:10BEB0000F900BBE0F900FBE0F901F9018951F9202
:10BEC0000F920FB60F9211240BB60F922F933F9340
:10BED0004F935F936F937F938F939F93AF93BF9392
:10BEE000EF93FF9386EF98E07ADAFF91EF91BF919D
:10BEF000AF919F918F917F916F915F914F913F9102
:10BF00002F910F900BBE0F900FBE0F901F901895A2
:10BF1000CF93DF93EC01E881F9810680F781E02D72
:10BF20001995EA89FB8980818F7E8083EA89FB8964
:10BF30008081877F8083EA89FB8980818F778083F6
:10BF4000EA89FB8980818F7D80838A8D898FDF914B
:10BF5000CF910895CF92DF92EF92FF921F93CF93EC
:10BF6000DF93EC016A017B01122FE889F98982E0F5
:10BF700080834115514E61057105B1F060E079E0B3
:10BF80008DE390E0A70196010E94BDBEDA01C901D0
:10BF90000197A109B109B695A79597958795AC0129
:10BFA000411580E15807A8F0E889F989108260E816
:10BFB00074E88EE190E0A70196010E94BDBEBA012F
:10BFC000A901415051096109710976956795579505
:10BFD0004795EC85FD855083EE85FF854083188E5F
:10BFE000EC89FD891083EA89FB89808180618083E7
:10BFF000EA89FB89808188608083EA89FB89808166
:10C0000080688083EA89FB8980818F7D8083DF91CE
:10C01000CF911F91FF90EF90DF90CF900895CF9335
:10C02000DF93282F30E0F901E25DFB4E8491F901A6
:10C03000E851FC4ED491F901EE55FC4EC491CC234D
:10C0400089F08111FBDAEC2FF0E0EE0FFF1FE857CB
:10C05000FC4EA591B491EC91ED2381E090E021F4A8
:10C0600080E002C080E090E0DF91CF9108951F93BF
:10C07000CF93DF93282F30E0F901E25DFB4E8491EE
:10C08000F901E851FC4ED491F901EE55FC4EC491F2
:10C09000CC23C1F0162F8111D1DAEC2FF0E0EE0F96
:10C0A000FF1FE259FC4EA591B4918FB7F89411117E
:10C0B00005C09C91ED2FE095E92302C0EC91ED2B9A
:10C0C000EC938FBFDF91CF911F910895CF93DF93B2
:10C0D00090E0FC01E851FC4E2491FC01EE55FC4E31
:10C0E0008491882361F190E0880F991FFC01EC5A3C
:10C0F000FC4EC591D491FC01E259FC4EA591B4913E
:10C10000611109C09FB7F8948881209582238883A4
:10C11000EC912E230BC0623061F49FB7F894388104
:10C12000822F809583238883EC912E2B2C939FBFA5
:10C1300006C08FB7F894E8812E2B28838FBFDF913C
:10C14000CF9108951F93CF93DF93182FEB0161E0F8
:10C15000BDDF209711F460E004C0CF3FD10531F47A
:10C1600061E0812FDF91CF911F9181CFE12FF0E02E
:10C17000E25DFB4EE4914E2F50E0FA013197E2313F
:10C18000F10508F09DC08827ED56FE4F8F4F0C94A7
:10C19000ADC084B5806884BDC7BD97C084B58062DA
:10C1A00084BDC8BD92C0809180008068809380006B
:10C1B000D0938900C093880088C0809180008062FD
:10C1C00080938000D0938B00C0938A007EC08091C2
:10C1D0008000886080938000D0938D00C0938C0095
:10C1E00074C08091B00080688093B000C093B300A9
:10C1F0006CC08091B00080628093B000C093B400A6
:10C2000064C080919000806880939000D0939900E2
:10C21000C09398005AC080919000806280939000F3
:10C22000D0939B00C0939A0050C08091900088608A
:10C2300080939000D0939D00C0939C0046C0809155
:10C24000A00080688093A0008091A0008F7B8093E5
:10C25000A000D093A900C093A80037C08091A0008F
:10C2600080628093A000D093AB00C093AA002DC041
:10C270008091A00088608093A000D093AD00C0930F
:10C28000AC0023C080912001806880932001D0936E
:10C290002901C093280119C08091200180628093F8
:10C2A0002001D0932B01C0932A010FC0809120015F
:10C2B000886080932001D0932D01C0932C0105C08C
:10C2C000C038D1050CF04CCF46CFDF91CF911F91F4
:10C2D0000895863308F0865390917B00282F2870AC
:10C2E000977F922B90937B008770806480937C0073
:10C2F00080917A00806480937A0080917A0086FD34
:10C30000FCCF809178002091790090E0922B0895E5
:10C3100080910C02882311F0599801C0599A90918C
:10C320000C0281E0892780930C02089561E089E284
:10C330009ECE1092030B40914A0650914B0660E04E
:10C3400070E02DED31E680913806909139060C941D
:10C35000F3540F931F93CF93DF9360E08BE287DE5C
:10C3600000918E1210918F12C0913806D09139062B
:10C37000B801CE010E948C54882341F0B801CE014F
:10C38000DF91CF911F910F910C94A454DF91CF9125
:10C390001F910F91089580915506882369F080912F
:10C3A000020B882349F081E08093FF0A80915406B4
:10C3B0000E9463420C9483900895CF93DF93CDB78E
:10C3C000DEB765970FB6F894DEBF0FBECDBF81E034
:10C3D0008093030B80918B12882371F182E390E0AC
:10C3E0009A83898388E290E09C838B838EE690E039
:10C3F0009E838D8384EF91E098878F831D8A84E0EC
:10C400008F938DB79EB745970FB6F8949EBF0FBE1A
:10C410008DBFADB7BEB7119685E1FE013196019093
:10C420000D928A95E1F78DE09AE00E946F850FB634
:10C43000F894DEBF0FBECDBF65960FB6F894DEBF91
:10C440000FBECDBFDF91CF91089560E089E20FDE8E
:10C4500026E931E642E350E060E070E08091380682
:10C46000909139060C94F35461E08BE200DEE89A77
:10C4700029EA31E648E853E160E070E0809138064F
:10C48000909139060E94F35490938F1280938E12EC
:10C49000089561E08BE2EBDDE89A29EA31E648E8AD
:10C4A00053E160E070E080913806909139060E9477
:10C4B000F35490938F1280938E12089581E2AFDD32
:10C4C00021E0892B09F420E0822F08958091500605
:10C4D000882309F44CC08091020B882309F447C0DB
:10C4E00081E08093FF0AEADF882329F080915306D8
:10C4F0008823D9F106C080915106811105C0809131
:10C5000050060E94634231C090915006963069F502
:10C51000823081F08330D1F0813039F5E091670AC3
:10C52000F091680A74978081918145E550E060E060
:10C5300070E017C0E091670AF091680A74978081F3
:10C5400091814AE550E060E070E00BC0E091670A3D
:10C55000F091680A7497808191814FE550E060E026
:10C5600070E08959954F0E94088C0C94839008952F
:10C5700080918D12882339F080918C12882319F0D4
:10C5800081E08093FC0A80913A0690913B06DC01A1
:10C59000ED91FC91008CF18DE02D19958091871221
:10C5A000811153DF80918612882389F061E088E051
:10C5B0005EDD409184125091851260E070E027E2C8
:10C5C00033E980913806909139060E94F3548091A6
:10C5D0008D12882321F080918C12811101C076DFA9
:10C5E00080918C12882379F080918D12882359F0E4
:10C5F00080918A12882339F0E0918812F091891293
:10C6000082810E94625695CE1F920F920FB60F92B2
:10C6100011240BB60F922F933F934F935F936F9319
:10C620007F938F939F93AF93BF93EF93FF938091EB
:10C630008D128823A9F0489917C0E89829EA31E6B5
:10C640004CE251E060E070E080913806909139064C
:10C650000E94F35480918C12882331F089DF04C04A
:10C66000489B02C0E89875DEFF91EF91BF91AF91B2
:10C670009F918F917F916F915F914F913F912F91FA
:10C680000F900BBE0F900FBE0F901F9018958091CA
:10C69000010B811156C012DF8823F1F081E08093F5
:10C6A000010B80913A0690913B06DC01ED91FC91E3
:10C6B0000488F589E02D19950E94439127E631E918
:10C6C00048E95AE360E070E08091380690913906BD
:10C6D0000E94F3542EDE09C080918C12882329F128
:10C6E00080918D12882311F0D4DEF0CEBDDE8091D2
:10C6F0008A12882339F0E0918812F09189128281A0
:10C700000E946256409182125091831214161506AF
:10C71000BCF4052E000C660B770B28EB32E68091FB
:10C720003806909139060C94F35480918A1288232C
:10C7300039F0E0918812F091891282810E9462564C
:10C7400017CF08950F931F9320918112211136C0A6
:10C750004EEB50EA61E077279C01220F331F820FD6
:10C76000931F092E000CAA0BBB0B0296A11DB11D35
:10C77000840F951FA61FB71FABBFFC0187910EEB5F
:10C7800010EA21E033274091661293E0499FA0010F
:10C790001124052E000C660B770B4E5F5F4F6F4F19
:10C7A0007F4F040F151F261F371F2BBFF80107915E
:10C7B000801720F01F910F910C945E741F910F91C0
:10C7C0000895833091F028F4813049F0823051F09F
:10C7D0000895853081F060F0863081F0089589E019
:10C7E00090E00EC08AE090E00BC08BE090E008C0C3
:10C7F0008CE090E005C08DE090E002C08EE090E01B
:10C80000A1CF8F929F92AF92BF92CF92DF92EF9281
:10C81000FF920F931F93CF93DF93EC01A62E80918D
:10C82000811281116BC04EEB50EA61E077276E01F7
:10C83000CC0CDD1CCC0EDD1E0D2C000CEE08FF0810
:10C84000D701C6010296A11DB11D480F591F6A1FCD
:10C850007B1F6BBFFA0187914EEB50EA61E07727AF
:10C86000B090661293E0B99E80011124012E000C55
:10C87000220B330B0E5F1F4F2F4F3F4F400F511FA7
:10C88000621F731F6BBFFA014791481708F036C04B
:10C89000809064129090651200917A1210917B1230
:10C8A000B401C8010E948C54882321F0B401C8014E
:10C8B0000E94A4548EEB90EAA1E0BB278C0D9D1D35
:10C8C000AE1DBF1DABBFFC016791769182E00E9457
:10C8D0001456B0926312C0936612AA2079F0109297
:10C8E00062122EE534E742E350E060E070E0C801F8
:10C8F0000E94F3549093651280936412DF91CF915C
:10C900001F910F91FF90EF90DF90CF90BF90AF906D
:10C910009F908F900895CF92DF92EF92FF92809137
:10C920008112811134C080918012882381F161E0ED
:10C930008EE090E066DF60917E1270917F12CB01F5
:10C94000A0E0B0E0C0907C12D0907D12E12CF12CE0
:10C95000C816D906EA06FB0664F4BC01CD016C19C1
:10C960007D098E099F090E94945CC60ED71EE81EA1
:10C97000F91E2BE834E6B701A60180917A12909156
:10C980007B120E94F3549093791280937812FF9057
:10C99000EF90DF90CF900895CF92DF92EF92FF92C9
:10C9A00080918112811134C080917712882381F1A6
:10C9B00061E08DE090E025DF609175127091761254
:10C9C000CB01A0E0B0E0C0907312D0907412E12CC3
:10C9D000F12CC816D906EA06FB0664F4BC01CD01A9
:10C9E0006C197D098E099F090E94945CC60ED71EA2
:10C9F000E81EF91E2CEC34E6B701A60180917A12EC
:10CA000090917B120E94F354909372128093711252
:10CA1000FF90EF90DF90CF900895CF92DF92EF924A
:10CA2000FF9280918112811134C08091701288230D
:10CA300081F161E08CE090E0E4DE60916E12709133
:10CA40006F12CB01A0E0B0E0C0906C12D0906D12DC
:10CA5000E12CF12CC816D906EA06FB0664F4BC01E9
:10CA6000CD016C197D098E099F090E94945CC60E48
:10CA7000D71EE81EF91E2DE035E6B701A60180910C
:10CA80007A1290917B120E94F35490936B128093D0
:10CA90006A12FF90EF90DF90CF90089580918112FD
:10CAA00081112CC080916912882341F0809170120D
:10CAB000811104C081E080937012AFDF8091681211
:10CAC000882361F080918112811108C080917712D2
:10CAD000811104C081E0809377125EDF809167123C
:10CAE000882361F080918112811108C080918012A9
:10CAF000811104C081E0809380120DCF08952F92A0
:10CB00003F924F925F926F927F928F929F92AF92DD
:10CB1000BF92CF92DF92EF92FF920F931F93CF932A
:10CB2000DF9300D01F92CDB7DEB75C010E94843F37
:10CB30000E94567A0E948D7A8091D1069091D206F9
:10CB40007CD80E94F17F24E0A216B10409F49BC0B6
:10CB50000CF04EC0A3E0AA16B10409F03BC18CE171
:10CB600090E00E94C1C09C838B8380EF95E0AB81F5
:10CB7000BC8111969C938E931396BC92AE921297A1
:10CB800081E09FEF15969C938E9314978FEF90E022
:10CB900017969C938E93169719961C921E9218972F
:10CBA00058961C925897CD010E94AE5784EE95E09E
:10CBB000EB81FC8191838083E0917613F091771370
:10CBC000D08C009153111091541116950795E09057
:10CBD0005111F0905211F694E79466E775E1809157
:10CBE000D1069091D2063CD8812C9924939412C1FD
:10CBF000B5E0AB16B10409F4A6C0E6E0AE16B10488
:10CC000009F0E8C08CE190E00E94C1C09C838B8356
:10CC100080EF95E0AB81BC8111969C938E93139627
:10CC2000BC92AE92129781E09FEF15969C938E93E3
:10CC300014978FEF90E017969C938E931697199602
:10CC40001C921E92189758961C925897CD010E94DC
:10CC5000AE5784EE95E0EB81FC8191838083E09177
:10CC6000BD06F091BE06D08C0091921110919311E7
:10CC700016950795E0909011F0909111F694E79435
:10CC800069EA75E1A0C08CE190E00E94C1C09C837C
:10CC90008B8380EF95E0AB81BC8111969C938E9342
:10CCA0001396BC92AE92129781E09FEF15969C93DB
:10CCB0008E9314978FEF90E017969C938E93169710
:10CCC00019961C921E92189758961C925897CD014F
:10CCD0000E94AE5784EE95E0EB81FC8191838083C6
:10CCE000009168111091691116950795E0906611F1
:10CCF000F0906711F694E79480912D0F8C5082305C
:10CD000040F4E091CF06F091D006D08C69EE75E149
:10CD10005AC08091750F823009F07AC080912B0F34
:10CD20008C3009F075C0E091BD06F091BE06D08C44
:10CD300069EC75E18091D1069091D2060E94305E37
:10CD40008824839466C08CE190E00E94C1C09C83DB
:10CD50008B8380EF95E0AB81BC8111969C938E9381
:10CD60001396BC92AE92129781E09FEF15969C931A
:10CD70008E9314978FEF90E017969C938E9316974F
:10CD800019961C921E92189758961C925897CD018E
:10CD90000E94AE5784EE95E0EB81FC819183808305
:10CDA000E091CB06F091CC06D08C00917D111091D2
:10CDB0007E1116950795E0907B11F0907C11F6940A
:10CDC000E79469E875E18091D1069091D2060E94BE
:10CDD000305E1EC06DE575E18091D1069091D2065E
:10CDE0000F900F900F900F90DF91CF911F910F91A7
:10CDF000FF90EF90DF90CF90BF90AF909F908F907B
:10CE00007F906F905F904F903F902F900C94305E8A
:10CE1000812C912C0E94F17F60E575E18091D10613
:10CE20009091D2060E94305E64E475E18091D10653
:10CE30009091D2060E94BF5CB8018091D10690917A
:10CE4000D2060E946D4668E375E18091D10690910B
:10CE5000D2060E94BF5CB7018091D1069091D206A4
:10CE60000E946D466CE275E18091D1069091D206E8
:10CE70000E94BF5C8D2D0E94C77F8091D10690914A
:10CE8000D2060E941D5EAB81BC81ED91FC91119791
:10CE90000280F381E02DCD011995CA2C8A2D0E94C4
:10CEA000CB568D3D9540A8F464E378E08A2D0E942E
:10CEB000C356EB81FC81F78AE68AB70182810E9422
:10CEC000DB566CED75E08A2D0E94C756DD20C1F05F
:10CED0001AC064E873E08A2D0E94C756AB81BC81FA
:10CEE00057961C930E935697B80112968C910E94F8
:10CEF000DB566CED75E08A2D0E94C356DD2019F0DB
:10CF00003324339401C0312C21E02983212C2A833E
:10CF10000E94A64C8091FC10882359F1AB81BC8102
:10CF2000ED91FC91119760910111709102110190A6
:10CF3000F081E02DCD0119958C2D0E94CB568D3DB1
:10CF4000B5E09B075CF48438E3E09E0784F08C0135
:10CF50008D3D954074F00CED15E00BC07C018533E0
:10CF600098403CF064E3E62E68E0F62E02C004E848
:10CF700013E02A8121111FC08091F2108823C9F18A
:10CF8000E091F910F091FA10858196814091F510A9
:10CF90005091F6109C0121533109421753074CF16F
:10CFA000C196841795072CF10E9488936415750526
:10CFB00086059705F0F08091F2108823C1F040912A
:10CFC000F5105091F610E091F910F091FA1085816A
:10CFD00096819C01285C3109421753072CF0885335
:10CFE0009F4F841795071CF481E0382605C021E087
:10CFF0002A83222009F47CC0332009F445C0DD20B7
:10D00000F9F064E873E08C2D0E94C756992009F46A
:10D0100058C06091470F7091480F41E08C2D0E94DD
:10D0200082560E941399AB81BC8112968C910E940A
:10D03000CB5608171907ACF38C2D0E94545641C0EB
:10D0400064E378E08C2D0E94C3569920B1F0609182
:10D05000470F7091480F40E08C2D0E9482560E942D
:10D060001399AB81BC8112968C910E94CB568E1580
:10D070009F05ACF38C2D0E945456EB81FC81F78AFE
:10D08000E68AB701828110C0DD20B1F064E378E068
:10D090008C2D0E94C356AB81BC815796FC92EE92B8
:10D0A0005697B70112968C910E94DB566CED75E095
:10D0B0008C2D0E94C75612C064E873E08C2D0E942C
:10D0C000C756EB81FC81178B068BB80182810E94C9
:10D0D000DB566CED75E08C2D0E94C3560E94889340
:10D0E0002B013C01F8EC4F0E511C611C711C1A8283
:10D0F00029812223D9F18091E8108823A9F1409158
:10D10000EB105091EC10E091EF10F091F010858150
:10D1100096819C01285C3109421753072CF08853F3
:10D120009F4F8417950704F581E0D8268091D1069A
:10D130009091D206DD2039F06DE175E10E94305EFC
:10D1400082E090E006C06BE075E10E94305E81E015
:10D1500090E00E945E7A0E948893AB81BC815896D1
:10D16000DC922224239403C0212C1EC0212C809108
:10D17000E810882309F472C2E091EF10F091F010EA
:10D18000858196814091EB105091EC109C012153C8
:10D190003109421753070CF461C2C19621E029837B
:10D1A000841795070CF45AC20E94C1590E94B545D4
:10D1B0008EE89BE00E94035580911B0B882309F4A5
:10D1C000A7CE80911D0B882309F4A2CE0E94B545FD
:10D1D0000E9429498823D1F384E0A816B104D9F12B
:10D1E00034F4B3E0AB16B10409F438C1C4C1E5E0CE
:10D1F000AE16B10409F4CDC0F6E0AF16B10409F0E3
:10D20000BAC110933B0F00933A0FF0923D0FE0929A
:10D210003C0FD0923E0FB8018CE291E00E9446454F
:10D22000B7018EE291E00E9446456D2D80E391E0CA
:10D230000E94A246B80186E00E94F955B70186E037
:10D240000E94DE55E091BD06F091BE06D08E6CEDD9
:10D2500075E086E091C08820C1F010933B0F0093E9
:10D260003A0FF0923D0FE0923C0FD0923E0FB80182
:10D270008CE291E00E944645B7018EE291E00E9467
:10D2800046456D2D80E391E017C010932F0F00935A
:10D290002E0FF092310FE092300FD092320FB80182
:10D2A00080E291E00E944645B70182E291E00E944F
:10D2B00046456D2D84E291E00E94A246B80184E0CB
:10D2C0000E94F955B70184E00E94DE55882049F09C
:10D2D000E091BD06F091BE06D08E6CED75E084E065
:10D2E0004BC0E091CF06F091D006D08E80912D0FEB
:10D2F0008D3029F4E0919112F0919212D08E6CED64
:10D3000075E084E00E94DB5666E970E080E090E022
:10D310000E94509380912D0F8D3011F584E00E9472
:10D32000CB56A091CF06B091D0068D3D95404CF0E4
:10D33000ED91FC9111970190F081E02D6FEF7FEF5F
:10D3400008C0ED91FC9111970190F081E02D61E012
:10D3500070E0CD0119958091CF069091D0066FC0F5
:10D360008091CF069091D006DC01ED91FC91048074
:10D37000F581E02D1995FFC00E94DB5666E970E04B
:10D3800080E090E00E9450938091BD069091BE068F
:10D39000EBCF1093360F0093350FF092380FE092D9
:10D3A000370FD092390FB80187E291E00E944645CD
:10D3B000B70189E291E00E9446456D2D8BE291E034
:10D3C0000E94A246B80185E00E94F955B70185E0A8
:10D3D0000E94DE55E091CB06F091CC06D08E6CED2C
:10D3E00075E085E00E94DB5666E970E080E090E041
:10D3F0000E94509380912C0F8D3059F585E00E944A
:10D40000CB56A091CB06B091CC068D3D95404CF00B
:10D41000ED91FC9111970190F081E02D6FEF7FEF7E
:10D4200008C0ED91FC9111970190F081E02D61E031
:10D4300070E0CD0119958091CB069091CC06DC016E
:10D44000ED91FC910190F081E02D60E070E0199584
:10D4500092C08091CB069091CC0686CF10934A0F54
:10D460000093490FF0924C0FE0924B0FD092430F74
:10D47000B8018BE391E00E944645B7018DE391E04E
:10D480000E9446456D2D85E391E00E94A246B801B9
:10D4900083E00E94F955B70183E00E94DE55809138
:10D4A000430FE0917613F0917713808F8091430FB3
:10D4B0000E94114583E00E94CB562091430F222306
:10D4C00069F1B9E0BC1538F0209153113091541135
:10D4D0003695279502C02EEE32E08217930709F4A5
:10D4E0004AC06091470F7091480F41E083E00E946D
:10D4F00082560E941399EB81FC8182810E94CB5657
:10D5000008171907B4F383E00E945456AB81BC811D
:10D5100057961C930E935697B80129C029E02C15F5
:10D5200008F49EC0209151113091521136952795E3
:10D530008217930701F16091470F7091480F40E007
:10D5400083E00E9482560E941399EB81FC818281C4
:10D550000E94CB568E159F05B4F383E00E9454566B
:10D56000AB81BC815796FC92EE925697B70112960A
:10D570008C910E94DB568091D1069091D2060E9438
:10D580001D5E0E94F17FB4E0AB16B10459F0E5E0F6
:10D59000AE16B10451F0F3E0AF16B10471F461ECD2
:10D5A00074E105C061EF74E102C068ED74E180913F
:10D5B000D1069091D2060E94305E0E94F17F66EB08
:10D5C00074E18091D1069091D2060E94305E6AEAA1
:10D5D00074E18091D1069091D2060E94BF5CB8019F
:10D5E0008091D1069091D2060E946D466EE974E159
:10D5F0008091D1069091D2060E94BF5CB7018091C4
:10D60000D1069091D2060E946D4662E974E1809144
:10D61000D1069091D2060E94BF5C8D2D0E94C77FDB
:10D620008091D1069091D2060E941D5E0F900F90BE
:10D630000F900F90DF91CF911F910F91FF90EF907E
:10D64000DF90CF90BF90AF909F908F907F906F9022
:10D650005F904F903F902F900C94897A1982A4CDBF
:10D660002AEC38E065CFCF93DF93CDB7DEB72897AC
:10D670000FB6F894DEBF0FBECDBF80919012882305
:10D68000E1F1109290120E94017A81E080930302EE
:10D690008091D406882389F163E874E18091D106F2
:10D6A0009091D2060E94BF5CE091170BE4300CF021
:10D6B000E0E08EEB95E09A8389838AEB95E09C838A
:10D6C0008B8385EB95E09E838D8380EB95E0988737
:10D6D0008F83EE0FFF0BEC0FFD1F61817281809134
:10D6E000D1069091D20628960FB6F894DEBF0FBEF1
:10D6F000CDBFDF91CF910C94305E28960FB6F89491
:10D70000DEBF0FBECDBFDF91CF9108958091901203
:10D71000811113C00E94843F81E0809390120E9487
:10D720001D7A8091D306882341F064E774E18091EB
:10D73000D1069091D2060C94305E08950895089514
:10D74000FC01828193818830910529F410922B018C
:10D7500010922A010895099721F41092290110923C
:10D7600028010895FC01178A168A6CED75E0828104
:10D770000C94DB56CF93DF93EC011F8A1E8A8A81BB
:10D780000E9454568B8D882331F08A810E94CB569B
:10D790009A8F898F1B8EDF91CF910895DF92EF9240
:10D7A000FF920F931F93CF93DF93EC018A8189300F
:10D7B00010F40E943B56DD8C6B8D7C8D098D1A8D8B
:10D7C000EA80FB8089E08E1508F466C00F301105F1
:10D7D00038F001369DE6190728F000E61DE602C084
:10D7E0000FE010E06F30710538F061368DE6780794
:10D7F00028F060E67DE602C06FE070E080E090E037
:10D800000E944CBD20E030E04AE754E40E9453BF40
:10D8100020E030E04CE852E40E94ADBD9B01AC0139
:10D8200060E070E08AEF94E40E9453BF0E94BBBFA7
:10D83000FF2425E12E9DF0012F9DF00D1124E15FC5
:10D84000FE4EDD2071F023813481AB0177FF04C0EF
:10D8500044275527461B570B88279927841B950B70
:10D860000AC025813681AB0177FF04C044275527C4
:10D87000461B570BCA014FB7F89455E15E9DF00166
:10D880005F9DF00D1124E15FFE4E108B0787328BF8
:10D89000218B948B838B4FBF9D8D6B8D7C8D8A816B
:10D8A0009923F9F08A3058F495E1899FF001112409
:10D8B000E15FFE4E058116811695079502C00EEEBA
:10D8C00012E041E00E94825661E070E080E090E06A
:10D8D0000E9450938A810E94CB5608171907A0F323
:10D8E0001EC08A3058F495E1899FF0011124E15F50
:10D8F000FE4E038114811695079502C00AEC18E0CC
:10D9000040E00E94825661E070E080E090E00E947A
:10D9100050938A810E94CB5680179107A0F38A8189
:10D920000E945456B8018A81DF91CF911F910F91C7
:10D93000FF90EF90DF900C94DB56CF93DF93EC01D8
:10D940008A81893010F40E943B5648EE53E05B8791
:10D950004A8720ED37E03D872C878CED95E09F8747
:10D960008E87598B488B3B8B2A8B9D8B8C8BDF91C1
:10D97000CF910895CF93DF93EC017F8B6E8B8885D9
:10D9800099856817790769F48A810E9454568B8DAE
:10D99000882329F18A810E94CB569A8F898F1B8E0A
:10D9A0001EC0CE010E944689EA81EA30B0F49C0193
:10D9B000C39714F022E330E02E3C8FEF380714F4C5
:10D9C0002EEC3FEF8FB7F89495E1E99FF001112419
:10D9D000E15FFE4E318720878FBF81E08B8FDF9123
:10D9E000CF9108950F931F93CF93DF938C01FC0188
:10D9F000778B668B0E944689EC01F80182819381C6
:10DA000088309105D1F4D7FF06C060E08AE00E941B
:10DA1000376061E005C061E08AE00E94376060E045
:10DA200086E00E943760D7FF03C0D195C195D10928
:10DA3000D0932B01C0932A011BC00997C9F4D7FFCB
:10DA400006C060E08DE00E94376061E005C061E0E3
:10DA50008DE00E94376060E08BE00E943760D7FF66
:10DA600003C0D195C195D109D0932901C093280154
:10DA7000DF91CF911F910F910895CF93DF93EC0128
:10DA80008A81893010F40E943B562EEC3FEF3B8791
:10DA90002A8782E390E09D878C871F861E86398BBC
:10DAA000288B9B8B8A8B1D8A1C8A6EEE72E08A8182
:10DAB0000E94C7566AEC78E08A810E94C3568CEDBA
:10DAC00095E09A8F898F1B8EDF91CF910895CF9328
:10DAD000DF93EC0121E03FEF3B872A878FEF90E057
:10DAE0009D878C871F861E86398B288B9B8B8A8B04
:10DAF0001D8A1C8A61E08AE00E94666061E086E01F
:10DB00000E94666061E08DE20E94666061E08DE0E7
:10DB10000E94666061E08BE00E94666061E08EE2D8
:10DB20000E9466608A819B818830910529F4109259
:10DB30002B0110922A0106C0099721F410922901A5
:10DB400010922801DF91CF9108950F931F93CF93E7
:10DB5000DF938C01FC01178A168AEC01699640E07C
:10DB600068E0CE010E94349A4FE766E0CE010E9441
:10DB7000349A40E06CE0CE010E94349A4FE767E0AF
:10DB8000CE010E94349A0E948893F801648F758FA9
:10DB9000868F978FDF91CF911F910F910895EF920C
:10DBA000FF920F931F93CF93DF938C01FC01778B30
:10DBB000668B0E944689EC01F8018281938188304E
:10DBC000910531F57801F9E1EF0EF11CD7FF06C0A0
:10DBD0006AE0C1388FEFD80754F001C068E02C2FFD
:10DBE0009D2FC038D1052CF02FE790E002C021E82E
:10DBF0009FEF422F592F57FF03C05195419551096F
:10DC0000C7010E94349ACD2B69F54FE766E027C023
:10DC1000099741F57801E9E1EE0EF11CD7FF06C046
:10DC20006EE0C138FFEFDF0754F001C06CE02C2F2D
:10DC30009D2FC038D1052CF02FE790E002C021E8DD
:10DC40009FEF422F592F57FF03C05195419551091E
:10DC5000C7010E94349ACD2B29F44FE767E0C70132
:10DC60000E94349A0E948893F801648F758F868F82
:10DC7000978FDF91CF911F910F91FF90EF900895B3
:10DC80000F931F93CF93DF93EC010E9488930C8D29
:10DC90001D8D2E8D3F8DDC01CB01801B910BA20BC6
:10DCA000B30B853F9140A105B10540F06E897F8996
:10DCB000CE01DF91CF911F910F9171CFDF91CF9165
:10DCC0001F910F910895CF93DF93EC0180919412EF
:10DCD000811109C06A8D7B8DCE0149960E948445D1
:10DCE00081E08093941221E83FEF3B872A878FE7FA
:10DCF00090E09D878C871F861E86398B288B9B8B97
:10DD00008A8B1D8A1C8ADF91CF9108956F927F9232
:10DD10008F929F92AF92BF92CF92DF92EF92FF923B
:10DD20000F931F93CF93DF938091A2139091A3132E
:10DD3000DC01ED91FC910084F185E02D1995B12C69
:10DD4000181619060CF0D1C0AA24A3948091A2132E
:10DD50009091A313DC01ED91FC910084F185E02DFD
:10DD60001995892B09F4C1C0C091EE1281E08C0F86
:10DD70008093EE128091A2139091A313DC01ED9198
:10DD8000FC910284F385E02D1995EC2FF0E0E2552B
:10DD9000FD4E80838A30D1F6E090EE12F12C109285
:10DDA000DA0D1092D90D1092D50D1092D60D109259
:10DDB000D70D1092D80D1092D40D1092D30D109251
:10DDC000D20D8EEAC82E82E1D82E00E010E0D0E01D
:10DDD000C0E00E151F050CF06CC0F60191916F01AB
:10DDE0009D3009F463C09C3789F19A3009F052C024
:10DDF000D33009F059C0CC2309F456C06C2E712CD5
:10DE0000C30101970E94DE487093DA0D6093D90D2B
:10DE10000E9488936093A5137093A6138093A71311
:10DE20009093A81380919312882309F45BC080908B
:10DE3000D90D9090DA0DB801661977098EEA92E152
:10DE40000E94729B8816990679F54CC08C2F90E041
:10DE5000FC01ED5FF14F1082D13099F068F0D230C3
:10DE6000B1F40E94DE486093D50D7093D60D809377
:10DE7000D70D9093D80D0BC00E94DE486093D20D51
:10DE800006C00E94DE487093D40D6093D30DDF5F0F
:10DE9000C0E00CC00F3311053CF4EC2FF0E0ED5F57
:10DEA000F14F9083CF5F02C01092AD120F5F1F4FF2
:10DEB00090CF8091AD1281110EC08091CF0D9091C5
:10DEC000D00D01969093D00D8093CF0D60E087E840
:10DED0000E94189C02C0BB24B3941092AE12109200
:10DEE000EE1234CFA092AD12E1CF8B2DDF91CF9106
:10DEF0001F910F91FF90EF90DF90CF90BF90AF9068
:10DF00009F908F907F906F900895CF931092D10D36
:10DF10001092CE0D1092D00D1092CF0D61E089E3DA
:10DF20000E9437600E94199B8091A2139091A313C5
:10DF3000DC01ED91FC910084F185E02D1995892B90
:10DF400061F08091A2139091A313DC01ED91FC91FB
:10DF50000284F385E02D1995E7CF0E94939C809170
:10DF6000A2139091A313DC01ED91FC910680F7813F
:10DF7000E02D19951092A4130E9488936093A51325
:10DF80007093A6138093A7139093A813C1E0BEDEED
:10DF900081110E94AE340E94569B0E94C15980910B
:10DFA000CF0D9091D00D0A9724F48091A41388236B
:10DFB00031F060E08AE80E94189CC093D10D8091F6
:10DFC000D10D882321F38091CE0D882341F040EEBE
:10DFD00051E060E070E08EE09EE00E9461BE60E093
:10DFE00089E30E94376060E08AE3CF910C94376048
:10DFF000EF92FF920F931F93CF93DF9300D000D047
:10E00000CDB7DEB769E276E0CE0101960E94805C72
:10E010000D811E81F02EEE24E3948091A213909145
:10E02000A313DC01ED91FC910084F185E02D19959D
:10E03000892B21F18091A2139091A313DC01ED9122
:10E04000FC910284F385E02D19958F3439F4E09228
:10E05000AC128093A112E092A012DFCF9091AC128B
:10E060009923D9F2E091A01291E09E0F9093A01213
:10E07000F0E0EF55FD4E80839F1578F28091A0125D
:10E080008F1510F4F12C21C04BE050E065E972E1EE
:10E09000CE0101960E943E48A1EAB2E1E9E2F6E033
:10E0A000FF24F3941127CF018952964080179107DE
:10E0B00034F49D9181919817B1F3F12CF4CF109223
:10E0C000A1121092AC121092A012CE0101960E94E1
:10E0D000505C8F2D26960FB6F894DEBF0FBECDBFD5
:10E0E000DF91CF911F910F91FF90EF900895DC0188
:10E0F000ED91FC910190F081E02D1994CF93DF9385
:10E10000EC017F8B6E8B0E944689BC018A81DF9176
:10E11000CF910C94DB5608950895089508950895BD
:10E12000623039F0633041F0613041F4409369125C
:10E1300008954093681208954093671208956230DD
:10E1400069F06330A1F06130D1F450936D124093C7
:10E150006C1230936F1220936E12089550937412C4
:10E160004093731230937612209375120895509352
:10E170007D1240937C1230937F1220937E1208957B
:10E18000FC018581089508950895089508952091CA
:10E190008112211102C0FC01628308952091811235
:10E1A000211102C0FC016483089520918112211184
:10E1B00002C0FC016383089508950895809181123F
:10E1C000811101C092C30895089580E008950895D3
:10E1D00008950895089508950895809181128111F8
:10E1E00004C08FE090E00C94A26308952091811206
:10E1F000211108C0FC018481882321F082E090E095
:10E200000C94A263089520918112211108C0FC0191
:10E210008381882321F081E090E00C94A26308952B
:10E2200080918112811104C08BE090E00C94A26374
:10E23000089580918112811105C060E080E190E035
:10E240000C940164089580918112811105C060E0F1
:10E250008FE090E00C940164089580918112811107
:10E2600027C06330A1F028F4613049F0623059F0E2
:10E2700008956530A1F078F06630A9F0089560E067
:10E2800089E090E013C060E08AE090E00FC060E0B9
:10E290008BE090E00BC060E08CE090E007C060E0B5
:10E2A0008DE090E003C060E08EE090E00C940164AB
:10E2B000089580918112811127C06330A1F028F464
:10E2C000613049F0623059F008956530A1F078F07E
:10E2D0006630A9F0089561E089E090E013C061E044
:10E2E0008AE090E00FC061E08BE090E00BC061E05D
:10E2F0008CE090E007C061E08DE090E003C061E059
:10E300008EE090E00C940164089520918112211117
:10E3100009C0FC018281882329F061E088E090E057
:10E320000C940164089520918112211109C0FC010F
:10E330008481882329F061E082E090E00C940164FC
:10E34000089520918112211109C0FC018381882345
:10E3500029F061E081E090E00C94016408958091DF
:10E360008112811105C061E086E090E00C940164A7
:10E37000089580918112811105C060E08BE090E0EA
:10E380000C940164089580918112811105C061E0AF
:10E3900087E090E00C9401640895809181128111CE
:10E3A00005C061E085E090E00C94016408958091DF
:10E3B0008112811105C061E08AE090E00C94016453
:10E3C0000895CF93DF93FC0125812223A1F1EC0175
:10E3D0008091811281112EC060916A1270916B122E
:10E3E00080917A1290917B120E94A4541092701224
:10E3F0008091811281110CC0609171127091721222
:10E4000080917A1290917B120E94A45410927712FC
:10E410008091811281110CC06091781270917912F3
:10E4200080917A1290917B120E94A45410928012D3
:10E430001092EF121D82DF91CF910895CF93DF9359
:10E44000FC01258121111EC0EC01809181128111F6
:10E4500017C08091EF12811113C02EE435E648EB0E
:10E460005BE060E070E080917A1290917B120E94F4
:10E47000F35490936B1280936A1281E08093EF12B1
:10E4800081E08D83DF91CF910895862F9091811245
:10E49000911102C00C94E1630895CF93C1E0809183
:10E4A0008112811103C08C2F0E94E163CF5FC730BE
:10E4B000B1F7CF91089580918112882329F06CEDF6
:10E4C00075E081E00C94145684E090E00C94A26313
:10E4D00080918112882329F068EE73E081E00C942A
:10E4E000145660E084E090E00C9401648091811205
:10E4F00081111BC08091F3128823B9F068EE73E09C
:10E5000081E00E9414561092F31225E734E748E99F
:10E510005AE360E070E080917A1290917B120E9441
:10E52000F3549093F2128093F11208956CED75E01C
:10E5300080E00C94145624EF31E0DB010E94BBC054
:10E540002FEF30E040E050E00E9491BECA01B901D7
:10E5500064527A4F8F4F9F4F80E00C9414568091F5
:10E560008112882331F060ED77E081E00E9414563B
:10E57000DFC161E083E090E00C940164209181129E
:10E58000211108C02091F012222321F00296E3D13C
:10E590001092F012089520918112222389F06FE6E3
:10E5A00076E080E00E9414562CE734E742E350E026
:10E5B00060E070E080917A1290917B120C94F35499
:10E5C0002091F012211105C00296C5D181E08093FF
:10E5D000F012089580E00E943B5681E00E943B5675
:10E5E00080918112811103C082E00E943B566CED44
:10E5F00075E080E00E9414566CED75E081E00E94A9
:10E6000014568091811281110CC08EEB90EAA1E02A
:10E61000BB27ABBFFC016791769182E00E94145644
:10E620004DC10895FC0184859585978386838685F1
:10E630009785918780878089918993878287808D4C
:10E64000918D938B828B828D938D958B848B848D12
:10E65000958D978B868B0895FC018089918993878E
:10E66000828782899389958784878489958997870A
:10E670008687089526E00C94AA5F8091FD12909100
:10E68000FE1291609093FE128093FD120895809186
:10E69000FD129091FE1280689093FE128093FD12FD
:10E6A00008958091FD129091FE1280619093FE1268
:10E6B0008093FD120895FC018281882371F083818B
:10E6C000882359F013828091FD129091FE1224E06C
:10E6D00082279093FE128093FD120895FC0182819F
:10E6E000882371F0838181110BC081E08383809145
:10E6F000FD129091FE1284609093FE128093FD12A1
:10E700000895FC018481882371F08581882359F064
:10E7100015828091FD129091FE1228E0822790933D
:10E72000FE128093FD120895FC018481882371F00C
:10E73000858181110BC081E085838091FD129091CC
:10E74000FE1288609093FE128093FD1208958091CE
:10E75000FD129091FE1220E282279093FE12809388
:10E76000FD1208958091FD129091FE1280629093A7
:10E77000FE128093FD120895DC01ED91FC9106805C
:10E78000F781E02D60E070E0199477FF03C0719588
:10E79000619571096F3F710519F014F06FEF70E02A
:10E7A0008091FD129091FE128C7B91709093FE12DD
:10E7B0008093FD128091FD129091FE126F307105D1
:10E7C00014F480641FC06733710514F481641AC0A7
:10E7D0006F3571051CF48164906114C06738710550
:10E7E0001CF4816490630EC06F3A71051CF481645F
:10E7F000906408C0673D71051CF48164906502C097
:10E80000816490669093FE128093FD12089580E0DB
:10E8100094E09093FE128093FD1208958091FD1272
:10E820009091FE1292609093FE128093FD120895D3
:10E8300008950895089508950895089508950895F0
:10E840000895089580E0089508950895089508951D
:10E8500008950895089508950895089508950895D0
:10E8600008950895089508950895089508950895C0
:10E8700080E00895089508950895FC016483089543
:10E88000FC0162830895FC011382148215821682B2
:10E890001782108611860895089508950895FC0141
:10E8A00083810895FC0165830895FC0164830895C4
:10E8B000FC0160870895FC016683089580918112B0
:10E8C000811112C08EEB90EAA1E0BB27ABBFFC0127
:10E8D0006791769182E00E94145681E080936212E3
:10E8E0001092661210926312089581E08093F312E1
:10E8F0006CED75E00C9414566CED75E080E00C94B2
:10E900001456FC01128213821482158261E086E1A2
:10E910000E94666061E086E10E943760E2E7F0E015
:10E920008081816080831092FE121092FD12089502
:10E930001092F31225E734E744EF51E060E070E015
:10E9400080917A1290917B120E94F3549093F2126C
:10E950008093F11208958091811281110AC08091F3
:10E96000F312882331F060ED77E081E00E941456C5
:10E97000DFCF08950F931F93CF93DF93EC01709334
:10E980007B1260937A124093811281E090E00E94A2
:10E99000C1C08C010E94AE57109300130093FF1268
:10E9A00091E09093F312909362121092F2121092EF
:10E9B000F112109265121092641210926612109267
:10E9C00063121092F01224EF31E030936D12209315
:10E9D0006C1228EB3BE030936F1220936E1220E212
:10E9E00033E030937412209373122CEA3DE030939D
:10E9F00076122093751228E037E030937D12209331
:10EA00007C1224E931E130937F1220937E12109220
:10EA1000691210926812109267121092701210927E
:10EA20007712109280121092EF1210926B121092C5
:10EA30006A12109272121092711210927912109240
:10EA40007812988399839A83DF91CF911F910F91C8
:10EA500008951F920F920FB60F9211240BB60F92CA
:10EA60000F931F932F933F934F935F936F937F93D6
:10EA70008F939F93AF93BF93EF93FF938091FC127B
:10EA80008F5F8093FC129091FB12891708F42FC1BD
:10EA90001092FC128091FA1290E08730910508F0F4
:10EAA00026C1FC018827EB55FE4F8F4F0C94ADC05B
:10EAB00060E086E10E94376080E48093FB1281E091
:10EAC00048C061E086E10E94376088E08093FB12D5
:10EAD00036C060E086E10E9437608091F812909124
:10EAE000F91297FF05C088E18093FB1284E031C0E2
:10EAF00088E08093FB1283E02CC061E086E10E94F5
:10EB0000376088E18093FB128091F7128F5F8093CA
:10EB1000F712803150F01092F71285E01AC061E0D0
:10EB200086E10E94376088E0EDCF8091F8129091E5
:10EB3000F912880F991F9093F9128093F81282E0CE
:10EB400008C060E086E10E94376088E08093FB1295
:10EB500086E08093FA12CBC061E086E10E943760C4
:10EB600080EC8093FB128091FD129091FE129093A5
:10EB7000F9128093F8128091FD129091FE1291FF8C
:10EB80001CC08091F612882369F08091FD1290914B
:10EB9000FE1222E092279093FE128093FD121092B3
:10EBA000F6120BC081E08093F6128093F5128093E9
:10EBB000F41287E89AE00E948B418091F412882336
:10EBC000D1F08091F5128823B1F00E9488930091D2
:10EBD000870A1091880A2091890A30918A0ADC01FB
:10EBE000CB01801B910BA20BB30B8D369042A1057C
:10EBF000B10508F070C08091FD129091FE1292FF55
:10EC000012C08091F612882339F01092FE121092F1
:10EC1000FD121092F61207C081E08093F612109256
:10EC2000F5121092F4128091FD129091FE1284FF61
:10EC300014C08091F612882369F08091FD129091A2
:10EC4000FE1220E182279093FE128093FD12109213
:10EC5000F61203C081E08093F6128091FD1290912C
:10EC6000FE1287FF13C08091F612882361F0809115
:10EC7000FD129091FE1280589093FE128093FD1227
:10EC80001092F61203C081E08093F6128091FD127B
:10EC90009091FE1290FF14C08091F612882369F0C3
:10ECA0008091FD129091FE1221E092279093FE1226
:10ECB0008093FD121092F61203C081E08093F61249
:10ECC0008091FD129091FE129093F9128093F812A8
:10ECD0001092FA120CC01092F4128091FD129091D1
:10ECE000FE1280649093FE128093FD1284CFFF91F8
:10ECF000EF91BF91AF919F918F917F916F915F91B4
:10ED00004F913F912F911F910F910F900BBE0F903C
:10ED10000FBE0F901F901895FF920F931F93CF93E4
:10ED2000DF938C01C62FF42ED22F6AED70E0DC0148
:10ED30001A968D919C911B97DAD9F801828593855B
:10ED4000DC01ED91FC910190F081E02D6C2F199583
:10ED5000F80182859385DC01ED91FC910190F081B1
:10ED6000E02D6F2D1995F80182859385DC01ED91D9
:10ED7000FC910190F081E02D6D2F1995EC2FF0E0C2
:10ED8000BF0166527F4F6F0D711D6D0F711D6F7743
:10ED90007727F80182859385DF91CF911F910F919D
:10EDA000FF90A5C920E040E0B7CF65E4FBCF68E461
:10EDB000F9CFCF93DF93FC012381222321F0EC01D3
:10EDC00061E4F0DF1B82DF91CF910895CF93DF9351
:10EDD000FC012381211105C0EC0160E4E3DF81E047
:10EDE0008B83DF91CF91089563E5DCCFFC01258112
:10EDF000222311F060E5D6CF0895FC01248122235F
:10EE000011F06CE3CFCF0895FC012085222331F06F
:10EE10002185222319F011866BE3C4CF0895FC01EC
:10EE20002085222339F02185211104C021E021878A
:10EE30006AE3B8CF0895FC012681222331F02781AF
:10EE4000222319F0178269E3ADCF0895FC012681D2
:10EE5000222339F02781211104C021E0278368E3B0
:10EE6000A1CF089567E39ECF6AE49CCF69E49ACF6F
:10EE700066E398CF65E396CF6EE494CF64E392CFD8
:10EE800063E390CF242F462F6CE446CF462F20E03B
:10EE900067E442CF462F20E066E43ECF262F64E4AD
:10EEA0003BCFCF92DF92FF920F931F93CF93DF93CD
:10EEB0008C01F62E443F81E0580738F0413187E25B
:10EEC000580728F040E157E202C044EF51E0243FE8
:10EED00081E0380738F0E9012131374228F0C0E1FC
:10EEE000D7E202C0C4EFD1E0CA01845F914022E3BF
:10EEF000C22ED12CB6010E9486C0462F2F2D62E46F
:10EF0000C8010ADFCE01845F9140B6010E9486C02D
:10EF1000462F2F2D63E4C801DF91CF911F910F91F0
:10EF2000FF90DF90CF90F8CE242F462F62E5F4CEED
:10EF3000242F462F61E5F0CE262F40E06FE3ECCE84
:10EF4000262F40E06EE3E8CE262F40E06DE3E4CECE
:10EF5000462F20E06FE4E0CE60E089E30E94376056
:10EF600060E08AE30E94376060E085E30E943760DA
:10EF700060E085E00E94376060E084E00E943760D6
:10EF800060E087E00E94376059980895CF93C09160
:10EF900011026C2F89E30E94376081E0C8276C2F33
:10EFA0008AE30E943760C0931102CF910895CF93F6
:10EFB000DF93C09110026C2F89E30E943760D1E08B
:10EFC000DC276D2F8AE30E9437606C2F85E30E9457
:10EFD00037606D2F85E00E9437606D2F84E00E94BE
:10EFE00037606C2F87E00E943760CC2311F059986E
:10EFF00001C0599A9091100281E0892780931002F4
:10F00000DF91CF910895CF93DF93809116138111F3
:10F010000DC0109215131092141381E090E090939C
:10F020001313809312138093161336C08091141318
:10F0300090911513863191057CF18F38910534F448
:10F040008091121390911313019609C08D3521E020
:10F05000920754F480911213909113130296909397
:10F0600013138093121318C0863222E0920734F4EF
:10F0700080911213909113130496F1CF883E934020
:10F080003CF480911213909113138A5B9F4FE7CF4A
:10F0900010921313109212138ADFC0911413D0919F
:10F0A0001513C93E83E0D80754F01092161354DFAD
:10F0B0002BE738E748EE53E060E070E007C023E05C
:10F0C00038E7AE010D2E000C660B770B8EE89BE047
:10F0D0000E94F35490931113809310138091121394
:10F0E000909113138C0F9D1F9093151380931413FD
:10F0F000DF91CF910895CF93DF938091D606882337
:10F1000019F0DF91CF917FCFC0911013D0911113DF
:10F11000BE018EE89BE00E948C54882329F0BE013A
:10F120008EE89BE00E94A454DF91CF9115CFCF933E
:10F13000C0910D136C2F70E088E00E94A26089E1FD
:10F1400080930C1390910F02992311F0CD5F01C0B1
:10F15000C350C0930D1380910D13873970F099231C
:10F1600021F08FEF80930D1308C08D3D30F086E9BC
:10F1700080930D1388E780930C1380910D138F3FBC
:10F1800019F410920F0205C08A3118F481E08093BF
:10F190000F0240910C1350E060E070E027E938E77F
:10F1A0008EE89BE00E94F35490934813809347139A
:10F1B000CF910895CF92DF92EF92FF92CF93DF939A
:10F1C000EC019C01AFEFB0E00E94DFBECC24CA94FA
:10F1D00023E0D22EE12CF12CA70196010E9491BED2
:10F1E000B90188E00E94A2609E01A4E6B0E00E94FE
:10F1F000DFBEA70196010E9491BE8091E10F8213AC
:10F200002093E10FDF91CF91FF90EF90DF90CF90AF
:10F210000895CF93DF93C0914713D0914813BE0157
:10F220008EE89BE00E948C54882329F0BE018EE872
:10F230009BE00E94A45460E088E00E9437608091C7
:10F24000D3068823D1F080914913882319F06DE00B
:10F2500077E10DC080914613882319F064EF76E1C1
:10F2600006C080919012811108C065EE76E1809110
:10F27000D1069091D2060E94305E109249131092EE
:10F280004613DF91CF91089561E088E00E943760D6
:10F290008091D306882361F080914913811108C0C1
:10F2A00067ED76E18091D1069091D2060C94305EA4
:10F2B000089580914913811110C0ABDF81E08093E4
:10F2C00049138091D306882341F06CE377E1809164
:10F2D000D1069091D2060E94305E80910B13882354
:10F2E00029F060E088E00E94376001C0CDDF909196
:10F2F0000B1381E0892780930B13882329F0409119
:10F30000DD0F5091DE0F04C04091DF0F5091E00FF0
:10F3100060E070E029E539E78EE89BE00E94F35455
:10F3200090934813809347130895CF9380910913C6
:10F3300081110FC081E0809309138091D306882347
:10F3400041F065EA76E18091D1069091D2060E9463
:10F35000305EC09108136C2F85E00E9437604091A9
:10F36000E60F50E060E070E025E939E78EE89BE0C9
:10F370000E94F354909307138093061381E06C2F3F
:10F38000682760930813CF9108958091070180FF4B
:10F390001BC08091D306882351F08CE59BE00E942E
:10F3A0001A87811108C08091680B811104C08CE517
:10F3B0009BE00C9407876CE176E18091D1069091F7
:10F3C000D2060E94305EF3CF08958091070180FF3E
:10F3D00017C08091D306882331F08CE59BE00E9412
:10F3E0001A87882321F08CE59BE00C942E8766E039
:10F3F00076E18091D1069091D2060E94305EF3CFE3
:10F400000895CF93DF93C0910E13D0910F13BE01D7
:10F410008EE89BE00E948C54882361F0BE018EE848
:10F420009BE00E94A45410920F1310920E13DF91D0
:10F43000CF9192CDDF91CF91089560910E1370918D
:10F440000F138EE89BE00E948C5481112EC060E067
:10F4500089E30E94376060E08AE30E94376060E0E1
:10F4600085E30E94376060E085E00E94376060E0DD
:10F4700084E00E94376060E087E00E94376059981E
:10F480008091E30F882319F027ED37E702C026ECBF
:10F4900037E742E350E060E070E08EE89BE00E94D6
:10F4A000FB5490930F1380930E13089560E08AE34A
:10F4B0000C94376061E08AE30C9437600F931F93DC
:10F4C000CF93DF938C01C1E0D0E00C171D079CF0B7
:10F4D000F1DF64E670E080E090E00E945093E6DFA8
:10F4E000C017D10734F46AE570E080E090E00E9434
:10F4F00050932196EACFDF91CF911F910F910895FC
:10F5000083E090E0DBCF82E090E0D8CF81E090E034
:10F51000D5CF60E089E30C94376061E089E30C9417
:10F5200037600F931F93CF93DF938C01C1E0D0E03E
:10F530000C171D079CF0F1DF64E670E080E090E0BE
:10F540000E945093E6DFC017D10734F46AE570E0FB
:10F5500080E090E00E9450932196EACFDF91CF9116
:10F560001F910F91089583E090E0DBCF82E090E05F
:10F57000D8CF81E090E0D5CF6091E10F70E088E0D6
:10F580000E94A2608091D306882341F066E277E171
:10F590008091D1069091D2060C94305E089510921D
:10F5A0000A138091BF06811104C060E084E00E94CC
:10F5B00037608091D306882341F064EC76E1809136
:10F5C000D1069091D2060C94305E089581E080932C
:10F5D0000A138091BF06811106C06091011370E08B
:10F5E00084E00E94A2608091D306882341F062EB00
:10F5F00076E18091D1069091D2060C94305E089508
:10F600001092BF0680910A13811104C060E084E06B
:10F610000C9437606091011370E084E00C94A26058
:10F62000CF93DF9360E085E00E94376080910913FB
:10F6300081110BC08091CD069091CE06DC01ED9139
:10F64000FC9104ACF5ADE02D1995C0910613D09155
:10F650000713BE018EE89BE00E948C54882329F09A
:10F66000BE018EE89BE00E94A4548091D3068823BB
:10F6700079F0209109138091D1069091D20622232E
:10F6800019F069E976E102C06DE876E10E94305E2A
:10F6900010920913DF91CF91089561E085E00E94F7
:10F6A00037608091CD069091CE06DC01ED91FC9102
:10F6B00004ACF5ADE02D19958091D306882341F077
:10F6C00062E876E18091D1069091D2060C94305E8A
:10F6D000089560E085E30E9437608091CD069091A7
:10F6E000CE06DC01ED91FC9100ACF1ADE02D199559
:10F6F0008091D306882341F066E776E18091D106B8
:10F700009091D2060C94305E089561E085E30E94EA
:10F7100037608091CD069091CE06DC01ED91FC9191
:10F7200000ACF1ADE02D19958091D306882341F00E
:10F730006BE676E18091D1069091D2060C94305E12
:10F7400008958F929F92AF92BF92CF92DF92EF92E5
:10F75000FF9285E40E946961BC01990F880B990BA7
:10F760000E944EBD20E030E040E85AE30E94ADBD6B
:10F7700020E030E040EA50E40E94ADBD6B017C0126
:10F7800080910E02882351F0C0920213D09203138D
:10F79000E0920413F092051310920E0226E636E66C
:10F7A00046E65FE3609102137091031380910413A6
:10F7B000909105130E94ADBD4B015C0120ED3CEC26
:10F7C0004CEC5DE3C701B6010E94ADBD9B01AC01ED
:10F7D000C501B4010E94EFBE60930213709303133E
:10F7E00080930413909305132DE33CE248E450E426
:10F7F0000E94ADBD2AE939E949E95EE30E94EFBE06
:10F80000FF90EF90DF90CF90BF90AF909F908F9040
:10F81000089580910D02882351F093DF20E030E0BD
:10F8200040E050E40E9448BD87FF39C0089589DF59
:10F8300020E030E04AE754E40E94ADBD0E94C0BF22
:10F840002091D60F3091D70F4091D60662177307DB
:10F8500010F4442351F1442309F445C072DF20E041
:10F8600030E04AE754E40E94ADBD0E94C0BF209141
:10F87000D60F3091D70F62177307A8F11092D606F2
:10F8800081E08093D5068091D306882361F163E3FC
:10F8900076E18091D1069091D2060C94305E109260
:10F8A0000D0281E08093D506089581E08093D6060D
:10F8B0001092D5068091D306882391F062E576E117
:10F8C0008091D1069091D2060E94BF5C0E947F87F2
:10F8D0006FE476E18091D1069091D2060E94305E6D
:10F8E0000E94843F08CC0895CF93DF938091070155
:10F8F00080FD2AC0C0916806D091690680916C068F
:10F90000882371F08EE30E946961813092402CF06F
:10F9100010926906109268060AC081E090E003C068
:10F920008EE30E94696190936906809368068091D6
:10F930006806909169068C179D0719F410926A0663
:10F9400003C081E080936A06DF91CF910895809192
:10F95000D4068093D306089580913F13882359F0ED
:10F9600080913D1390913E13DC01ED91FC91048058
:10F97000F581E02D1994089580913F13882369F053
:10F9800080913D1390913E13DC01ED91FC9101902B
:10F99000F081E02D6FEF73E01994089580913F138B
:10F9A000882389F080914113882321F080E090E042
:10F9B000D3DF03C080E090E0DFDF9091411381E06E
:10F9C000892780934113089520913F13222369F0E2
:10F9D000A0913D13B0913E13ED91FC9111970190D0
:10F9E000F081E02DBC01CD011994089580913C1364
:10F9F000882359F080913A1390913B13DC01ED91EB
:10FA0000FC910480F581E02D1994089580913C13B8
:10FA1000882369F080913A1390913B13DC01ED91BA
:10FA2000FC910190F081E02D6FEF73E0199408953F
:10FA300080913C13882389F080914013882321F022
:10FA400080E090E0D3DF03C080E090E0DFDF9091C2
:10FA5000401381E0892780934013089520913C133F
:10FA6000222369F0A0913A13B0913B13ED91FC91E0
:10FA700011970190F081E02DBC01CD0119940895FA
:10FA800020913913222369F0A0913713B0913813D4
:10FA9000ED91FC9111970190F081E02DBC01CD0119
:10FAA0001994089520913613222369F0A0913413FC
:10FAB000B0913513ED91FC9111970190F081E02DFB
:10FAC000BC01CD011994089520913313222369F0CC
:10FAD000A0913113B0913213ED91FC9111970190E7
:10FAE000F081E02DBC01CD011994089520913013CF
:10FAF000222369F0A0912E13B0912F13ED91FC9168
:10FB000011970190F081E02DBC01CD011994089569
:10FB100020912D13222369F0A0912B13B0912C1367
:10FB2000ED91FC9111970190F081E02DBC01CD0188
:10FB30001994089520912A13222369F0A091281383
:10FB4000B0912913ED91FC9111970190F081E02D76
:10FB5000BC01CD011994089520912713222369F047
:10FB6000A0912513B0912613ED91FC91119701906E
:10FB7000F081E02DBC01CD01199408958091CD064E
:10FB80009091CE06DC01ED91FC91EE59FF4F019072
:10FB9000F081E02D19948091CD069091CE06DC0184
:10FBA000ED91FC91E05AFF4F0190F081E02D199406
:10FBB0008091CD069091CE06DC01ED91FC91E25A48
:10FBC000FF4F0190F081E02D19948091D406882395
:10FBD00061F00E94884C029741F064EF77E18091D8
:10FBE000D1069091D2060C94305E0895CF93DF93A6
:10FBF000209144133091451328173907D1F0909381
:10FC00004513809344132091D306222391F0EC01F5
:10FC100065EC77E18091D1069091D2060E94BF5C9D
:10FC2000BE018091D1069091D206DF91CF910C94C4
:10FC30004D42DF91CF910895CF93DF9320914213EE
:10FC40003091431328173907D1F0909343138093D1
:10FC500042132091D306222391F0EC016BEA77E165
:10FC60008091D1069091D2060E94BF5CBE01809126
:10FC7000D1069091D206DF91CF910C944D42DF9145
:10FC8000CF91089520913913222339F0BC0180913E
:10FC90002313909124130C947E70089520913613B1
:10FCA000222339F0BC0180912113909122130C94EE
:10FCB0007E70089520913313222339F0BC01809186
:10FCC0001F13909120130C947E700895209130138F
:10FCD000222339F0BC0180911D1390911E130C94C6
:10FCE0007E70089520912D13222339F0BC0180915C
:10FCF0001B1390911C130C947E70089520912A136D
:10FD0000222339F0BC018091191390911A130C949D
:10FD10007E70089520912713222339F0BC01809131
:10FD20001713909118130C947E700895CF92DF9260
:10FD3000EF92FF9220910002213019F42091620F7E
:10FD400004C02230C9F52091680F2223A9F19C013B
:10FD5000211584E0380710F02FEF33E0ADE0B0E07C
:10FD60000E94DFBE2FEF33E040E050E00E9491BEE2
:10FD700069017A018FEFC81AD80AE80AF80A809157
:10FD8000BC138C15C9F0C092BC138091D306882394
:10FD900099F064E977E18091D1069091D2060E94B2
:10FDA000BF5C6C2D8091D1069091D206FF90EF90B0
:10FDB000DF90CF900C94F344FF90EF90DF90CF90C2
:10FDC0000895CF92DF92EF92FF92209100022130AE
:10FDD00019F420915F0F04C02230C9F52091650FFE
:10FDE0002223A9F19C01211584E0380710F02FEFA0
:10FDF00033E0ADE0B0E00E94DFBE2FEF33E040E043
:10FE000050E00E9491BE69017A018FEFC81AD80AAA
:10FE1000E80AF80A8091BA138C15C9F0C092BA1397
:10FE20008091D306882399F06DE777E18091D10620
:10FE30009091D2060E94BF5C6C2D8091D10690916A
:10FE4000D206FF90EF90DF90CF900C94F344FF9098
:10FE5000EF90DF90CF90089581E08093CA060E94D2
:10FE6000B93D8091D306882341F063E677E1809124
:10FE7000D1069091D2060C94305E089583E0809371
:10FE8000CA060E94CE3C8091D306882341F060E7E9
:10FE900077E18091D1069091D2060C94305E08955E
:10FEA00082E08093CA060E94CE3C8091D3068823CC
:10FEB00041F066E577E18091D1069091D2060C94ED
:10FEC000305E089580914E0F811111C080914706D8
:10FED00090914806FC0121A132A1121613061CF4D0
:10FEE00060E070E002C06FEF70E00C942854089559
:10FEF00080914E0F811108C060E070E0809147064C
:10FF0000909148060C942854089580914E0F8111C9
:10FF100008C06FEF70E080914706909148060C94FE
:10FF2000285408950C94F4988091010281110C9446
:10FF3000D8980C94F4980C94D89884E60C94C23F0A
:10FF400089E10C94C23F682F8091D1069091D2062E
:10FF50000E940A4562EF77E18091D1069091D20626
:10FF60000C94BF5C2091D1063091D206882319F001
:10FF700066EB77E002C06AEB77E0C9010C94BF5CE6
:10FF8000F1DF8091D1069091D2060C941D5E2091F4
:10FF9000D1063091D206882319F067EE77E102C0CE
:10FFA0006CEE77E1C9010E94BF5C8091D10690910F
:10FFB000D2060C941D5E8091D1069091D2060C94CD
:10FFC0001D5E65EE77E18091D1069091D2060C948A
:10FFD000BF5C61EE77E18091D1069091D2060C94DE
:10FFE000BF5CCF93CDE26FED77E18091D106909128
:10FFF000D2060E94BF5CC150B1F78091D1069091AA
:020000021000EC
:10000000D2060E941D5E8091D1069091D206DC013D
:10001000ED91FC910680F781E02DCF911994CF935B
:10002000DF93EC011F861E86198A188A1B8A1A8A9A
:100030000E948B41198618861C86DF91CF91089506
:10004000CF93DF93CDB7DEB7A0970FB6F894DEBF9E
:100050000FBECDBF80310CF080E028EC38E13A8350
:10006000298321EC38E13C832B8323EB38E13E8369
:100070002D8327EA38E138872F832DE938E13A8745
:10008000298723E938E13C872B872FE838E13E8731
:100090002D8728E838E1388B2F872DE738E13A8B18
:1000A000298B20E738E13C8B2B8B25E638E13E8B12
:1000B0002D8B29E538E1388F2F8B27E438E13A8FF3
:1000C000298F26E338E13C8F2B8F21E338E13E8FE7
:1000D0002D8F24E238E138A32F8FE82FEE0FFF0B8E
:1000E000EC0FFD1F81819281A0960FB6F894DEBFC0
:1000F0000FBECDBFDF91CF910895AF92BF92CF9247
:10010000DF92EF92FF920F931F93CF93DF9383E5DC
:1001100093E17EE1D72ED80ECC24C39402E010E008
:10012000C3E0D0E0E2E0BE2EEE24E394F12C809117
:10013000EA119091EB11DC01ED91FC910084F185C5
:10014000E02D1995892B09F4ADC0A0903001809164
:10015000EA119091EB11DC01ED91FC910284F385A1
:10016000E02D199596B3B39A2091840030918500C3
:10017000285A344E30938D0020938C002A2D2C71F8
:1001800019F01092D4114BC093FB992790F9E0918C
:10019000D411E11116C0992351F2803241F6C09278
:1001A000D4118093531380910C1290910D12892BCE
:1001B00009F0BDCFF0920D12E0920C121092D61100
:1001C000B6CF9111DECFE13041F4803409F0AFCFEA
:1001D000B092D41180935413E6CF91E09E0F909388
:1001E000D411F0E0ED5AFC4E8083903209F09FCF9D
:1001F0001092D411E3E5F3E12FEF3FEF8191281B3B
:100200003109DE12FBCF409171138091721390E09F
:10021000982F8827840F911D2817390729F0D0932C
:100220000D12C0930C1283CF80910C1290910D127D
:10023000019739F48091D6118F5F8093D611843065
:1002400020F010930D1200930C128091D5118F5F46
:100250008093D5119091D311981708F5C0920E1282
:1002600020E030E0F901ED5AFC4E4281838190E0BC
:10027000982F8827840F911DAC014F5E52404B3D53
:10028000554028F4F901E451FE4E918380832E5F9E
:100290003F4F2C31310531F71092D51148CF1092D4
:1002A0000E1245CFDF91CF911F910F91FF90EF90EC
:1002B000DF90CF90BF90AF900895EF92FF920F9391
:1002C0001F93CF93DF9310920E0E82E080930F0E58
:1002D00068EE73E07093110E6093100E40ED57E0DE
:1002E0005093130E4093120E2CED35E03093150E03
:1002F0002093140E8FE08093160E1092170E94E048
:100300009093180E70931A0E6093190E50931C0E52
:1003100040931B0E30931E0E20931D0E80931F0ED4
:100320001092200E93E09093210E7093230E609311
:10033000220E5093250E4093240E3093270E2093C7
:10034000260E8093280E1092290E91E090932A0E8B
:1003500070932C0E60932B0E50932E0E40932D0E07
:100360003093300E20932F0E8093310E1092320E68
:10037000E3E3FEE0ACE3BEE080E008EE13E060ED16
:1003800077E04CED55E031E022E095E0980F908366
:10039000128301837483638356834583ED0122971F
:1003A00091E03883219628831C928F5F3A961A96A3
:1003B0008C3059F71092AB0E9093AC0E1092AD0E9C
:1003C0009093AE0E8AE892E09093B00E8093AF0EB9
:1003D0009093B20E8093B10E80E090E09C01225F7A
:1003E000314FF901EB55FF4F118210823296108286
:1003F00003968837910591F784E290E09093B40ECC
:100400008093B30E81E08093B50E2CE030E0309302
:10041000B70E2093B60E94E09093B80E21E230E030
:100420003093BA0E2093B90E27E02093BB0E29E03B
:1004300030E03093BD0E2093BC0E20E12093BE0E21
:10044000FAE0F0932B0F2BE020932C0F20932D0F2D
:1004500048EE53E050932F0F40932E0F20ED37E0DE
:100460003093310F2093300F1092320FE4E6E09377
:10047000330FE093340F5093360F4093350F309382
:10048000380F2093370F1092390F50933B0F409342
:100490003A0F30933D0F20933C0F10923E0F109275
:1004A0003F0F8093400F1092420F1092410F8093A4
:1004B000430F8093440F68EC70E07093460F609395
:1004C000450F60E273E07093480F6093470F5093BD
:1004D0004A0F4093490F30934C0F20934B0F1092CB
:1004E0004D0F80934E0F69E570E07093500F60934D
:1004F0004F0F60E870E07093520F6093510F6FEFF1
:1005000070E07093540F6093530F7093560F609385
:10051000550F1092570F1092580F70935A0F609307
:10052000590F70935C0F60935B0F70935E0F609335
:100530005D0F80935F0F9093600F1092610F809317
:10054000620F9093630F1092640F1092650F809367
:10055000660F1092670F1092680F8093690F1092C8
:100560006A0F98E290936B0F50936D0F40936C0F4E
:1005700050936F0F40936E0F3093710F2093700F55
:100580008093720F92E39093730F62E06093740F05
:100590008093750FE093760F66E46093770F9093E6
:1005A000780F1092790F10927A0F10927B0F1092A1
:1005B0007C0F10927D0F10927E0F6AEF70E07093A7
:1005C000800F60937F0F1092810F1092820FE09343
:1005D000830F61E46093840F1092850F9093860FD0
:1005E0001092870F9093880F6EE571E070938A0FD9
:1005F0006093890F10928B0FACEDB5E0B0938D0F27
:10060000A0938C0F00EA1FE010938F0F00938E0FC2
:100610003093910F2093900FC8E8D3E1D093930FBC
:10062000C093920F68EBE62E6BE0F62EF092950FDA
:10063000E092940F60E47FE17093970F6093960FC0
:100640001092980F1092990F10929A0FE9E1E0938F
:100650009B0F80939C0F80939D0F80939E0F5093D0
:10066000A00F40939F0F3093A20F2093A10FF09201
:10067000A40FE092A30F1093A60F0093A50FD093A1
:10068000A80FC093A70F20E737E13093AA0F20935C
:10069000A90F1092AB0F1092AC0F1092AD0F909368
:1006A000AE0F9093AF0F9093B00F1092B10F1092C6
:1006B000B20F1092B30F8093B40F1092C40F109228
:1006C000B50F99E09093B60F1092B70F1092B80F34
:1006D0001092B90F1092BA0FB093BC0FA093BB0F3A
:1006E0007093BE0F6093BD0F8093BF0FF093C00F48
:1006F0001092C10F21E030E03093C30F2093C20F5E
:1007000040E052EC61E070E04093C50F5093C60F9B
:100710006093C70F7093C80F4093C90F5093CA0FCF
:100720006093CB0F7093CC0F40E056E960E070E02F
:100730004093CD0F5093CE0F6093CF0F7093D00F97
:100740004093D10F5093D20F6093D30F7093D40F77
:100750001092D50F20E039E13093D70F2093D60FB8
:100760001092D80F9EE19093D90F1092DA0F2EE1DC
:1007700030E03093DC0F2093DB0F3093DE0F2093BB
:10078000DD0F3093E00F2093DF0F9093E10F9093F4
:10079000E20F8093E30F8093E40F1092E50F9093A4
:1007A000E60F8093E70F9CE09093E80F8093E90FAA
:1007B0008CE49DE5A0E0B0E08093EA0F9093EB0F0E
:1007C000A093EC0FB093ED0F0EE01EE0C0E0D0E080
:1007D000CE010E9471BEF80161918F01861719F058
:1007E000CE010E9483BE2196C03EF1E0DF0781F773
:1007F000DF91CF911F910F91FF90EF9008954F924D
:100800005F926F927F928F929F92AF92BF92CF92A0
:10081000DF92EF92FF92CF93DF93EB01A091511300
:10082000B09152139D012F5F3F4F45E0429F200141
:10083000439F500C1124052C000C66087708812C6E
:10084000912C54012A34E1E03E07ECF441EF50EAE8
:1008500061E0772775016401C40CD51CE61CF71C08
:100860004C0D5D1D6E1D7F1D6BBFFA0147915691AA
:1008700065E0860E911CA11CB11CC417D50729F197
:100880002F5F3F4FDFCF25E0822E912CA12CB12C82
:1008900021E030E0A217B30708F44CC041EF50EA62
:1008A00061E07727480D591D6A1D7B1D6BBFFA015A
:1008B00047915691F5E08F0E911CA11CB11CC417F5
:1008C000D50719F02F5F3F4FE5CF41EF50EA61E0C8
:1008D0007727E5E0E29F6001E39FD00C11240D2C07
:1008E000000CEE08FF084E5F5F4F6F4F7F4F4C0DBF
:1008F0005D1D6E1D7F1D6BBFFA0147915691FC0176
:100900005383428341EF50EA61E077274C5F5F4FAA
:100910006F4F7F4FC40ED51EE61EF71EEBBEF601CD
:10092000C790FC01C4823093521320935113C90124
:10093000019606C0109252131092511380E090E07D
:10094000DF91CF91FF90EF90DF90CF90BF90AF906D
:100950009F908F907F906F905F904F9008950F932E
:100960001F9380914C1381111EC00E9488930091A7
:100970004D1310914E1320914F1330915013AB0132
:10098000BC01401B510B620B730B80914A13909179
:100990004B13A0E0B0E084179507A607B70718F43B
:1009A00081E080934C131F910F91089580914A1319
:1009B00090914B13892B89F080914C13882381F0FF
:1009C0000E94889360934D1370934E1380934F133E
:1009D0009093501310924C13089581E080934C1320
:1009E00008951F920F920FB60F9211242F938F9399
:1009F0009F93109295001092940080910B0B8F5F43
:100A000080930B0B9091B613891784F010920B0B07
:100A100020910D0B8091C1139091C213820F911DF3
:100A200027FD9A959093C2138093C11380910A0B6E
:100A30008F5F80930A0B9091C613891784F01092F0
:100A40000A0B20910C0B8091C4139091C513820F57
:100A5000911D27FD9A959093C5138093C4139F9180
:100A60008F912F910F900FBE0F901F90189580912E
:100A7000090B811104C08091080B882321F080911B
:100A80007100826003C0809171008D7F809371003E
:100A90000895CF93DF93EC01198618861F861E8672
:100AA000198A188A1B8A1A8A0E948B411EA61D86E3
:100AB000DF91CF910895FC018385882311F061E0D7
:100AC00001C060E082850C943760FC018385882337
:100AD00011F060E001C061E082850C9437600F93F3
:100AE0001F93CF93DF93CDB7DEB78C0198DAF8016F
:100AF000148A85E1FE013896D801559601900D9231
:100B00008A95E1F7F80185899689938B828B8D8D83
:100B10008B3008F08AE090E0F801918B808BC8015F
:100B2000D4DFC8010E948B4181E0F8018487DF9106
:100B3000CF911F910F910895CF92DF92EF92FF9284
:100B40000F931F93CF93DF93CDB7DEB765970FB6A3
:100B5000F894DEBF0FBECDBF8C01FC0185858823D4
:100B6000E1F082899389892B09F442C10E9488931C
:100B7000F801C080D180E280F380AB01BC014C1948
:100B80005D096E097F0982899389A0E0B0E084172E
:100B90009507A607B70718F12BC1F8018085918545
:100BA000892B09F48FC00E948893F801C480D580F6
:100BB000E680F780AB01BC014C195D096E097F0925
:100BC00080859185A0E0B0E084179507A607B70758
:100BD00008F078C0C8016FDFC80121DAB5C0F8019C
:100BE000868597850196978786876089718986179C
:100BF000970768F580E090E00E944CBD9B01AC0136
:100C00006BED7FE089E490E40E9453BFF80122A5D8
:100C100033A544A555A50E94EFBEF80162A773A7AE
:100C200084A795A70E94F0BF20E030E04FEF52E488
:100C30000E94ADBD20E030E04FEF52E40E94EFBED5
:100C40000E94BBBFF80182850E94A2606CC0F801BF
:100C50008585823019F4C8012EDF76C0F80186A59B
:100C6000882309F471C0C80114DF82E390E09A83FD
:100C7000898388E290E09C838B838EE690E09E835C
:100C80008D8384EF91E098878F831D8A84E08F9312
:100C90008DB79EB745970FB6F8949EBF0FBE8DBF18
:100CA000ADB7BEB7119685E1FE01319601900D9268
:100CB0008A95E1F7C80113DF0FB6F894DEBF0FBEC7
:100CC000CDBF96C0F80182899389892B09F490C021
:100CD0000E948893F801C080D180E280F380AB014C
:100CE000BC014C195D096E097F0982899389A0E0D6
:100CF000B0E084179507A607B70708F079C0F80198
:100D000086859785019697878687208931898217FE
:100D1000930708F04EC080FF27C0C801CCDEF80161
:100D20008489882321F1C80165960FB6F894DEBF47
:100D30000FBECDBFDF91CF911F910F91FF90EF902C
:100D4000DF90CF900C948B41C80165960FB6F89454
:100D5000DEBF0FBECDBFDF91CF911F910F91FF90EE
:100D6000EF90DF90CF9095CEC801AFDED8CF8685CB
:100D700097858B30910590F0C8019DDEC80165967E
:100D80000FB6F894DEBF0FBECDBFDF91CF911F919C
:100D90000F91FF90EF90DF90CF9041C9880F991F7E
:100DA000F801E80FF91F85899689F801938B828BEA
:100DB000BACFF80181A5882349F085899689938B5C
:100DC000828B17861686C80180DEADCFF80186A516
:100DD000882391F216A682E08587C80120D984E68F
:100DE00090E0F801918B808B87A590A9938B828BE3
:100DF00065960FB6F894DEBF0FBECDBFDF91CF91E1
:100E00001F910F91FF90EF90DF90CF900895CF93B7
:100E1000DF93EC018C85882321F0CE014CDECE01DE
:100E2000FED88D85882311F0CE0133DECE01DF910F
:100E3000CF9141CEFC018385882339F082850E94C1
:100E40000F6021E0892B41F006C082850E940F606F
:100E500021E0892B09F420E0822F0895CF93DF93BE
:100E6000EC018C85882321F0CE0125DECE01D7D878
:100E70008D85882311F0CE010CDECE01DF91CF915C
:100E800024CE1F93CF93DF931F92CDB7DEB710E030
:100E9000181729F0898395D81F5F8981F9CF0F90A2
:100EA000DF91CF911F910895CF93DF9360E088E0A9
:100EB0000E94376010924913C0914713D091481394
:100EC000BE018EE89BE00E948C54882329F0BE016D
:100ED0008EE89BE00E94A45481E0809346138091A9
:100EE000D306882341F06AE078E18091D1069091A1
:100EF000D2060E94305EDF91CF910C94977860917A
:100F0000D60F7091D70F80E090E00E944CBD20E09A
:100F100030E04AE754E40E9453BFAB01BC0121E03A
:100F20008091D1069091D2060C94405D0895089569
:100F3000089508950F931F93CF93DF93EC011F8AB9
:100F40001E8A8C01075E1F4F40E060E0C8010E94CE
:100F5000695840E064E0C8010E9469580E94889383
:100F60006C8F7D8F8E8F9F8FDF91CF911F910F910F
:100F700008950F931F93CF93DF93EC018091731328
:100F8000811112C00A8D1B8D6AEA70E0C8010E94AF
:100F90007770D801ED91FC910680F781E02DC801B2
:100FA000199581E0809373134AE06EE0CE01499673
:100FB0000E94695821E83FEF3B872A878FE790E03E
:100FC0009D878C871F861E86398B288B9B8B8A8BEF
:100FD0001D8A1C8ADF91CF911F910F9108950F9365
:100FE0001F93CF93DF93EC011F8A1E8A8C01075E4B
:100FF0001F4F40E060E0C8010E942C5840E064E0D0
:10100000C8010E942C580E9488936C8F7D8F8E8F10
:101010009F8FDF91CF911F910F9108950F931F9391
:10102000CF93DF93EC01E8A1F9A180819181A281A6
:10103000B3818E01075E1F4F81159649A105B10549
:1010400009F452C040E056E960E070E08CEB97E0B4
:101050000E943A7364E170E080E090E00E94509357
:10106000E8A1F9A180819181A281B38181152BE44E
:101070009207A105B105E9F068F4803629E09207EE
:10108000A105B105A1F080389542A105B105C1F4D3
:1010900042E012C0811521EE9207A105B10559F079
:1010A0008115924CA140B10559F445E005C041E0DD
:1010B00003C043E001C046E06FE0C8010E942C5825
:1010C0008CEB97E00E94D45AE8A1F9A140815181AC
:1010D000628173818CEB97E00E943A7364E170E067
:1010E00080E090E00E9450934AE06EE0C8010E94C8
:1010F0002C5841E067E1C8010E942C584AA168E1E0
:10110000C8010E942C584BA18FEF840F8E3108F03C
:101110004CE066E1C8010E942C5821E83FEF3B8774
:101120002A878FE790E09D878C871F861E86398BE4
:10113000288B9B8B8A8B1D8A1C8ADF91CF911F91F4
:101140000F9108950C947E70CF93DF93CDE8DAE091
:1011500081E090E09A8389831092FB0A0E942B938E
:101160006C837D838E839F83E49AEC9ADF91CF9189
:101170000895EF92FF920F931F93CF93DF93EC01AB
:101180006623E1F0262F653608F024E60A891B89DC
:10119000E888F988D801AE19BF0930E00E94BBC0C9
:1011A00028EC30E040E050E00E94BDBEE20EF31EAD
:1011B000FB86EA86021B130B1D870C87DF91CF91FC
:1011C0001F910F91FF90EF900895CF93DF93CDB7CC
:1011D000DEB7A2970FB6F894DEBF0FBECDBF803149
:1011E0000CF080E12FE839E13A83298327E839E1DF
:1011F0003C832B832FE739E13E832D8327E739E1B9
:1012000038872F832FE639E13A87298727E639E1A6
:101210003C872B872FE539E13E872D8727E539E18C
:10122000388B2F8729E439E13A8B298B27E339E181
:101230003C8B2B8B2AE139E13E8B2D8B25E039E16C
:10124000388F2F8B2BEF38E13A8F298F21EF38E140
:101250003C8F2B8F24EE38E13E8F2D8F28ED38E127
:1012600038A32F8F20ED38E13AA329A3E82FEE0F02
:10127000FF0BEC0FFD1F81819281A2960FB6F894AF
:10128000DEBF0FBECDBFDF91CF9108958F929F92A9
:10129000AF92BF92CF92DF92EF92FF920F931F9384
:1012A000DC0118968D919C9119971E96CD90DC903B
:1012B0001F976817790709F456C05896FC905897FD
:1012C0004C01092E000CAA08BB088B01072E000C4C
:1012D000220B330B861797073CF41696ED91FC9181
:1012E0001797FF2039F015C01496ED91FC911597D2
:1012F000FF2079F00D2C000CEE08FF08A9019801E1
:10130000281939094A095B091C966D917C911D9732
:101310000EC00D2C000CEE08FF08A9019801281939
:1013200039094A095B091A966D917C911B97CB018B
:10133000770FAA0BBB0BBC01CD016C197D098E097F
:101340009F090E9477C08F01FF0F220B330BA90169
:101350009801281939094A095B090E9491BEC20EF9
:10136000D31EE41EF51EC6011F910F91FF90EF9052
:10137000DF90CF90BF90AF909F908F900895CF93C4
:10138000DF93EC017F8B6E8B81DF9C018A819B81D7
:1013900088309105C1F437FF06C061E021388FEF36
:1013A00038074CF001C060E0A901203831052CF06D
:1013B0004FE750E002C041E85FEF57FF1FC0519573
:1013C000419551091BC00997E9F4922F832F2038CA
:1013D000310514F09FE780E0492F582F41388FEFF7
:1013E000580714F441E85FEF57FF03C0519541954A
:1013F0005109632F661F6627661F6C5FCE014996F1
:101400000E9469580E9488936C8F7D8F8E8F9F8F6A
:10141000DF91CF9108950F931F93CF93DF93EC014A
:101420000E9488930C8D1D8D2E8D3F8DDC01CB018C
:10143000801B910BA20BB30B853F9140A105B10519
:1014400040F06E897F89CE01DF91CF911F910F917E
:1014500096CFDF91CF911F910F910895CF93DF9396
:10146000EC017F8B6E8B12DF9C018A819B8188301F
:101470009105C1F437FF06C061E021388FEF3807CE
:101480004CF001C060E0A901203831052CF04FE795
:1014900050E002C041E85FEF57FF1FC051954195F2
:1014A00051091BC00997E9F4922F832F2038310589
:1014B00014F09FE780E0492F582F41388FEF5807ED
:1014C00014F441E85FEF57FF03C05195419551096E
:1014D000632F661F6627661F6C5FCE0149960E94C8
:1014E0002C580E9488936C8F7D8F8E8F9F8FDF91F9
:1014F000CF9108950F931F93CF93DF93EC010E9438
:1015000088930C8D1D8D2E8D3F8DDC01CB01801BB2
:10151000910BA20BB30B853F9140A105B10540F0A3
:101520006E897F89CE01DF91CF911F910F9196CF68
:10153000DF91CF911F910F910895CF93DF93EC012D
:1015400061E089E00E94666060E089E00E943760A7
:101550001092000A82E395E099838883DF91CF910E
:101560000895CF92DF92EF92FF928091010A83302B
:1015700009F061C08091020A8130D1F488EE93E0D5
:10158000A0E0B0E08093930990939409A09395090B
:10159000B093960980E797E1A0E0B0E080939709C7
:1015A00090939809A0939909B0939A0932E001C0E9
:1015B00030E0E091020AF0E0ED5FF54F2081A0E11C
:1015C000A30F48EE53E060E070E088EBC82E8BE09C
:1015D000D82EE12CF12C832F90E0FC01EE0FFF1FA1
:1015E000EE0FFF1FED56F64F27FF10C0C082D182CD
:1015F000E282F382880F991F880F991FFC01E95638
:10160000F64F40835183628373830FC040835183BD
:1016100062837383880F991F880F991FFC01E95615
:10162000F64FC082D182E282F3823E5F220F3A13EC
:10163000D2CF3093FC09FF90EF90DF90CF900895C8
:10164000CF93DF938091000A811153C01092FE095D
:101650001092FB09C1E0C093000AD091FF0961E03C
:1016600089E00E94666060E089E00E9437602D2F6B
:1016700030E040E050E060E47FE180E090E00E94F4
:1016800091BEC093B00089E08093B1002093B30075
:101690008BEA289F212D112426952093B400809158
:1016A0006F008B7F80936F008091B0008062809389
:1016B000B0002091840030918500E091FB0981E029
:1016C0008E0F8093FB0984E0E89FF0011124ED5612
:1016D000F64F80819181A281B381820F931F9093F5
:1016E0008B0080938A00B29A80916F00846080930F
:1016F0006F00DF91CF9108954F925F926F927F922A
:101700008F929F92AF92BF92CF92DF92EF92FF9211
:101710008AE18093FC092093FD0988E28093FF0908
:1017200081E08093020A8093030A8EE08093010A8D
:1017300080EC92E1A0E0B0E080939309909394094B
:10174000A0939509B093960980EB94E0A0E0B0E0F7
:101750008093970990939809A0939909B0939A0957
:10176000A4E1440F551F661F771FAA95D1F722E009
:1017700030E0B0EBCB2EB4E0DB2EE12CF12C80E698
:10178000482E89E0582E612C712C90E4892E9CE91A
:10179000992EA12CB12CC901880F991F880F991F70
:1017A000FC01ED56F64F77FF05C040825182628200
:1017B000738204C0C082D182E282F382C9010196A1
:1017C000880F991F880F991FFC01ED56F64F28319D
:1017D00029F0C082D182E282F38204C080829182A9
:1017E000A282B382440F551F661F771F2E5F3F4FA3
:1017F0002A31310581F6FF90EF90DF90CF90BF90B6
:10180000AF909F908F907F906F905F904F9018CF88
:101810008F929F92AF92BF92CF92DF92EF92FF9200
:1018200082E18093FC0986E08093FD0996E2909323
:10183000FF0991E09093020A9093030A8093010AB2
:1018400088ED90E4A0E0B0E0809393099093940930
:10185000A0939509B09396098CE19CE0A0E0B0E0DC
:101860008093970990939809A0939909B0939A0946
:10187000742F66275527442722E030E0ACE1CA2EBA
:10188000ACE0DA2EE12CF12CB8E38B2EB8E19B2EE4
:10189000A12CB12CC901880F991F880F991FFC0139
:1018A000ED56F64F77FF05C080829182A282B38207
:1018B00004C0C082D182E282F382F901EE0FFF1FE1
:1018C000EE0FFF1FE956F64FC082D182E282F3820B
:1018D000440F551F661F771F2E5F3F4F2231310582
:1018E000C9F68CE199E8A0E0B0E08093D709909325
:1018F000D809A093D909B093DA09FF90EF90DF904F
:10190000CF90BF90AF909F908F909ACE1F920F92E2
:101910000FB60F9211240BB60F922F933F934F9354
:101920005F936F937F938F939F93AF93BF93EF9347
:10193000FF939091FB098091FC09981316C01092B7
:10194000FB098091020A8F5F8093020A9091020A3C
:101950008091030A891740F481E08093020A809104
:10196000FE098F5F8093FE09FCDD9091FE09809156
:10197000FD0998130DC08091B0008F7D8093B00059
:1019800080916F008B7F80936F001092000A27C0B8
:101990008091B00085FF04C08091B0008F7D03C0AE
:1019A0008091B00080628093B000209184003091DB
:1019B0008500E091FB0981E08E0F8093FB0984E0B4
:1019C000E89FF0011124ED56F64F80819181A281AC
:1019D000B381820F931F90938B0080938A00FF91B5
:1019E000EF91BF91AF919F918F917F916F915F9197
:1019F0004F913F912F910F900BBE0F900FBE0F9004
:101A00001F9018950C94857B80917E13882319F084
:101A10000E94697B02C00E94857B90917E1381E0C9
:101A2000892780937E1308958091020B81110C9475
:101A300076950C947E950E9476958091D3068823A6
:101A400041F069E17BE18091D1069091D2060C943E
:101A5000305E08950E947E958091D3068823D1F050
:101A60002091B40F8091D1069091D206211107C028
:101A70002091B70F211103C06FEC7AE109C02091CA
:101A8000020B222319F06EE07BE102C06AEF7AE1DB
:101A90000C94305E08950C94744180918C128111E5
:101AA0000C945E410C9474410C945E410E94107B36
:101AB0008091CD069091CE06DC01ED91FC9106A0BF
:101AC000F7A1E02D19940E9495798091CD0690910F
:101AD000CE06DC01ED91FC9104A0F5A1E02D199456
:101AE0000F931F93CF93DF9300917C1310917D137D
:101AF000C0913806D0913906B801CE010E948C54AD
:101B0000882379F0B801CE010E94A45480913A064E
:101B100090913B06DC01ED91FC9102A0F3A1E02D38
:101B2000199500917A1310917B13C0913806D091CA
:101B30003906B801CE010E948C54882321F0B801E7
:101B4000CE010E94A45459988091D306882361F055
:101B500067EC7AE18091D1069091D206DF91CF9126
:101B60001F910F910C94305EDF91CF911F910F91D7
:101B70000895CF93DF93C0913806D09139066091D4
:101B80007C1370917D13CE010E948C54811129C069
:101B90004091781350E060E070E028E831E6CE0133
:101BA0000E94FB5490937D1380937C1380913A069E
:101BB00090913B06DC01ED91FC9100A0F1A1E02D9C
:101BC000199580915506882361F060917A13709180
:101BD0007B1380913806909139060E948C5488239B
:101BE00071F08091D3068823E9F06EEB7AE1809161
:101BF000D1069091D206DF91CF910C94305E0E9475
:101C0000CB612BEC31E644E650E060E070E080917F
